:080000000C94EF0D0C940000BC
:100008000C9400000C9400000C9400000C94000068
:100018000C9400000C94753B0C9400000C940000A8
:100028000C94A5150C9400000C9400000C9400008E
:100038000C9400000C9400000C9444150C940000DF
:100048000C9427380C9400000C9463380C9400002E
:100058000C9400000C9400000C9400000C94000018
:100068000C9400000C9400000C9400000C94000008
:100078000C94D1390C9400000C94143B0C9400009F
:100088000C940000000001000200040008001000A9
:100098002000400080000001000200040008001059
:1000A8000020004000800001020408102040800069
:1000B800E4024A0D80100000E8024A0D821F000089
:1000C800F2024A0D81030000FA024A0D01040200FF
:1000D80004034B0D010602000E034D0D01800000C4
:1000E8001A03540D020F000022034E0D020F0000E8
:1000F8002A03500D020FD0123203520D01100000D6
:100108003C03A20D011000004603530D000100003E
:100118004E03560D010801005803570D030801004E
:100128006603580D030700006E036E0D017F3F0044
:1001380078036D0D010500008203590D03040000CA
:100148008A036C0D01641E0096035A0D000100001D
:10015800A2035B0D00010000AE036B0D010200005D
:10016800BA035C0D00010000C8035D0D020F00001A
:10017800D4035F0D020FE703DE03A10D0163000046
:100188003C04A30D011000004604A40D0102020066
:10019800EA03610D03080100F003620D0308000083
:1001A800F603630D03080000FC03640D0308000058
:1001B8000204650D030800000804660D030800002A
:1001C8000E04670D0308000014046F0D040A2E00C6
:1001D8001C04790D040A2E002404830D040A2E0041
:1001E8002C048D0D040A2E003404970D040A2E00E9
:1001F80000000000FF0000004E0400025604040442
:100208005C04080762040C0562048C066804800913
:100218007004100B7804500C820440038A04140AFA
:10022800940418089C041C010000000200002A0025
:1002380054007F00800E563100810E563200820E27
:100248005633000031000B00312041424300003298
:10025800000B003220444546000033000B003320D9
:10026800474849000043000C00430000000000001C
:1002780034000B0034204A4B4C000035000B00358D
:10028800204D4E4F000036000B00362050515200D2
:100298000030000B003020202E202C0037000B00EF
:1002A8003720535455000038000B00382056575853
:1002B800000039000B003920595A2F00003D000A70
:1002C800004352000000000050726F64756B742088
:1002D8000000537061727465202000005F4944007B
:1002E8005F5273323332494400005F526F74617455
:1002F80065005F54617374656E5800005F546173E4
:1003080074656E5900005F44656661756C744B6571
:1003180079002A436F64653000002A436F646531B1
:1003280000002A436F64653200002A4D61784D6FE2
:1003380064756C005F4572774D6F64756C002A5464
:100348006973636845005F4D795465726D4E72003C
:100358005F4D61737465725465726D7300005F451B
:100368004D6F646500005F454372656457747200A1
:100378005F5273304D6F646500005F5634756E646C
:1003880035005F50756C736554696D6500005F4199
:10039800736B43726564697400005F53656E6444EF
:1003A8006562697400005F4372656469744D6F64C7
:1003B80065005F4372656469744D617374657200AA
:1003C8002A5461626C655374617274002A546162C4
:1003D8006C65456E64002A4669727374426F6E508C
:1003E80000002A4A6F6231002A4A6F6232002A4AA4
:1003F8006F6233002A4A6F6234002A4A6F623500FE
:100408002A4A6F6236002A4A6F6237005F45727265
:100418006F7231005F4572726F7232005F4572729F
:100428006F7233005F4572726F7234005F4572728B
:100438006F7235005F4672656967616265005F4B80
:100448006F6D6D61000054617374657200004C69D2
:10045800745A00004C656974540050756C73000040
:10046800546173742030000073657269656C6C00A8
:1004780073657269656C20320000546173742032B0
:10048800000054617374207061720000466F6C67DD
:10049800655400005377697463680000706F727464
:1004A800696F6E696572656E00002E666F6C6765B0
:1004B8000000506F7274696F6E656E2073696368AF
:1004C80065726E0000000F00E003EF0300780F78FC
:1004D800E07BEF7BF7BD1F00E007FF0700F81FF880
:1004E800E0FFFFFF00000000000000000000000027
:1004F80000000000000000000000000000000000F4
:1005080000000000070018C0202020204D904D90CA
:1005180040104010489047102020202018C00700A5
:100528000000000007001FC03FE03FE072707270DB
:100538007FF07FF0777078F03FE03FE01FC0070062
:100548000000000000000000000018C03DE03FE08F
:100558003FE03FE01FC00F800700020000000000DE
:1005680000000000000000000000020007000F80EB
:100578001FC03FE01FC00F800700020000000000FE
:10058800000000000000000007000F800F800F80AF
:1005980037607FF07FF07FF0326007000F80000047
:1005A80000000000000000000200020007000F80A9
:1005B8001FC03FE03FE03FE01AC007000F80000087
:1005C8000000000000000000000000000000000023
:1005D80006000F000F0006000000000000000000E9
:1005E80000000000FFF0FFF0FFF0FFF0FFF0FFF069
:1005F800F9F0F0F0F0F0F9F0FFF0FFF0FFF0FFF0A5
:10060800FFF0FFF0000000000000000006000900F5
:100618001080108010801080090006000000000083
:1006280000000000FFF0FFF0FFF0FFF0F9F0F6F037
:10063800EF70EF70EF70EF70F6F0F9F0FFF0FFF089
:10064800FFF0FFF000000000000001E000601EA0C5
:10065800332061806180618033001E00000000004B
:10066800000000000000000007800CC0186018603F
:1006780018600CC00780030003000FC003000300CC
:100688000000000002000300038003C002C002C093
:100698000280020002000E001E001E000C00000076
:1006A800000000000C000E000B0009800CC00E407A
:1006B8000B4009C038C07840784031C003C003C03F
:1006C8000180000000000200020027201FC018C09F
:1006D80030607070306018C01FC027200200020010
:1006E8000000000000000000100018001C001E00A0
:1006F8001F001F801F001E001C00180010000000B3
:1007080000000000000000000080018003800780D6
:100718000F801F800F800780038001800080000009
:10072800000000000000020007000F801FC0020048
:1007380002000200020002001FC00F800700020032
:1007480000000000000019801980198019801980A4
:100758001980198019801980198000001980198062
:100768000000000000001FE036C066C066C066C01A
:1007780036C01EC006C006C006C006C006C006C0F9
:100788000000000000001F8030C0300030001F80D3
:1007980030C030C01F8000C000C030C01F800000C3
:1007A8000000000000000000000000000000000041
:1007B800000000000000000000001FE01FE01FE034
:1007C80000000000020007000F801FC002000200A6
:1007D80002000200020002001FC00F800700020092
:1007E8001FC000000000020007000F801FC00200A9
:1007F80002000200020002000200020002000200E1
:1008080000000000000002000200020002000200D6
:1008180002000200020002001FC00F800700020051
:10082800000000000000000000000000010001803E
:1008380001C03FE001C0018001000000000000008D
:1008480000000000000000000000000004000C0090
:100858001C003FE01C000C00040000000000000029
:100868000000000000000000000000000000000080
:1008780000000000400040004000400040007FE0D1
:10088800000000000000000000000000088018C000
:1008980038E07FF038E018C0088000000000000051
:1008A800000000000000000000000000000002003E
:1008B80007000F801FC03FE07FF00000000000002D
:1008C80000000000000000000000000000007FF0B1
:1008D8003FE01FC00F80070002000000000000007A
:1008E8000000000000000000000000000000000000
:1008F80000000000000000000000000000000000F0
:1009080000000000060006000F000F000F000F0097
:100918000F000600060006000000000006000600A2
:10092800000000000000000019801980198019805B
:1009380000000000000000000000000000000000AF
:100948000000000000000660066006603FF00CC072
:100958000CC0198019807FC03300330033000000B9
:1009680000000000060006001F803FC03600360069
:100978003F801FC006C006C03FC01F80060006009B
:10098800000000000000000000103830387038E027
:1009980001C0038007000E001C0038E070E060E032
:1009A80000000000000007000D80198019801B005E
:1009B8000E001E003E00336033C031803BC01E6015
:1009C800000000000E000E000E00060006000C00DD
:1009D800000000000000000000000000000000000F
:1009E80000000000038006000E000C001C001C0024
:1009F8001C001C001C001C000C000E0006000380DC
:100A0800000000001C0006000700030003800380AC
:100A180003800380038003800300070006001C0096
:100A28000000000000000000000036C036C01F8033
:100A38000F003FC00F001F8036C036C00000000006
:100A48000000000000000000000000000600060092
:100A580006003FC03FC00600060006000000000078
:100A6800000000000000000000000000000000007E
:100A7800000000000000000000000E000E000E0044
:100A880006000C000000000000000000000000004C
:100A980000003FC03FC00000000000000000000050
:100AA800000000000000000000000000000000003E
:100AB800000000000000000000000E000E000E0004
:100AC80000000000000000100030007000E001C0CD
:100AD800038007000E001C00380070006000000052
:100AE800000000000F803FE03060607060F061B08F
:100AF800633066306C307830703030603FE00F80A3
:100B080000000000030007001F001F00030003008F
:100B18000300030003000300030003001FE01FE0BD
:100B2800000000001FC03FE070706030607000E09F
:100B380001C0038007000E001C0038007FF07FF022
:100B4800000000001FC03FE070706030003000708F
:100B58000FE00FC000600030603070703FE01FC0D1
:100B68000000000001C003C007C00EC01CC038C090
:100B780070C060C07FF07FF000C000C000C000C03F
:100B8800000000007FF07FF06000600060007FC020
:100B98003FE0007000300030603070703FE01FC0F0
:100BA8000000000003C007C00E001C003800300021
:100BB8007FC07FE070706030603070703FE01FC0B1
:100BC800000000007FF07FF00060006000C000C0FF
:100BD8000180018003000300060006000C000C00E1
:100BE800000000000F801FC038E03060306038E03F
:100BF8001FC03FE070706030603070703FE01FC011
:100C0800000000001FC03FE07070603060307070FE
:100C18003FF01FF0006000E001C003801F001E00CD
:100C28000000000000000000000000000E000E00A0
:100C38000E000000000000000E000E000E00000074
:100C48000000000000000000000000000E000E0080
:100C58000E000000000000000E000E000E0006004E
:100C680006000C0000C001C0038007000E001C0035
:100C7800380038001C000E000700038001C000C0C7
:100C880000000000000000000000000000003FE03D
:100C98003FE0000000003FE03FE0000000000000EF
:100CA80000000000300038001C000E000700038020
:100CB80001C001C0038007000E001C00380030008E
:100CC800000000001F803FC070E0606060E001C06D
:100CD8000380070006000600060000000600060064
:100CE800000000001FC03FE0306067B06FB06DB01B
:100CF8006DB06DB06DB06FE067C070003FC00FC0E1
:100D080000000000060006000F000F000F00198009
:100D18001980198030C03FC03FC06060606060606B
:100D2800000000007F007F8061C060C060C061C0BB
:100D38007F807FC060E06060606060E07FC07F802F
:100D4800000000000F801FC038E0306060006000C5
:100D58006000600060006000306038E01FC00F80F5
:100D6800000000007F007F8061C060C0606060603C
:100D7800606060606060606060C061C07F807F00AC
:100D8800000000007FE07FE060006000600060001D
:100D98007F807F8060006000600060007FE07FE00F
:100DA800000000007FE07FE06000600060006000FD
:100DB8007F807F80600060006000600060006000ED
:100DC800000000000FC01FE03860300060006000C5
:100DD80063E063E060606060306038601FE00FE0EF
:100DE800000000006060606060606060606060607B
:100DF8007FE07FE0606060606060606060606060AD
:100E0800000000001F801F80060006000600060084
:100E18000600060006000600060006001F801F8068
:100E2800000000000060006000600060006000607A
:100E38000060006000606060606070C03FC01F803C
:100E480000000000606060E061C0638067006E00C1
:100E58007C007C006E006700638061C060E06060B9
:100E6800000000006000600060006000600060003A
:100E78006000600060006000600060007FE07FE06C
:100E880000000000606070E070E079E079E06F6079
:100E98006F6066606660606060606060606060602F
:100EA8000000000060607060706078606C606C606A
:100EB800666066606360636061E060E060E0606097
:100EC800000000000F001F8039C030C06060606003
:100ED800606060606060606030C039C01F800F0073
:100EE800000000007F807FC060E06060606060603C
:100EF80060E07FC07F80600060006000600060008C
:100F0800000000000F001F8039C030C060606060C2
:100F1800606060606060636033C039C01FE00F606C
:100F2800000000007F807FC060E0606060606060FB
:100F380060E07FC07F806700638061C060E06060C0
:100F4800000000001F803FC070E06060600070001B
:100F58003F801FC000E00060606070E03FC01F80FD
:100F6800000000003FC03FC0060006000600060063
:100F78000600060006000600060006000600060039
:100F880000000000606060606060606060606060D9
:100F98006060606060606060606030C03FC01F80FB
:100FA8000000000060606060606030C030C030C029
:100FB8001980198019800F000F000F000600060025
:100FC8000000000060606060606060606060606099
:100FD8006060666066606F6079E070E070E0606035
:100FE800000000006060606030C030C019800F00F1
:100FF800060006000F00198030C030C060606060D5
:10100800000000006060606030C030C01980198046
:101018000F000F0006000600060006000600060086
:10102800000000007FE07FE000C000C001800300F6
:10103800060006000C001800300030007FE07FE05A
:1010480000000000666066600F000F000F00198046
:101058001980198030C03FC03FC060606060606028
:10106800000000006F605FA039C030C06060606041
:10107800606060606060606030C039C01F800F00D1
:101088000000000060606060000060606060606098
:101098006060606060606060606030C03FC01F80FA
:1010A800000000001F801F8018001800180018009A
:1010B8001800180018001800180018001F801F805A
:1010C8000000000000000000000000000000000018
:1010D8000000000000000000000000000000000008
:1010E8007FF07FF0000007000700070006000600F9
:1010F80003000000000000000000000000000000E5
:1011080000000000000000000000000000001FC0F8
:101118003FE000601FE03FE0606060607FE03FE02C
:1011280000000000600060006000600060006F80E8
:101138007FC070E060606060606060E07FC07F805A
:1011480000000000000000000000000000001F80F8
:101158003FC0706060006000600070603FC01F802A
:1011680000000000006000600060006000601F6018
:101178003FE071E060606060606070603FE01FE0C9
:1011880000000000000000000000000000001F80B8
:101198003FC070607FE07FC0600070003FC01F806C
:1011A8000000000007800F801C00180018001800BD
:1011B8007F007F0018001800180018001800180099
:1011C80000000000000000000000000000001FE018
:1011D8003FE07060606070E03FE01F60006000E02A
:1011E8003FC03F80600060006000600060006F00EA
:1011F8007F8071C060C060C060C060C060C060C0F7
:1012080000000000000000000600060000000E00BC
:101218000E00060006000600060006001F801F805C
:101228000000000000000000018001800000038031
:101238000380018001800180018001800180198084
:101248001F800F0030003000300030003000318047
:10125800338037003E003E003700338031C030C055
:10126800000000000E000E00060006000600060042
:101278000600060006000600060006001F801F8004
:10128800000000000000000000000000000059807D
:101298007FC07FE066606660666066606660666004
:1012A80000000000000000000000000000003F8077
:1012B8003FC030E0306030603060306030603060B7
:1012C80000000000000000000000000000001F8077
:1012D8003FC070E060606060606070E03FC01F8089
:1012E80000000000000000000000000000007F80F7
:1012F8007FC060E06060606070E07FC06F80600009
:1013080060006000000000000000000000001FE016
:101318003FE070606060606070E03FE01F60006008
:10132800006000600000000000000000000037C0FE
:101338003FE03860300030003000300030003000CE
:1013480000000000000000000000000000003F0056
:101358007F8060007F003F80018001807F803F00A8
:1013680000000000000018001800180018007F0096
:101378007F00180018001800180018001F800F8040
:101388000000000000000000000000000000606095
:101398006060606060606060606070E03FE01F6097
:1013A8000000000000000000000000000000606075
:1013B800606030C030C0198019800F000F0006002F
:1013C800000000000000000000000000000066604F
:1013D80066606660666066606F603FC039C0108096
:1013E800000000000000000000000000000060C0D5
:1013F80071C03B801F000E001F003B8071C060C0A1
:10140800000000000000000000000000000030C0E4
:1014180030C0198019800F000F00060006000C006C
:101428000C001800000000000000000000007FC051
:101438007F80030006000C00180030007FC07FC0CA
:1014480000000000000000006060000000001FC0F5
:101458003FE000601FE03FE0606060607FE03FE0E9
:1014680000000000000000006060000000001F8015
:101478003FC070E060606060606070E03FC01F80E7
:1014880000000000000000006060000000006060D4
:101498006060606060606060606070E03FE01F6096
:1014A8000000000000003F007F8060C060C061C095
:1014B800678067C060E06060606060E067C0678008
:1014C80000000000000000000000000006000F00FF
:1014D800198030C0606060607FE07FE0000000003D
:1014E80000000000436865662D4D656E75004B2051
:1014F8006C697374656E00004B206C6F657363686C
:10150800656E00004B20647275636B656E00542035
:101518006C697374656E000054206C6F6573636842
:10152800656E00005420647275636B656E005379B4
:101538007374656D0000506F7274696F6E004B7242
:101548006564697465004B7265642E436C720000B3
:101558006D616E2E506F7274696F6E00546573748E
:101568000000506172616D657465720050726F643D
:10157800756B746500004B656C6C6E657200566522
:101588006E74696C650030EC1431F6143200153352
:101598000C15341615352015362C15463615413ED2
:1015A80015434615444E154A5815000000003036BC
:1015B80015376415396A15387415427E1545861530
:1015C800000000004572726F72004F70742E0000A8
:1015D800496D70756C73000054696D656F757400A2
:1015E800CC15B80D00010000D215BB0D000300009A
:1015F800D815B90D00010000E015BA0D001400005F
:101608002E202C3041424331444546324748493325
:101618004A4B4C344D4E4F35505152365354553732
:1016280056575838595A2F390500C1110000030080
:10163800D90B00000300C1110300170E0300D90BDA
:1016480000000500E00800000A00C1110A00170E9A
:101658000A00D90B0A00C1110A00170E2800D90B7D
:1016680000000000F8000000FF000000FF0000007C
:101678007F80001E0F80007FE7C0007FFFE0003FF3
:10168800FFE00007FFC00001FFC00001FF8000016C
:10169800FF0003FFFE0007FFFC0007FFF00003FF49
:1016A800F00003FFFE00001FFFC001FFFFF001FF75
:1016B800FFF801FFFFF8007FFFF80007FE00003F7A
:1016C800FF00007FFF80007FFF80007FC100001FB8
:1016D800E000001FF000001FF000000FE00000070E
:1016E800C0000007C0000007C0000007800000031A
:1016F80000000003000000020000000000000000DD
:1017080000000000E000000000000003900000005E
:101718000000000E1800000000000038080000005B
:10172800000000C0180000000000038070000000E6
:1017380000000C01C0000001800630070000000313
:10174800C00F401C00000006E01DC0700000000C27
:101758003039C1C0000000181871C7180000001CFB
:101768000CE1DC7C0000000E07C3F1C40000000798
:101778000386070600000003800E1C02000000011B
:10178800C01C300300000000E03818010080000091
:1017980070700FC183C0000038E003E08E6006005F
:1017A8001DC00020FC200F000F8000307030198011
:1017B80007000010003030C00000001800E0606032
:1017C80000000008038060300000000C0E00301894
:1017D800000000043800180C00000006E0000C06A9
:1017E8000000000380000603000000000000030161
:1017F8008000000000000180C0000000000000C060
:10180800C000000000000060C000000000000030C0
:10181800C000000000000030C000000000000030E0
:10182800C000000000000030C000000000000030D0
:10183800C000000000000030C000000000000030C0
:10184800C000000000000030C000000000000030B0
:10185800C000000000000030E00000000000003080
:101868007000000000000030180000000000003088
:101878000C00000000000030040000000000003FE1
:10188800FC0000000000003FFC001027E803640093
:101898000A000100001000011000010054696E796F
:1018A8002062616400507772552000424F757420A1
:1018B8000057646F672000454570726F6D20006C9B
:1018C8007C736368656E203F0058006E65696E0022
:1018D8006A61003E3E006B65696E204B7265646903
:1018E8007400546573740020204B653A0020204929
:1018F8006E3A0043616C6962726174696F6E004F81
:101908004B00567320312E353500546F74616C20AE
:10191800002D2D2D2D006B65696E20454570726F69
:101928006D006E6F20546F75636800496E69746945
:10193800616C697A65640049442000454520363465
:101948006B00533F000066616C73636865722054D6
:10195800697363682000546973636820766F6E202A
:101968004B20004665686C6572200056656E746988
:101978006C20616B7469760054696D656F757400CD
:10198800435349204E722000436F646520006B6505
:10199800696E204B72656469740066616C73636874
:1019A80065722054697363680054697363682076AC
:1019B8006F6E204B005831393931303000504C555A
:1019C80020203A00436F6465203A005469736368C5
:1019D800203A004D42005053004D31004F31005322
:1019E800500043500044590062757379004D50000F
:1019F8002067657370657272740025640000256441
:101A08000025303258002E3030004F4E00004B2356
:101A180000425300422100424600542300544F0024
:101A28004952004D5A004251004252004353005659
:101A38005300564300494C00426600004B230054B3
:101A480023004245004345004241004453004342BD
:101A58000023502241534349492D492F4F222C221C
:101A6800312E3030222C323030382D30312D30317B
:101A78003B0023482245636F222C22312E3030222E
:101A88002C323030382D30312D30313B0023532269
:101A980045636F222C22312E3030222C32303038E0
:101AA8002D30312D30313B00504F00504632333B02
:101AB8005055002564002B302B303B004162726585
:101AC80063686E756E67004B656C6C6E657220009E
:101AD800546F74616C004D6F64756C200020200099
:101AE800433F0073656300496D7000504C553A20C0
:101AF800005370617274653A20005072313A2000C8
:101B08005072323A200046756E6374203A200054B1
:101B180079703A20003A20563A2020302B203000A5
:101B28003A003A20544F3A20003A2050733A2000A5
:101B380053703A004B204D6F6465204A6F62204A0B
:101B48006F62466C616773004B20004D6F646520BF
:101B5800004A6F62202000562020204572722050D3
:101B6800676C20496D7020544F00562000506175F5
:101B78007365004B656C6C6E65723A004D49004D9B
:101B880042004D43004D50004D4C00746573742065
:101B98002E2E004F4E002530325800253034580084
:101BA800253664002533642E2530326400253564DB
:101BB8000025640025326400253364004444000095
:101BC800206E616E6F0001002D4E414E0000010035
:101BD8006D10CE1B0000F894EE27ECBBF1E0F5BFCA
:101BE800E5BFE0936C00F8E1F1BDE1BD8DE0A2E056
:101BF800BB27ED938A95E9F780E090E1A0E0B1E09A
:101C0800ED930197E9F7E6EDFBE185919591009752
:101C180061F0A591B59105901590BF01F00105906F
:101C28000D920197E1F7FB01F0CFEFEFEDBFE0E197
:101C3800EEBFC0E0D5E00C9413170A9902C0E1E0AA
:101C48000895E0E0089508950895E881E03011F0DE
:101C58001D9801C01D9A1BC40E94326B0E94326BF2
:101C68000E94376B0E943C6B0E94416B08950E9452
:101C7800456B0E944B6B19F50E94516B0E94326BA9
:101C88000E94566BE1E2EA930E94326B0E94326B2B
:101C98000E945F6B0E943C6B0E94566B0E94626BB5
:101CA8000E94326B0E945F6B0E94656B0E946A6B98
:101CB8000E94326B0E945564EBE9F0E022C00E945A
:101CC8006D6B0E94326B0E94566BE1E2EA930E94B0
:101CD800326B0E94326B0E94726B0E943C6B0E94B6
:101CE800566B0E94626B0E94326B0E94726B0E945C
:101CF800656B0E946A6B0E94326B0E945564E1EF2B
:101D0800FFEFFA93EA930E94756B0E947A6B0E9428
:101D1800326B0E94556408951A93E0E0E0930B0635
:101D280010E0133000F50E947D6B3196049000920C
:101D38000A060E94836BE2E3F0E00E94C4793496BD
:101D48000E94866BEEE2F0E00E948D6B0E947D6B34
:101D5800E491EA930E947D6B32960E94946B0E94F4
:101D680055641F5FDECFE0910B06E0930A060E94E0
:101D7800976B3EC30E94487C0E9492510E949B6BC5
:101D8800ECE00E94A16BE8E7F0E00E94A76B0E94DC
:101D98008D6B0E94AC6BE1E2EA93E1EDF8E10E9401
:101DA800946B0E945564EBE00E94A16BE4E0F0E0C4
:101DB8000E94A76BFA93EA93EEE6F0E00E94B16BFB
:101DC800E091C30DF091C40DE491EA93E091C30D45
:101DD800F091C40D31960E94737A0E94946B0E9410
:101DE800556431E00E94B46B0E94B76B11F03F5FFD
:101DF800F9CF0E94C56B301718F4E0E0E093BB07F9
:101E08000E94C56B11E00E94CD6B0E94B76B11F068
:101E1800143008F023C00E94D06B0E94836BE0E26C
:101E2800F0E00E94C4793496FA93EA930E94D56B45
:101E3800EAE1F0E00E94DA6B0E94DD6BE491EA933C
:101E48000E94CD6B0E94DD6B31960E94737A0E94CE
:101E5800946B0E9455640F5F1F5FD5CF0E94976BEC
:101E68000E944F7C26C327970E94487C30E00E943E
:101E78009B6B0E94456B10E0133010F00C948C0F94
:101E880000E0043010F00C948A0F0E94E96B32963F
:101E9800049000920A06E0E0E0930B06FE013496F7
:101EA800FA93EA930E94E96B3496FA93EA930E94B4
:101EB800B968EB85E03039F4AD81A13210F4E0E087
:101EC800ED83E0E0EE83A02FB0E0E8E2F0E00E94CE
:101ED800C4793296FA93EA930E94836BE0E2F0E0C9
:101EE8000E94C479B096FA93EA93E4E2F0E00E9483
:101EF800B16B0E94E96BE491EA930E94326B0E94F5
:101F0800EF6B0E9455643F5F0F5FBBCF1F5FB4CF7D
:101F18000E9407544BC40E94467C0E94326B0E9468
:101F2800326B0E946D513091A7090E94F46B0E9498
:101F38009B6B10E0E0914B0D1E17E8F400E0E09178
:101F48004A0D0E17B0F40E94016C81F00E94086CD3
:101F58000E94146C519FF0010E941E6C0E94236C19
:101F68000E94316C3A934A930E94DA203F5F0F5FD8
:101F7800E6CF1F5FDFCF0E94976B0E944D7CD7C1D1
:101F880022970E94467CEBEDF8E0EE83FF8340E069
:101F9800443190F4AE81BF8111960E94396C13963A
:101FA800EFEFEC93AE81BF81EC93EE81FF81349625
:101FB800EE83FF834F5FECCF0E94F46B3091A7094B
:101FC8000E943E6C10E0E0914B0D1E17B8F500E042
:101FD800E0914A0D0E1780F50E94016C51F1A09115
:101FE800230DE0E8EA23E03819F40E94086C06C0E3
:101FF800E7E0E0930B06E8E0E0930A060E94146C21
:102008000E94456C0E94836B0E94C4793396FA93B0
:10201800EA930E94236C0E94316CA091A709E32FD8
:102028000E94486CEA0FFB1F43833A934A930E942D
:10203800DA203F5F0F5FCCCF1F5FC5CFE0910B0663
:10204800E0930A060E944B6B41F50E944F6C71F4B5
:102058000E94516B0E94326B0E94566BEFE7EA9325
:102068000E94326B0E94326B0E9455640E94516B31
:102078000E943C6B0E94566B0E94626B0E94326BFE
:102088000E945F6B0E94656B0E946A6B0E94326BB4
:102098000E945564EBE9F0E027C00E944F6C71F490
:1020A8000E946D6B0E94326B0E94566BEFE7EA93B9
:1020B8000E94326B0E94326B0E9455640E946D6BC5
:1020C8000E943C6B0E94566B0E94626B0E94326BAE
:1020D8000E94726B0E94656B0E946A6B0E94326B51
:1020E8000E945564E1EFFFEFFA93EA930E94756B43
:1020F8000E947A6B0E94326B0E9455640E940754BA
:102108000E94FE360E944D7C289608950E943E6CDF
:10211800E0E0E0930B06ECE0E0930A060E94D06B47
:102128000E94546CE1E2EA93E3EDF8E10E94946BBB
:102138000E945564EAE0E0930A06E2E5F0E0FA93CB
:10214800EA930E94546CEDE3EA93E8EDF8E10E940B
:10215800946B0E9455640E94075408951A93A981AC
:10216800A23019F40E944F6C09F024C00E94616CDF
:102178000E94646CBF01E9810E946B6C0E94756CBF
:102188001E2FEFE00E94A16BE7E8F0E0FA93EA93D4
:10219800EB810E946B6C32960E947E6C0E94856C6B
:1021A800FA93EA93EFE7EA93EBEDF8E10E94946B78
:1021B8000E9455641DC10E949251E0E0E0930B0615
:1021C800A881A13051F40E94886C0E948D6C0E94F5
:1021D8006D51EEEDF8E10E94926C0E944F6C69F42B
:1021E800E2E0EA93BBDFE8E3F2E00E94966CEAE300
:1021F800F2E00E94966C0E94215439DD48C1E881C2
:102208000E946B6CFA93EA930E949B6C0E94646C28
:10221800FA93EA930E94C351E881EA939FDF37C19A
:102228001A930A93EC81EA93EADF1BE90E949E6CF9
:102238000E94646CBF01EC810E946B6C0E94756CFB
:102248000E2FAC81A43019F40E944F6C09F009C01C
:1022580012E8AA81BB811B96E0E0EC93EC81EA933B
:102268007DDF0E94086CEC810E94A16CFF93EF93C4
:102278000E948D6CEE810E946B6C31960E94A76C57
:102288000E94DA6BFA93EA93EC85E058EA930E948D
:10229800326BED85FE85FA93EA930E945564AF91FF
:1022A800BF91EC93EC810E946B6CFA93EA93EE81F8
:1022B800F0E00E94646CFA93EA930E9421540C9413
:1022C8000815E5C01A930A93E0914B0DAFE70E94F9
:1022D800CE790E2F11270E94326B0E94326B0E941A
:1022E800376B1A930A930E94416B0E94886C0E9474
:1022F800886C0E946D51EC81FD810E94926CAA81CC
:10230800BB81A030E0E8BE0731F0EA81FB81FA9397
:10231800EA930E94F7610E94AA6C0E94C4630E941B
:10232800326B1A930A930E942154198108812696C8
:1023380008950E944C68E0E0E0930A06E0930A06DC
:102348000E944B6B19F4E1E9F0E002C0E1EFFFEF06
:10235800FA93EA93E0E6F0E00E94B16B0E94AC6B5E
:102368000E947A6B0E94326B0E94556408951A93FA
:1023780011E00E94DA220E94AF6C0E94B46CB897F8
:102388000CF414E00E94326B0E94856C0E94BA6CB7
:10239800E9810E94C06C0E94CC6C0E94BA6C0E94B9
:1023A800D06C0E94D56CE981EA930E948122E9836E
:1023B800ACEAB8E00E94616C0E94D96C3B9754F07B
:1023C800ACEAB8E00E94616C0E94D96C0E94E06C93
:1023D800E9E40BC0ACE6B8E00E94616C0E94D96CDD
:1023E8000E94E46C0E94DF61E3E7EA930E940051D7
:1023F8001881229608950E94326B0E94326B0E94C7
:102408006D51EAEEF8E10E94926C0E94326B0E94D4
:10241800E96C0E94376BECE3F0E00E94EE6C0E94DE
:10242800326B0E94886C0E946D51E09116080E94E0
:10243800F16CEFEEF8E10E94926CE091B909EA9331
:102448000E9409620E94326B0E94F36CE0912D0891
:102458000E94F16C0E94326B0E948D6C0E946D513B
:10246800E09144080E94F16CE5EFF8E10E94926C5B
:10247800E0910B08EA930E9409620895E881E064FC
:10248800E7B9369A349BFECF349AE4B1F5B1219678
:102498000895E881F981AA81BB81AE17BF071CF4B2
:1024A800EA1BFB0B06C0A881B981EA81FB81EA1B04
:1024B800FB0B2496089528970E94487CEFE0E09350
:1024C80061000E944B6B11F4E1E001C0E4E4E09389
:1024D800620085E88A95F1F7E5E0E093610085E818
:1024E8008A95F1F70E94F66CE0936A07F0936B0700
:1024F800E0917607F0917707E0936807F093690712
:10250800E1E0EA93BBDFE0937607F0937707EFE02B
:10251800E09361000E944B6B11F4E2E001C0E8E037
:10252800E093620085E88A95F1F7EAE0E0936100BC
:1025380085E88A95F1F70E94FB6CE0936607F093B3
:102548006707E0917407F0917507E0936407F093CB
:102558006507E0E0EA9392DFE0937407F09375076C
:102568000E94FB6CA0916607B0916707EA0FFB1FFA
:10257800A0917407B09175070E94006D8F010E94A9
:10258800F66CA0916A07B0916B07EA0FFB1FA09148
:102598007607B09177070E94006D9F01E09166076A
:1025A800F09167070E94076DFF93EF930E94FB6C01
:1025B8000E94076DAF91BF91EA0FFB1FFF93EF9346
:1025C800E0917407F09175070E94076DAF91BF9174
:1025D800EA0FFB1FE0937007F0937107E0916A0719
:1025E800F0916B070E940D6DFF93EF930E94F66CBC
:1025F8000E940D6DAF91BF91EA0FFB1FFF93EF9300
:10260800E0917607F09177070E940D6DAF91BF9129
:10261800EA0FFB1FE0937207F0937307A09170070E
:10262800B0917107E4E1F0E00E9496790E2EA09136
:102638007207B0917307E4E1F0E00E949679E0290F
:1026480019F00E940966B2C000936C0710936D07D9
:1026580020936E0730936F07A0915F07A23328F489
:10266800E0915F07EF5FE0935F070E94136D989713
:1026780024F40E94186D98970CF00EC0A0915F0783
:10268800AA3019F4E1E0E0935C07A0915F07A83253
:1026980019F4E2E0E0935C070E94136DAB35E0E0CB
:1026A800BE0734F00E94186DAB35E0E0BE070CF4AD
:1026B8007DC0E0916207EF5FE09362070E941D6DA5
:1026C8000E94136D0E94226DE887F9876A877B87CD
:1026D800A885B9858A859B85E0EAF0E060E070E02E
:1026E8000E94C9797F936F93FF93EF930E94296D9E
:1026F8000F010E941D6DDF01F001EA1BFB0BAF917A
:10270800BF918F919F910E942E6DE887F9876A8704
:102718007B870E94336D0E94186D0E94226D0E9473
:10272800386DE0E8F0E060E070E00E94C9797F93DE
:102738006F93FF93EF930E94416D0F010E94336DD9
:10274800DF01F001EA1BFB0BAF91BF918F919F91C5
:102758000E942E6D0E94386D0E94407C64F4AC810A
:10276800BD818E819F81A038E0E0BE07E0E08E0742
:10277800E0E09E070CF01AC0E885F985E09354075D
:10278800F0935507EC81FD81E0935607F0935707C6
:10279800E0915407F0915507FA93EA93E0915607B0
:1027A800F0915707FA93EA930E9494650E944F7C30
:1027B8002C9608950E949251EAE0F0E00E947E6C07
:1027C8000E948651EBEFF8E10E94926CE4E1EA93F3
:1027D8000E946E610E94466DE4E1EA930E946E6178
:1027E800A0916207A13010F0A895FACF0E94326B31
:1027F8000E944C6D0E9486510E94516DEBE10E942F
:10280800576DA0916207AF3110F4A895FACF0E94D6
:102818005B6DA0E0B0E00E949E7A0E94326B0E943D
:102828004C6D0E94646D0E94326B0E946B6D0E9419
:1028380086510E941D6D0E94E06CA0916207AE3126
:1028480010F0A895FACF0E94516D0E94706D0E94F9
:102858008651EAE10E94576DA0916207AF3110F4EA
:10286800A895FACF0E945B6DA2E0B0E00E949E7A24
:102878000E94706D0E94646D0E946B6D0E946B6D6A
:102888000E9486510E94296D0E94E06CA091620707
:10289800AE3110F0A895FACFE2E0E0930806E6E43E
:1028A800F0E00E94946B0E948651E8E1EA930E944E
:1028B8000051E1E0E0930806A0916207AF3110F4FF
:1028C800A895FACF0E94756DA4E0B0E00E949E7AA8
:1028D800E6E4F0E00E94946BE8E1F0E00E947E6C90
:1028E8000E94416B0E947E6D0E94836D0E948651FA
:1028F8000E94336D0E94E06CA0916207AE3110F027
:10290800A895FACF0E94516D0E946B6DEFE5F0E03B
:102918000E94886DE9E10E94576DA0916207AF316E
:1029280010F4A895FACF0E94756DA6E0B0E00E9459
:102938009E7A0E946B6DEFE5F0E0FA93EA93E8E186
:10294800F0E00E94B16B0E94416BE8E2F0E00E9467
:10295800866B0E9486510E94416D0E94E06CA09196
:102968006207AE3110F0A895FACFE2E8F0E00E94D5
:102978008C6D0E948651E7E0F9E10E94926C0E94FA
:102988008F6DA8950E948F6DA8950E949251089509
:102998001A930A93AC810E94956DEA81E030A1F107
:1029A8000E949D6D1081EA81AC81EA2351F01038B4
:1029B80010F0103B08F001C01F5F103808F410E851
:1029C80019C0103208F41F5F103189F4A091A209D0
:1029D800A23031F0A83021F0A13011F0A53039F43F
:1029E800EB81E058EA93E7E0EA930E949463103B96
:1029F80008F010E00E949D6D1083EA81EE0FEA83D3
:102A0800EB81EF5FEB83C9CF198108812596089583
:102A18001A93A9810E94956D1091CA0DA981AF3FA3
:102A280021F0E091C90DEA1751F0103810F0103B71
:102A380008F001C01F5F103808F410E81BC01032FE
:102A480008F41F5F103199F4A091A209A23031F067
:102A5800A83021F0A13011F0A53049F4A981EFEF99
:102A6800EA27E158EA93E7E0EA930E949463103B6F
:102A780008F010E0E981E093C90D1093CA0DCCC1AC
:102A88000E94A26DE2EBE2BF7894ABEEBCE00E943C
:102A9800B16D0E945765442009F40DDDA091590DD0
:102AA800A27039F0E6B3EA93E0E0EA93E1E0EA9352
:102AB8006FDFA091590DA47019F0E6B3EA93A8DF6F
:102AC8000E94F122A0919D09B0919E09E6E0F0E0F4
:102AD800AE27BF27E7E0F0E0EA231E2FA091590DAB
:102AE800A870B1F0A091A209A23091F4E0915D0D17
:102AF800F0915E0DA091AF09B091B009AE17BF0774
:102B08003CF0E0915F0DF091600DEA17FB070CF4C3
:102B180001C01160E2B3EF78AE2FE12FE295E07FBC
:102B2800EA2BE2BB0E9448407394EEE1E71539F4C2
:102B3800A0910506E3E8EA27E093050677241991B2
:102B480009C00E94A26D0A93E3E8E4BD0E942240F6
:102B580009911991E991EFBFF991E991B991A99179
:102B68009991899179916991F9901990099018959D
:102B7800E8EFFFEF4F010E9492510E944C680E94BB
:102B8800886C0E94F36CEAE0F9E10E94926C0E9462
:102B98005B680E94B76D0E94497908950E94D33FEF
:102BA8000E944D3F0E9474430E941A2008951A9370
:102BB800A8950E947563E13011F00C943916E091E4
:102BC800C107E1501E2FA091C007A13021F40E9437
:102BD800BC6DE03009F40CC0ADE01A9FF001E65F6F
:102BE800FA4FBF01E081E260DB01EC930E94C36D04
:102BF800A091C007A23011F0A430E9F40E94BC6D86
:102C0800E093D6070E94C86D31F0FD01E65FFA4FE8
:102C1800E081E27009F403C01A930E94D16DA0917B
:102C2800590DA67021F0A091D607A03808F403C06A
:102C3800E0E0E093D607A091C007A33019F41A93F7
:102C48000E94A528A091C007A53029F4E091C107EA
:102C5800EA930E94D528A091C007A73031F4E091EB
:102C6800C107E093D6070E949061E0910506E078DD
:102C7800B9F0E0910506EF77E09305060E94475406
:102C8800E0910506E07131F0E0910506E270EA9303
:102C98000E946C50E0910506E170EA930E94290EAB
:102CA800A091590DA67039F4E6B3AFEFAE27EFE364
:102CB800EA23E093B90972DF4EC01A930E94925139
:102CC800E1E0F0E00E94946B0E946D5110E00E94D8
:102CD8009B6B0E94326B0E94856C0E94D56CE091C0
:102CE800A909E03049F4E2E1F9E10E94926C0E94FE
:102CF800D56D0E94C9611E5FA091A909A130F0F0AD
:102D0800E091A909E150EA930E94221AA0913C0D92
:102D1800AD3229F40E94E06D0E94387C79F00E945F
:102D2800ED6D0E94F26D0E94D06C0E94D56C0E94DD
:102D3800E06D0E94777A0E94C9611E5FE091A9093F
:102D4800EF5FE093A909163020F4A091A909AB30F0
:102D580008F001C0BECF199108951A930E949251AC
:102D6800E981E03019F4E0E0E093A709A981A230F5
:102D7800A9F410E0A091A709A13010F0163008F0CE
:102D88000DC0E091A709E150E093A7090E94F66DF4
:102D980019F40E94046E09F01F5FECCF0E949B6B30
:102DA80010E00E94326B0E94856C0E94D56CA09145
:102DB800A709A03410F50E94F66D19F40E94046E5C
:102DC800C9F0E091A7090E94C06C0E94CC6C0E94D7
:102DD800D56C0E940F6E0E94E06CE8E7EA930E94AF
:102DE80000510E94146E0E94186E0E94777A0E9409
:102DF800C9611E5F0E94216E07C0E9E1F9E10E94E6
:102E0800926C0E94216E1E5F163020F4A091A709D3
:102E1800A23408F001C0C5CF18812296089514B7CE
:102E2800E0E0E4BFE5BFE0936D00E0936C00EBBB2E
:102E3800EFEFEABBE0E0E8BBE7BBE5BBEFEFE4BBE5
:102E4800E0E6E2BBE0E7E1BBE0E3E3B9E8EBE2B9E7
:102E5800E0E0E0936200E0936100E0936500EFE05A
:102E6800E0936400E0E0E0BFE7E0E3BFE2EBE2BF4D
:102E7800E0E0E1BFEFBDEEBDEDBDECBDE7BDE6BDF9
:102E8800EBBDEABDE9BDE8BDE0937900E0937800C9
:102E9800E3E0E5BDE3E8E4BDE0E0E3BDE0938B00FB
:102EA800EAE0E0938A00E0E0E0938900E09388009C
:102EB800E0938100E0938000E2E1E0938700E4E39F
:102EC800E0938600E0E0E0938500E0938400E093DF
:102ED8008300E0938200E0936A00E0E3EABFE0E465
:102EE800E9BFE8BFE1E4E7BFE0E0E0937D00EBB9CC
:102EF800E8EDEAB9E6E0E0939500E0E0E0939000C1
:102F0800E3E3E9B9E0E0E0939B00E8EDE0939A00A1
:102F1800E6E0E0939D00E0E0E0939800E9E1E093CB
:102F28009900E0E8E8B9E0E0E0BDE0E4E7B9E7E807
:102F3800E6B9E0B5EF7EE0BDE0E1E0937000E0E0E7
:102F4800E0937200E4E4E0937400EEE1E1BDEEE0AA
:102F5800E1BD0E9402550E942C6610FF03C0AAE042
:102F6800B0E00CC012FF06C0ABE0B0E00E94927A5D
:102F78000E94276E13FF06C0ACE0B0E00E94927A70
:102F88000E94276E0E94316EEE59F64F10830E9400
:102F9800316EED59F64FA9E00E94376EE9DD0E94C7
:102FA800886C0E943E6E0E945A50E4E0E0936100F3
:102FB800EFE0E0936200000000000000E0B1E17083
:102FC800E13011F0E1E04E2EEBE0E093620000000A
:102FD80000000000009B02C0E1E04E2EE8E0E09314
:102FE8006100EFE0E0936200000000000000E0B143
:102FF800E270E23011F0E1E04E2EE7E0E09362008B
:10300800000000000000019B02C0E1E04E2E0E947B
:103018000119E030D1F40E94886C0E943E6EEEE106
:10302800F9E10E94926CA8950E94416E0E94466E3A
:103038000E94836D0E9449790E94416E0E94466EEB
:10304800ECE2F1E00E944C6EEECF0E94E9377894F2
:10305800442021F0EAE2F9E10E94926CE0E0E415F4
:1030680089F40E941D6D0F010E94296D0E161F061E
:1030780044F40E94336D0F010E94416D0E161F0625
:103088000CF001C002C00E94DE130E94971CE030C1
:10309800B9F00E94506E0E94D56CE3E3F9E10E94FA
:1030A800926C0E94AA6C0E944979A8950E94AA6C09
:1030B8000E944979A8950E94AA6C0E944979A8950E
:1030C8000E94536EE53128F0A9E0B0E0E0E00E94EC
:1030D800A67A0E94506E0E94D56CEFE3F9E10E9437
:1030E800926C0E94536EEA930E9409620E94886C57
:1030F8000E943E6EE3E4F9E10E94926C4420B1F430
:10310800BB24E0E5BE1638F4EAE0F0E00E944C6E1D
:10311800A895B394F6CFE0E5BE1620F0A09162071B
:10312800AF3108F402C00E94DE132EC0BB240E94F7
:10313800536EBE1658F4A8950E94586E0E94466EAB
:103148000E94D56B0E944979B394F1CFA8950E944B
:10315800466DBB240E945D6EBE1658F4A8950E9469
:10316800586E0E94466E0E94D56B0E944979B394AE
:10317800F1CFA8950E94466DA8950E94466DE091F2
:103188000506EF77E09305060E945A400E94DB157A
:103198000E945B330E94D11EF9CFFFCF0E94626E5E
:1031A8000E94666E17FD02C0103011F4E0E076C38D
:1031B800E12F74C30E94626E0E94666E17FD10E0D4
:1031C8001A3008F41F5FE0EAEA930E949B6C0E94A1
:1031D8006E6E64C30E94626E0E94666E17FD02C026
:1031E800103011F4E0E05AC31150E0EAEA930E946B
:1031F8009B6C0E946E6EE1E051C31A930A9310E033
:103208000E94AA6C0E944979A8950E944A66E030FB
:1032180021F4E0EA0E94756E09F002C001E001C0E5
:1032280000E00E945B661F5F003011F4153008F063
:1032380001C0E6CFE02F0991199108950E947A6E96
:1032480058C40E947A6E0E94876E0895A881B98139
:103258000E943C7C24F4A83EE3E0BE070CF005C0C5
:103268000E948D6E0E94BD661AC3E0E018C3EA8111
:10327800E03011F4EFEFEA83A881B9810E943C7C29
:1032880024F4A83EE3E0BE070CF006C00E948D6E51
:10329800ED81EA930E94EB666CC10E94487C20E0B5
:1032A80030E0283EE3E03E077CF4A8953A932A9361
:1032B800CDDF1E2F1F3F29F0EFEFEA933A932A93B1
:1032C800D6DF2F5F3F4FEDCF0E944F7C4BC01A9344
:1032D8000A93E0E0F0E0E093D10DF093D20DAA81DB
:1032E800A03468F40E949B6C0E94966EE55FFB4FC9
:1032F8008F010E949B6EE1EDFDE00E94A46EE091BB
:10330800D10DF091D20D33C11A931FEF1F5F1A939D
:10331800DEDFA981BA81EA17FB0711F0113408F042
:1033280001C0F4CFE12F188124C11A930A930E9497
:10333800A86EA091A709EA0F0E2F013408F00FE339
:103348001091A709101758F41A93C1DFAA81BB81FD
:10335800EA17FB0711F4E12F03C01F5FF3CFEFEF6C
:1033680019810881249608950E94467C10E0103443
:1033780018F50E94836BE8E2F0E00E94C479E050FF
:10338800FC4FAF01E0EAEA93FA0170960E94AF6E33
:10339800EC713E2FE0EAEA93FA013F960E94AF6E85
:1033A8000E2FEF81E31719F4EE81E01709F002C040
:1033B800E12F03C01F5FDBCFEFEF0E944D7C289603
:1033C80008951A930A93E091120DAA81EA1701F160
:1033D800A034A8F40E949B6C0E94966EE050FC4FAB
:1033E8008F01E0EAEA930E947E6D1A930A93E3E163
:1033F800FDE00E94A46EEA81E093120D09C0EFEF90
:10340800E093120D0E94B36E0E94B86EE0931D0DFA
:10341800AEC00E94C26E0E94966EE050FC4F8F01B3
:10342800AA81A03450F4E0EAEA930E947E6D1A93D0
:103438000A93E3E1FDE00E94876E99C01A930A930C
:10344800E0913B0DAA81EA17B1F00E949B6C0E94A3
:10345800C56E40F40E94CF6E0E94A46EEA81E0938C
:103468003B0D09C0EFEFE0933B0D0E94ED6D0E940C
:10347800B86EE093460D7BC00E94C26E0E94C56E76
:1034880020F40E94CF6E0E94876E71C01A930A932F
:10349800E091BC0DAA81EA1761F10E949B6C0E9421
:1034A800DA6E08F50E949B6EEDEBFDE00E94A46EBB
:1034B800EA81E093BC0DE0E0E0931008A091BE0D16
:1034C800A13020F0A091BE0DA83008F00BC0A1E6F5
:1034D800BDE0E091BE0D0E94E26EAE0FBF1FEC9101
:1034E800E093100806C0EFEFE093BC0DE0E0E09336
:1034F800BD0D3DC00E94C26E0E94DA6E30F40E947B
:103508009B6EEDEBFDE00E94876E31C01A930A9323
:10351800E091B70DAA81EA17D1F00E949B6C0E9436
:10352800E56E70F4E0EAEA930E94D06B1A930A936E
:10353800E8EBFDE00E94A46EEA81E093B70D07C0B6
:10354800EFEFE093B70D0E94ED6E0E948E680FC0FA
:103558000E94C26E0E94E56E50F4E0EAEA930E946F
:10356800D06B1A930A93E8EBFDE00E94876E1981ED
:103578000881239608950E94ED6E0E948E68E88166
:10358800EF5FE093B90DCDC124970E94467C0E945D
:10359800F46EAA85A03458F5AB85A13010F0A6309A
:1035A80008F005C0EB850E94E26E0E94006FEB8573
:1035B800E030E9F4E0E0EE83EF83E887E98740E074
:1035C80050E020E030E02530E0E03E0774F4F901F7
:1035D8000E94006F0E940F6E4E0F5F1F0E94186EB0
:1035E8000E941B6F2F5F3F4FEECF0E94266F42C194
:1035F8001A930A93AB81A13010F0A63008F01DC0D1
:10360800EB810E94E26E0E9476790E947279DF0156
:103618000E949B6CAE0FBF1FE8E0F0E00E94C479E7
:10362800E050FA4E8F01E0EAEA930E94376F1A934E
:103638000A93E5EAFDE00E94876E198108810C94DF
:1036480018200E94487CEC810E943C6FE83109F404
:103658005BC00E94416F309729F00E94416F0E9421
:10366800466FEC830E94FC200E2F10E0101710F01C
:103678000C94881B0E944A6F87DFA7EABDE00E946E
:10368800B16DA091A90DB091AA0D8091AB0D90914B
:10369800AC0D0E944F6F0E945979E093A90DF093E9
:1036A800AA0D6093AB0D7093AC0D0E944A6FA0DF1A
:1036B800E0EAEA93EE810E94E26EEE0FFF1FE0500F
:1036C800F04F0E94AF6EE270E9F4ED81E093AD0D2A
:1036D8000E94416F309761F40E94536E0E94566FAA
:1036E800EF5EF84DDF010E949E6CEA0FFB1F02C0DF
:1036F8000E94416FE093AE0DF093AF0D0E945C6F96
:103708000E94616F1F5FB2CF0E944F7C269608957A
:103718001A930A930E94676FECE2F0E00E946E6FC2
:103728000E94726F0E94776F10E01034D8F41A93D9
:1037380048DEE091AA09EA931A9326DF0E94806F77
:10374800EA0FFB1F0F010E94806F0E94886FDF0144
:10375800CB010E94186E0E945979D0010E946E7A9E
:103768001F5FE3CFA091A209A330B9F500E00031B3
:10377800A0F50E94CD6B0E948D6F69F510E01A309C
:1037880050F5E02FE05DEA93EAE4F9E10E94926FD8
:10379800E12FE05D0E94996FE1F40E949E6F0E9404
:1037A800A56FEA0FFB1FFF93EF930E94A56F0E947E
:1037B800886F7F936F93FF93EF930E944C3CAF9178
:1037C800BF918F919F910E945979AF91BF910E94AB
:1037D8006E7A1F5FD4CF0F5FCACF10E01A3090F413
:1037E8000E94A56F0E94886FA091B109B091B2099B
:1037F8008091B3099091B4090E9459790E94776F1A
:103808001F5FECCF0C945E2024970E94467CEA85CB
:10381800EA935DDD9F01022E032A39F13A932A9338
:1038280073DD1E2F40E050E0E0E0EE83EF83E88791
:10383800E987AA851A17B1F4012F003498F40A937E
:1038480046DD2E173F0761F4EB85EA930A939CDE69
:103858000E940F6E4E0F5F1F0E94186E0E941B6F12
:103868000F5FEBCF0E94266F05C0EB85EA93EB85CF
:10387800EA938ADE0E944D7C2C9608951A93A895A7
:10388800A981A63058F40E94F46E10E0103430F488
:10389800E981EA931A93ACDE1F5FF8CF188122966C
:1038A80008951A9311E0163020F41A93E7DF1F5F8A
:1038B800FACF74C3E1E0E093BD0DE093BE0D31C0D3
:1038C800A8950E94ED6DEAEDF2E0FA93EA930E9462
:1038D800376F0E94AC6FE093440D0E94B56FE09380
:1038E800450DE0E0E093460D1CC0A895E2E1FDE03F
:1038F8000E94BC6FE9E2F0E00E946E6F0E94B36E16
:10390800E0EDF2E0FA93EA930E94376F0E94AC6F01
:10391800E0931B0D0E94B56FE0931C0DE0EBE09364
:10392800210D219608950E94467C0E945D6EE0322A
:1039380028F0AEE0B0E0E0E00E94A67A00E07EDC8D
:10394800A091470DB091480DA633E2E1BE0741F1C1
:1039580010E01A3030F41A93B3DF1A938DDD1F5F2D
:10396800F8CF10E0103430F41A93BFDF1A9351DD0A
:103978001F5FF8CF10E0103830F41A939BDF1A93CA
:10398800B9DD1F5FF8CF8DDFA9E0B0E0E0E00E946D
:10399800A67AE6E3F2E1E093470DF093480D01E0E3
:1039A80010E0183210F00C943C1D0E94856C0E94A7
:1039B800C16F9F010E94856C0E94C16FAF010E9478
:1039C800856C0E94C96F3496E491E03011F0E130C3
:1039D80089F4D901AC910E94856C0E94C96F359613
:1039E800E491EA1730F40E94856C0E94C96F0E9426
:1039F800CE6F3CC0E230A1F4DA010E94647AE03173
:103A0800A7E2FA0714F4FF2352F40E94856C0E947F
:103A1800C96F36960E94737ADA01ED93FC9326C03B
:103A2800E33059F4D901AC91AF3F31F40E94856C71
:103A38000E94C96F0E94CE6F19C0E430B9F4D90151
:103A4800AC91AF3F99F400E00E94856C0E94C96F69
:103A58003596E4910E1750F40E94856C0E94C96F48
:103A68000E94CE6F2F5F3F4F0F5FEECF1F5F99CF42
:103A7800E8DB10E0113060F41A9348DDA091B80D2E
:103A8800A23020F01A9377DD1A9362DD1F5FF2CF20
:103A9800E02F0C941E22E881EF5FE883A881A4360A
:103AA80010F0E0E0E883E8810C9493220E94D36F41
:103AB80030960C949322A091C00DBB27E091BF0DC6
:103AC800A6C0F9DF329774F00E94DA6FE091BF0D5B
:103AD8000E94E16F0E94876EE091BF0DEA93DBDFE1
:103AE800E093BF0D08950E94DA6FE091C00D0E9427
:103AF800E16FFA93EA930E940C670895EDEAFDE0FE
:103B08000E94E96F0E94DA6FE091C00D0E94E16F98
:103B18000E94876EE091C00DEA93BDDFE093C00D6F
:103B280008950E94487CE0E0E093BF0DE093C00D4B
:103B380010E030E0343680F5A8950E94DA6F3A93A9
:103B4800B5DFFA93EA93EDEAFDE00E94A46E00E087
:103B5800A091AD0DA13010F0A03808F001C001E02F
:103B6800E12FE03041F4013029F43093C00D309357
:103B7800BF0D11E00FC0E13031F4003019F430937B
:103B8800BF0D12E007C0E23029F4013019F4309378
:103B9800C00D13E03F5FCECF45C21A93A091580DD8
:103BA800A870B9F010E0E981FA810E94836BAE1722
:103BB800BF077CF4ED81E093AD0DEB81FC81E8510A
:103BC800FC4F0E94F06FE0E0F0E00E94616F1F5F21
:103BD800EACF18810C942022E881EF5FE883A8815E
:103BE800A43610F0E0E0E883E8810C949322E881A1
:103BF800E150E883A881A43610F0E3E6E883E88181
:103C08000C949322A091C20DBB27E091C10DF0E066
:103C180031960E94F56FEC59FF4FDF01E4E6F0E0C2
:103C28000E94217A08950E94D36FE050FE4F0C94B1
:103C380093220E94FA6FE881EA93C0D10C949322F0
:103C48001A932BDBE1E0E0930F0DA8C1A89510E0D3
:103C5800143680F41A93ABD1A091B20DAF3F31F472
:103C68000E94FD6FAF3FEFEFBE0711F01A93E1DF3F
:103C78001F5FEECF0E940270689420F88FC10E94E7
:103C8800487C1091C20DAD81AA23CAF5E091C10DFF
:103C9800E11719F0AD81AA230AF030C01A9387D131
:103CA8000E94FD6FEE81FF81EA17FB0729F4E88582
:103CB800A091B20DEA1709F01EC00E940870EC81AD
:103CC800FD810E945E79EA17FB0744F40E940D709B
:103CD8000E941670E0E0EC83ED830BC00E940D702B
:103CE800EC83FD83E0E0F0E00E941670E0E0E093F2
:103CF800B20D1A9363D10E941B70C8CF46C0E091E1
:103D0800C10DE11729F0AC81BD810E943C7C0CF00B
:103D18001BC01A934CD10E94FD6FEE81FF81EA17F8
:103D2800FB0729F4E885A091B20DEA1709F009C04C
:103D38000E940D700E9416701A9340D1E0E0EC8347
:103D4800ED830E941B70DBCFAC81BD810E943C7C5F
:103D58001CF458DF33970CF418C0E885E093B20DD3
:103D6800EE81FF810E942070EC81FD810E94167017
:103D7800E091C10DEA9322D1E091C10DEA932CDFC5
:103D8800E093C10DE0E0EC83ED83689420F8EC81CA
:103D9800FD810E944F7C299608951A93A091D30D16
:103DA800A03059F4E091D60DF091D70DFA93EA932B
:103DB800E8EBFBE00E94257009F40BC0E1E0E0931A
:103DC800D30DE091C10DE093D50DE091C10DE093C5
:103DD800D40DA091D30DA13011F00C94541FE09193
:103DE800C20DA091D50DEA1711F40C94451FE0916E
:103DF800D50DEA93FCDEE093D50DEA93D8D0A091D7
:103E0800B20DA13010F0A03808F034C0E091D40D04
:103E1800EA93EDDEE093D40DA091D50DEA1749F1B0
:103E2800EA93CCD0E0916B0DE030E9F410E0133068
:103E3800D0F4ABE01A9FF001DF01E852F84FE081BF
:103E4800E03049F0FD01E952F84FE081AE2FE091F2
:103E5800D50DEA1709F005C00E942B70A091D40D6A
:103E6800A0831F5FE4CF0E94FA6FE091D50DEA931B
:103E7800A5D006C00E94FA6FE091D50DEA939ED0B6
:103E88000FC0E091D40DE093C20DE0E0E093D30DB4
:103E9800689420F80E942668E093D60DF093D70D19
:103EA8007DC01A93A8951091C20DE091C10DE1173C
:103EB800C1F00E9431700E943C7C64F4EB81A091B7
:103EC800B20DEA1739F40E94FD6FE981FA81EA1709
:103ED800FB0709F003C0E12F1881A6C00E941B70E0
:103EE800E4CFEFEF1881A0C00E9408700E943C7CCC
:103EF80084F4E0911008E87031F4E091B709A091DA
:103F0800B20DEA1731F40E9435700E94466FE03412
:103F180008F001C086C10C94EF22A895E091C10D6C
:103F2800A881EA1761F0E8810E943A7019F0E881E7
:103F38000C949322E881EA934FDEE883EFCFEFEF0A
:103F48000C9493221A93A8951091C20DE091C10D7B
:103F5800E117E1F00E9431700E943C7C8CF4E09102
:103F68001008E87031F4E091B709A091B20DEA1792
:103F780039F40E94FD6FE981FA81EA17FB0709F01D
:103F880002C00C94D6220E941B70E0CFEFEF0C9475
:103F9800D7221A931091C20D1A93BFDF1991089571
:103FA800E881EA9319DEE883EA93B7DFB8C20E9492
:103FB800DA6F0E9441700E94A46EB1C20E94DA6F4B
:103FC8000E9441700E94876EAAC20E94487C0E948B
:103FD800027010E030E0343628F5A8953A93E7DF10
:103FE80000E0A091B20DA03808F401E0E12FE03024
:103FF80041F4013029F43093C20D3093C10D11E022
:104008000FC0E13031F4003019F43093C10D12E0E3
:1040180007C0E23029F4013019F43093C20D13E0DF
:104028003F5FD9CF0E944F7C249608950E944A7022
:10403800A43009F43FC01091B7090091E20DE09156
:10404800B909E03059F0E093B709689424F80E9460
:104058004F70E0E0E093B809E0E520C0E091B809CE
:10406800E03021F0E093B709E2E518C0E0E0E09322
:10407800B709E093E20DE0914D0DE03031F0E091A9
:104088004D0DE150EA930E944A1AA091BD0DA1700E
:1040980039F0E0914D0DE093B709E4E4E093E20DC7
:1040A800A091B7091A1721F4A091E20D0A1711F08F
:1040B800689423F80991199108951A930A930E9414
:1040C800316EEE59F64F8F01D8011196EBE0EC9363
:1040D800EC81D8011696EC93EB81D8011796EC93F6
:1040E800D8011896E0E0F0E0ED93FC93D801129621
:1040F8000E945570D80114960E9455700E945A70FB
:10410800259608951A930A930E94316EEE59F64F38
:104118008F01D8011196ECE0EC930E945A7044C2CA
:104128001A9318E0113108F5E0919D09F0919E0964
:10413800A981BA81EA27FB27BF010E946670E6239E
:10414800F723309781F00E946670A981BA81EA232B
:10415800FB23309731F01A93E0E0EA931A93ADDF2E
:1041680002C01A93CFDF1F5FDDCF1DC2A091A30D40
:10417800A93030F0E091EA0DA091E90DEA1709F4B1
:1041880014C0E091EA0DE03021F4E3E6EA93BADFE7
:1041980008C0E091A30DEA93E0E0EA93E3E6EA932E
:1041A8008CDFE091EA0DE093E90D08951A93A09150
:1041B800A209A13011F0A93009F4F5C110E01530B9
:1041C80088F40E94717039F0FD01E25DF74FE081DB
:1041D800AA81EA1709F004C00E947A700E947F70D1
:1041E8001F5FEDCFE0C1A091230DECE1EA23089514
:1041F800A091230DA07411F0E2E00895A091230D81
:10420800A07809F0E8C10DC0A091120DAF3F09F4E4
:10421800E2C1E9DFE43009F4DEC1E5DFE03109F4A9
:10422800DAC1E1E008950895A881AF3F11F4E0E014
:1042380076C1D9DFE43011F4E1E071C1E0E06FC18B
:10424800A881A23019F4CFDFE83011F0E1E067C1AE
:10425800E0E065C1A881B981AC91A130A8F0A8813E
:10426800B981AC91A43180F4A881B981EC910E9404
:10427800AF6CE050FB4FE081EF770E2EA881B9813B
:104288001296EC91E01509F002C0E1E00EC1E0E001
:104298000CC1A881A13118F0E881E051E883E881D8
:1042A8000E9484700E948E70A091590DA13018F060
:1042B800A881A43009F006C0E6E9F0E00E94737A0C
:1042C8000E948E702CC1A881A13010F0A23008F095
:1042D80006C0E8810E949970EC5DF74F1FC1E0E0CD
:1042E8001EC1A881A13010F0A23008F006C0E881F4
:1042F8000E949970E75DF74F11C1E0E010C10E947C
:10430800487CEC81EA93EDDFEF731E2F1030E1F06B
:10431800EC81EA93E6DFE0743E2FE12FE150A1E063
:104328000E946A79A0910808EA230E2F303011F410
:10433800003009F002C0E1E00BC5303011F0003068
:1043480009F402C0E1E004C5E0E002C50E94467C31
:1043580000E00130A0F50A930E948A1A0E949E701C
:10436800A7E10A9FF001E95EF74F0E94BC6F0E9427
:10437800E96C0E948E68E091B90DDA015096EC93D1
:10438800A091B80DEFE3EA23AE2FE091BB0DE295C3
:10439800E07FEE0FEE0FEA0FDA015596EC93E0910D
:1043A800B90DE1503E2F3F3F41F0E091BA0D0E9418
:1043B800566FDA015196ED93FC930F5FCACF10E068
:1043C8001034C0F51A930E94E5191A932DDFE130D5
:1043D80079F5E091260DEA9376DFE1500E2F0F3F35
:1043E80039F10E949E70E12FDA011396EC93E09167
:1043F800260DDA011496EC93E0912C0DF0912D0D19
:10440800DA011696ED93FC930E944F6FA4E6B0E094
:1044180080E090E00E94C979DF01CB01E0912C0D8A
:10442800F0912D0D0E942E6DDA011A96ED93FC93F2
:104438001F5FC6CF0E944D7C26960895A091A209C1
:10444800A23031F0A83021F0A73011F0A53009F4DE
:104458000AC00E94676FEFEFF0E00E946E6F76DF90
:10446800E0E0E0932B0808951A93E981E058E98386
:1044780010E01530C0F4A3E21A9FF001E25DF74F97
:10448800E081AE2FE981EA1749F4F001E35DF74FC7
:10449800E081AE2FE091B709EA1709F002C0E12FD9
:1044A80003C01F5FE6CFEFEF1881229608950E94A0
:1044B800487CED81EA93D8DF1E2F1F3FD1F0A3E29D
:1044C8001A9FF001E45DF74F9F01D9011296EC9114
:1044D800EF77EC93EC81D901EC930E94AF6C0E94CA
:1044E800A570EF77DB01EC93EC810E94AF6C0E9422
:1044F8007F70E12F0E944F7CA4C40E94AA70E081C3
:10450800E03051F4E091DC0DEF5FE093DC0D0E94A8
:10451800AA70A091DC0DA0830E94AA70E081219668
:1045280008951A931FEFE0915D0DF0915E0DA9813A
:10453800BA81AE17BF073CF0E0915F0DF091600DB6
:10454800EA17FB070CF412C00E94AF700E942A19E8
:104558001E2F103031F01F3F21F0E091B709E1170D
:1045680029F4E1E0E093EA0DE0E01DC0E0E0E0932B
:10457800EA0D18C01A930E94AF70D3DF1E2F1030B7
:1045880089F01F3F39F4EEE4F9E1FA93EA93EB81FD
:10459800FC8104C0EEE5F9E10E94A76CFA93EA9366
:1045A8000E946611E12F188123960895E091600713
:1045B800E03009F00895E0911108E03009F008951D
:1045C8000AC0E0916107E03009F00895E09112080F
:1045D800E03009F00895E0E0089528970E94467CAD
:1045E80030910B0810E01130B8F5A7E11A9FF001DF
:1045F800E65DF74F0081E12FA1E00E946A792E2F36
:10460800E22FE32391F0003810F0003C08F001C0DD
:104618000F5F003C31F4E22FA0910808EA2BE093E9
:104628000808003808F400E80FC0003408F40F5FE9
:10463800003439F4EFEFE227A0910808EA23E09369
:104648000808003808F000E0A7E11A9FF001E65DCD
:10465800F74F00831F5FC7CFE0E0E0931108E0E069
:10466800F0E0E0939F09F093A009E091EA0DE030B3
:1046780021F0E091A30DEA930CDEE091A609EF5F2B
:10468800E093A609E0916C0DA091A609EA1751F4F0
:10469800E0916C0DF0E0A0E0B1E00E94877AEA1B9F
:1046A800E093A609A091A209A13019F0A93009F058
:1046B80096C0A091EB0CB091EC0CE4E1F0E00E9404
:1046C800217A309719F4E1E0E093A8096FDFE03030
:1046D80019F077DFE07809F462C073DFEF775E2FB7
:1046E8005A930E94E5190E94456CE45DF74F50818A
:1046F800503011F40C94D32387DDE13031F4E0918C
:10470800A309EA939DDDE03009F449C00E94B47022
:10471800AE0FBF1FEC91EC71EC3021F4E091A609CB
:10472800E07851F40E94BA70EC91EA93B2DD0E94ED
:10473800C270EC91EA93ADDD0E94BA70AC91A630DC
:1047480070F5ACE6B8E00E94456C0E94CA700E9401
:10475800B16D0E94BA70EC91EA93B5DD1E2F11304D
:10476800F0F00E94CF700E94D270CF010E94CF70EB
:104778000E94CA706D917C91E12F0E949970EA5E47
:10478800F74F0E94D770E60FF71FDC01ED93FC93FB
:10479800E12F0E949970EA5EF74FA0E0A08310E035
:1047A8001130E8F40E94DA7013965C915F3FA9F02B
:1047B8005A93A3DE5E2F0E94E4700E94CF700E947D
:1047C800D270BF010E94CF700E94CA700E94EA7026
:1047D800AE81BF811296E0E0EC931F5FE1CFA0911C
:1047E800A209A23039F0A83029F0A53019F0A73075
:1047F80009F0DFC100E0053010F00C94DD25A3E2DC
:104808000A9FF001E45DF74FEA87FB87AA85BB851D
:10481800AC91A03019F0A281A07809F0C8C1AA858E
:10482800BB8513960E94647A309771F0AA85BB8580
:1048380013960E94F7700E94FD7029F4AA85BB8523
:1048480013960E945570B3C1BCDEE03021F00E947F
:10485800FD7009F4ACC120E030E0333010F00C9466
:1048680086250E940771DF010E94B46B0E940D71BA
:10487800A27031F4E885F985A481B581109709F40F
:104888000FC1E885F985A181A47011F40C94AE24B8
:10489800A181A87021F40E94C034E03009F459C005
:1048A8000E94316E0E941871EBE0EC93A885B985DF
:1048B8000E942071A885B9851396EC91AC85BD85B9
:1048C8001796EC93EC85FD8538960F01E885F985F8
:1048D800A181E1E0EA230E942771ED93FC93A8856A
:1048E800B98514960E94647AAC85BD851296ED93BD
:1048F800FC930E942A71AC85BD851496ED93FC93B8
:10490800A02FEAE0EA9FF001E30FEF5F0E94307109
:10491800E885F985A085B185E2E0F0E00E94C479D8
:10492800A885B9851896ED93FC930E942A71309753
:1049380039F4A885B9851896E8EEF3E0ED93FC9371
:10494800E885F985A181E8E0EA2BA885B985119663
:10495800EC936CC0E885F985A181A17031F4A88534
:10496800B98514960E94F77041C00E943971ABDC7A
:10497800E1501E2F0E94DA701296EC91E030F1F4AB
:10498800AE81BF8153960E94B16DEE81FF81A189EE
:10499800B289109751F003881488AE81BF8151966F
:1049A8000E94647AE015F1050CF007C00E943E7180
:1049B80011F00E9446710E944E710EC0E885F9857B
:1049C80034960E9456710E9427710E94F56F0E94CA
:1049D8005E7153960E945570E885F985A581AA23D2
:1049E8002AF4A885B98514960E945570A885B985BA
:1049F800EC91EC71EC3021F4E091A609E078B1F487
:104A0800E885F985A481B5815E971CF4A181A0721F
:104A180009F404C0E885F985A28106C00E943971AD
:104A280038DCE885F985A381AA9333DC0E942A71D2
:104A3800309781F0A885B98518960E94F7700E9472
:104A48002A71309739F40E943E7111F00E94467124
:104A58000E944E710E94397152DCE03009F10E94C7
:104A68003E7161F00E944671AA85BB85EC910E9457
:104A7800AF6C0E94A570E058DB01EC93AA85BB855A
:104A88001296EC91E058AA85BB851296EC93E3E068
:104A9800E09309080E94397124DCEF73E0930A0857
:104AA800A885B98514960E94647A309749F52F5FD6
:104AB800323030F5A885B98516960E94647A309709
:104AC80089F0E885F985A681B7810E946571AA8574
:104AD800BB851396ED93FC93A885B98516960E941D
:104AE80055700EC00E940771DF01E32FEF5FF0E001
:104AF8000E940D71EDEFEA23A885B9851196EC9314
:104B08003F5FABCE233011F00C94DB250E94C034FC
:104B1800E03079F00E94316E0E941871E8E0EC9361
:104B2800AA85BB850E942071AA85BB85EC910E944D
:104B380030710E943E7111F00E944671AA85BB85B2
:104B4800E0E0EC93EA85FB85A581ECE1EA23E83017
:104B580071F50E94536EAE2FEA85FB85E38DEA1747
:104B680041F4EA85FB85E48DE150EA930E94DE1862
:104B78001EC00E94C034E030D1F00E94316E0E9405
:104B88001871E3E0EC93AC85BD85EFEFEC931896D4
:104B9800EA85FB85E38D0E946A71AC85BD85129616
:104BA800EA85FB85E48D0E946A710E946E710F5F31
:104BB80022CE0E94747149F4A091A209A23021F07A
:104BC800A83011F0A53009F401C050C010E0113030
:104BD80010F00C943A260E94DA7013965C915F3FAD
:104BE80011F40C9438260E94E470AE81BF81BD0197
:104BF8000E94EA70EE81FF8138960E9456710E94E9
:104C08007A710E945E710E94647ADF010E943C7C86
:104C1800B4F4EE81FF81A681B7810E943C7C7CF4CC
:104C2800AE81BF810D901C90AE81BF8116960E9407
:104C3800647AD001AE1BBF0B0E943C7C0CF014C000
:104C4800AE81BF81BD010D901C90EE81FF81A681D0
:104C5800B781F001EA1BFB0BDB01ED93FC935A9340
:104C6800E5E0EA930E9494631F5FB1CFE091A50944
:104C7800E03041F4E0919F09F091A009E0939D098B
:104C8800F0939E090E944D7C2E9608950E94487CC0
:104C98000E94A86E1E2F2FE330E00091A709A09173
:104CA800A10DA13080F0E091A10DE150A091A709DC
:104CB800AE1728F0E091A10DE1503E2F04C0E0911D
:104CC800A10DE2502E2FEC81E03049F1EF3F51F475
:104CD800A091A709A11BA31720F0E091A709E11B48
:104CE8000E2F1DC0EE3F59F4E12FA091A709AE0F7A
:104CF800A21720F4A091A709EA0F0E2F10C0EC3FCD
:104D080049F4A091A10DA13020F0E091A10DE1504E
:104D18000E2F05C0AC81A1501A9FF0010E2FE09113
:104D2800A709E01751F00A930E94E519A091130D05
:104D3800AD3209F4032F0093A7090E949251A09164
:104D4800A209A83019F40E94C40F02C00E948F0F54
:104D58000E944F7C259608950E94467C44DAE031F3
:104D680011F40C94222720E030E040E050E010E0FD
:104D7800133050F50E947E710E94D96C309711F162
:104D88000E9481710E9484702E2B3F2B0E9481719A
:104D9800EA93B5DAE03029F0E3E0E0930908E0E0CF
:104DA8004EC00E9488710E9484702E2B3F2B0E9457
:104DB8008871EA93A4DAE03029F0E3E0E093090887
:104DC800E0E03DC01F5FD4CF00E0053068F5A3E206
:104DD8000A9FF001E45DF74FE081E03019F110E03F
:104DE800133000F50E940771DF010E94856C0E9454
:104DF8008F71AE0FBF1F1296EC910E9484704E2BDC
:104E08005F2B0E940771DF010E94856C0E948F71E1
:104E1800AE0FBF1F1396EC910E9484704E2B5F2B30
:104E28001F5FDECF0F5FD1CFF901E423F523309761
:104E380029F0E1E0E0930908E0E001C0E1E00E9428
:104E48004D7C269608951A93E091E00DE03011F418
:104E58000C947C27E0916D0DE13059F4A091E00DA0
:104E6800A13311F4EFE001C0E0E0EA930E949C381E
:104E78003FC0E23059F4A091E00DA13311F4E6E00F
:104E880001C0E5E1EA930E949C3832C0E53061F444
:104E9800A091E00DA13319F4E091220D01C0E0E0EA
:104EA800EA930E949C3824C0E330B1F410E0173034
:104EB80040F40E94856CE853F54F0E9496711F5F7D
:104EC800F6CFA091E00DA13311F4E1E301C0E0E3D6
:104ED800EA930E949C380CC00E949A71E9E4EA9314
:104EE8000E94F03CE091E00D0E94A1710E94A67121
:104EF80084C422970E94467C30E0A091A209A23087
:104F080029F0A83019F0A53009F017C1A985A034F7
:104F180010F00C94A028E091B709E03009F40DC115
:104F2800E9850E943C6FE03131F4E1E3E093E00D64
:104F38008ADFE1E002C168D9E03009F4FEC010E080
:104F4800153080F40E94717041F0FD01E25DF74F69
:104F5800E081AE2FE985EA1709F002C0E0E0EDC074
:104F68001F5FEECFF9DEE03011F40C94A02810E0BA
:104F7800A3E21A9FF001E45DF74FEE83FF83AE8151
:104F8800BF81EC91E03011F00C94992813960E949F
:104F9800557000E0033010F00C946A28A3E21A9FC1
:104FA800F001EF5CF74FDF010E94CD6B0E94AB71FF
:104FB800AF01DA0116960E9455700E94B371DA01AA
:104FC8001296EC930E94BA71DA011396EC93A091B1
:104FD800230DEEEFEA23DA01EC930E94C171DA01A6
:104FE8001196EC9300D9E43139F0FA01A181E2E09D
:104FF800EA2BDA011196EC930A9322D9E03011F4E6
:105008000C944C28FA01A281AA935DD9E1502E2F65
:105018002F3F81F0A7E12A9FF001EA5EF74FA0E059
:10502800A083A7E12A9FF001E95DF74FA0E0B0E077
:10503800A083B1830E94C9710E94D96CDA011496C9
:10504800ED93FC93013030F00E94C9710E94D96C35
:10505800309709F00EC0AE81BF811596E02F0E94EF
:10506800E26E0E948F71AE0FBF1F1196EC91E06245
:10507800EC93AE81BF815A96EC91E062EC930230DA
:1050880030F40E94CC71DA0116960E946A7104C04D
:10509800DA0114960E945570A6D8EC3019F4E0E0B5
:1050A800E093A6090E94D3710E94566FDA01189600
:1050B800ED93FC93FA01A281A63030F0A181E4E0DF
:1050C800EA2BDA011196EC930F5F64CFA091A20945
:1050D800A23011F0A53019F4A885AF3F08F007C039
:1050E800E091B709EA93EA85EA930E94251BE885CF
:1050F800AE81BF81EC93E091B709AE81BF81119673
:10510800EC93E985AE81BF811296EC93A885A43112
:1051180028F4E8850E94AF6C0E947F70AE81BF8141
:105128001696EC91ED7FEC9331E01F5F303011F46F
:10513800153008F001C01CCFE32F0E944D7C2A9641
:1051480008950E944A70A23021F0A091A209A530CA
:1051580021F40E94DA710E94D16DA091A209A830B1
:10516800E1F40E94DA71E1E0EA930E94F651E091DD
:105178006B0DE03081F4EA81ADE0EA9FF001E05088
:10518800FB4FE081EF771E2FABE01A9FF001EF5144
:10519800F84FA0E0A083689420F81981088123962D
:1051A800089564970E94467CA091A209A23039F420
:1051B800E091B709EA93EB8DEA930E94251BA09131
:1051C800A209A83011F00C944D290FEF20E02130EE
:1051D80050F4A7E12A9FF001E95EF74FE081AE2F76
:1051E800EA8DEA1709F402C02F5FF1CFA7E12A9FE1
:1051F800F001EC5EF74FAF01DA0115960C910F3F05
:1052080011F40C944D290E94E57110810E943170AF
:105218000E943C7CECF4A5EBBDE00E94F7700E9474
:10522800EB710E940870A083B1831A930E94E21F59
:10523800ABE00A9FF001E752F84F30810A93FE0174
:1052480037960E94F1713A93FE0137960E94F571E4
:105258000E94FB71F1F40E94E571AFEFA083DA01BF
:105268001396EFEFEC93DA011596EC930E94EB712D
:105278000E940172E0E0F0E00E941670E0E0E09326
:10528800B20D1A930E94E21F0A930E9403116894B8
:1052980020F80E944D7C6B9608951A9310E0103107
:1052A800B0F4A7E11A9FF001E75DF74FE081EF73D3
:1052B800AE2FE981EA1729F41A930E948321E0307E
:1052C80009F403C0E1E01881DEC01F5FE8CFE0E029
:1052D8001881D9C01A93E091E30DF091E40DFA9387
:1052E800EA930E94B76D0E943268E030E9F00E94AC
:1052F800067210E01130C0F4A091E70DAF5FE0E056
:10530800E093E70DEF5FEA93C8DFE03059F0E3E0A0
:10531800E0930908E091E70DF0E0EF5FFF4EE093BE
:105328000A086BC21F5FE6CF68C21A93E0910808AB
:10533800E093DF0DE8E7F0E0FA93EA93ECEDF0E0B4
:10534800FA93EA930E94C35110E01130E0F4E12F80
:10535800EF5FEA93A2DFE030A1F00E94326BE12F09
:10536800EA5F0E940D72EBE6F9E10E94926CAFE6EB
:10537800BDE00E94856C0E94AB71FA93EA930E948B
:10538800F26D1F5FE2CF39C2A5DFE0910908E13075
:1053980029F4E3E7F9E10E940F723CC0E23029F4F6
:1053A800E0E8F9E10E940F7235C0E33051F4EBE612
:1053B800F9E1FA93EA93E0910A08F0E0E050F04F3F
:1053C80029C0E43019F4E8E8F9E11FC0E53031F408
:1053D800E0910A08EA930E94651120C0E63019F4AA
:1053E800E0E9F9E112C0E73029F4E6E9F9E10E94C1
:1053F8000F7210C0E83029F4E2EAF9E10E940F7256
:1054080009C0E93059F4E1EBF9E1FA93EA93E09144
:105418000A08F0E0FA93EA930E946611E0E0E0934C
:1054280009080895A881B9811196E1E0EC930E94DA
:105438003570A881B9811296ED93FC930E94FC20E7
:10544800A881B9811796EC930E94536EA881B981FF
:1054580018960E946A71E091C107A881B981EC93FE
:10546800E091B20DA881B9811696EC93E091120DE6
:10547800A881B9811A96EC930E941472A881B98107
:105488001496ED93FC932296089564970E94487CA5
:10549800A0916B0DA230E1F4EB8DEA930E94E5191F
:1054A8000E94FC20A5EBBDE00E946A71A3EBBDE061
:1054B800EB8D0E946A71E091B709E093B20D0E94EA
:1054C800416F309721F00E94416F0E94207014C0F4
:1054D800AA8DAF3F09F4CCC0EA8DEA930E94DB1F86
:1054E800AB8DAF3F29F40E9435700E94466FEB8F59
:1054F800EB8DEA930E94E5190E94FC200E2FA98DDE
:10550800AF3F21F00E940821E03009F001C0B0C08F
:105518000E9408700E94CD6BAE17BF071CF01CDC00
:10552800E13009F0A5C0A0915A0DA03021F4A09156
:105538006B0DA23021F50E94536EE13041F00E94BC
:10554800C034E03021F00E94D634E03009F004C0C5
:105558000E94316E0E9419720E94536EE13021F44C
:105568000E94C634E03009F409C00E942072E55D4B
:10557800F64FFA93EA9356DF0E94267277C0EB8DB6
:10558800EA93EA8DEA93B5DC1E2F113011F00C94E2
:105598003A2BA0915C0DA13059F4E091B709EA9338
:1055A8000E943570FA93EA93EFEFFFEF0E942C7296
:1055B8000E9408700E94CD6B0E94F56F0E941670C1
:1055C800689420F8A0916B0DA03019F4A88DAF3F16
:1055D80009F437C00E943072E352F84F0E940870F5
:1055E800A083B183E88D0E94A16C3081E88DEA9395
:1055F800FE0135960E94F171E88D0E94A16CE08150
:10560800EA93FE0135960E94F5710E94F720E03179
:1056180031F00E943072EF51F84FA1E005C00E94AE
:105628003072EF51F84FA2E0A0830E943072E1522D
:10563800F84FFF93EF930E942668AF91BF91ED93C7
:10564800FC930E94FB7119F4E0E0E093B20DEA8D3F
:10565800EA930E94E21FE091B709EA930E94416F22
:105668000E94DA6BFA93EA930E94D11DE1E001C02F
:10567800E0E00E944F7C6C9608956EDBE13041F4C7
:105688000E94C034E03021F00E94D634E03009F0A6
:1056980009C00E94416F0E9420700E94316E0E94D2
:1056A80019723BC343C30E94487C0E9435721F3F56
:1056B80011F40C94A82BE091E00DE03011F00C945B
:1056C800A72B1A930E94E519E5E0E09309081093C7
:1056D8000A08A091A209A23031F40E943E720E94E9
:1056E800BE22E03009F00EC0A091E10DA13331F4E3
:1056F800E091B709EA931A930E94251BE1E3E0932E
:10570800E00D2CC2A091A209A83091F40E94416F2B
:105718000E9442720E2F0A930E943A353E2F1A9326
:105728000A93EFEFEA933A93B0DEE03009F016C23D
:10573800A091A209A53021F4A0DFE03009F00EC243
:10574800E0E3E093E00D06C0E0E3E093E00DE4E081
:10575800E093090803C2E091C80A0E9446720895BE
:105768001A93E6E0EA930E949C380E949A71A091ED
:10577800C80AA83539F4EDEBF9E10E945272E0E06D
:105788000E94A671A091C80AA33509F510E0A0915E
:10579800A209A83021F0A23011F0A53009F411E3D4
:1057A800E3E5EA930E94F03C1A930E94F03CE0E89B
:1057B800EA930E94F03CE0E8EA930E94F03CE0E8BB
:1057C8000E94A171E093E00DE0E00E94A671A09113
:1057D800C80AA93491F4A0916D0DA43019F4E0E041
:1057E800E093E00D0E945672E0930A080E946072EE
:1057F800EC91E093E10D57DF26DB199108950E94A3
:10580800487CA091C70AA53411F00C944A2C0E9438
:105818006572E2E3F0E0E093DA0DF093DB0DA0911E
:10582800C80AA73741F4ECECFAE00E946C720E94B7
:1058380071720E944672A091C80AA03310F0AA3370
:1058480008F023C02091AF093091B009E8ECFAE0E4
:105858000E946C72E2E0EA930E94963C0E2F0E942E
:105868007172E0930A080E9471720E9475720E9418
:1058780035720A931A930E94251B2093AF0930931F
:10588800B009E2E5EA930E949C381CC0E091D80D6B
:10589800F091D90DFA93EA93E091DA0DF091DB0DCE
:1058A8000E94257079F0E0E0E093C20AE5E4EA930B
:1058B8000E949C380E946572E8ECF0E0E093DA0DF3
:1058C800F093DB0D4BC10E947A720E9480720E9495
:1058D800326B0E94326B0E946D51A091A409A230D4
:1058E80021F4E5ECF9E10E94926CA091A409A130A1
:1058F80021F4ECECF9E10E94926CE091A409E0300B
:1059080021F4E3EDF9E10E94926C0E948A720E94F0
:105918006D510E948F720E9494723197FA93EA93A4
:10592800E0915A07F0915B070E9499720895E1E0AF
:1059380003C0E0E001C0E2E0E093A409C4DF0895F9
:105948000E94F720EC3109F0F1C1E091220DE33615
:1059580031F4A091A209A23009F4EBDF17C0E236B6
:1059680031F4A091A209A23009F4E5DF0FC0A0919B
:10597800C007A23011F0A63021F4E091220DEA937D
:1059880085D9A091C007A43009F4D1DFC6C11A9304
:105998000A93A0E023FCA1E0A03019F0AA81A0306E
:1059A80009F014C0E89423F8E7E0E093A1090E9405
:1059B800AF50A091B909A03019F40E949D7209F462
:1059C80005C00E94A272ACD7E89424F824FE27C030
:1059D800E091BB09F091BC090E94866B0E94326875
:1059E800E13019F0AA81A130C9F4C6D7E030B1F08E
:1059F8000E94A7720FEF1FEF0E943E720E9495222D
:105A0800E03021F40091AF091091B009EB81EA93DD
:105A1800E091B709EA931A930A9382D712C0E091EA
:105A2800BB09F091BC09FA93EA93ECE2F1E0FA932E
:105A3800EA930E943268E13021F40E94AE72E0934A
:105A4800B809198108818CC0E1E0E09309060E9439
:105A5800326B0E94326B0E94B2720E94326B0E94BB
:105A6800326B0E946D51E4EAF4E00E94926CE0917E
:105A7800A3090E94B672E2EBF4E00E94926CE2E0A5
:105A8800E093090608950E94676FE0ECF0E00E9439
:105A98006E6FE881E03009F406C0A091A309AF5FFA
:105AA800E3E00E941E7AE093A309E1E0E093DC0DB5
:105AB8000E94AA212AC20E94487C10E0103410F0EB
:105AC8000C94B22D0E94856CE45DF74F30813F3F06
:105AD80011F40C94B02D1A930E94E51900E00E946D
:105AE800BA720E94D96C3B97C4F00E94BD720F0134
:105AF8000E94BA720E94D96CD001ED93FC930E9467
:105B0800B470EA0FFB1F0F010E94B470AE0FBF1FE5
:105B1800EC91EE7FD001EC9301E00E94C3720E94E9
:105B2800D96C7597A4F00E94BD720F010E94C372D0
:105B38000E94D96CD001ED93FC930E94B470EA0FD7
:105B4800FB1F0F010E94B4700E94C67201E0013071
:105B580019F41A930E940D1A1F5FB0CF0E944F7C50
:105B6800249608950E944A70A93011F40E94CD72BB
:105B780023FE06C0E7E0E093A1090E94A272D0D6F6
:105B88000E94A663E030A1F1E0E00E94D4721038D0
:105B980038F5113231F4E7E0E093A1090E94A272CE
:105BA800BFD61D3439F40E94DB720E94003EE3E048
:105BB800E093A1091B3271F40E94E072EAE2EA93D1
:105BC800EEEDF9E1FA93EA93E091A309E05DEA9337
:105BD8000E94003E1F3219F4E1E0EA9357D834DFFF
:105BE800103830F00E94E6721A930E948122A8DED3
:105BF8000E94E5220E2F003810F40C94432E0F77E4
:105C08000034E0F5E091A809E03069F00A930E94B9
:105C18008122A091A209A13019F40A930E94BB1114
:105C2800E0E0E093A809E091E80DE01739F10A9364
:105C38000E94E5190E94BA70AC91A83028F40E941D
:105C4800C270AC91A830A8F0E02FEF5FE0932B086A
:105C58000A930E9481220E94BA70EC91EA930E94F2
:105C6800C270EC91EA93E0912B08EA930E946120BC
:105C780003C0E0E0E0932B080093E80D0EC0A0916C
:105C8800E80DAF3F51F0E0912B08E03019F0EA93AE
:105C98000E948620EFEFE093E80D0991199108958D
:105CA800A881A03310F0AA3308F01BC00E94EA7242
:105CB8000E94EF72AAE0B0E00E94C479DF01E88197
:105CC8000E94F472EA0FFB1FE093AD09F093AE094E
:105CD800E1E0E09309060E948A720E94B2720E9473
:105CE8008F72A881A33441F40E9480720E948A7244
:105CF8000E94B2720E948F7208C1E091500DF0911B
:105D0800510D0E94F77211F4E2E00895E0914E0DF2
:105D1800F0914F0D0E94F77211F4E1E00895E091BF
:105D2800540DF091550D0E94F77211F4E0E00895BA
:105D3800EFEF0895E0E0E093A409A091A209A23052
:105D480021F40E9492510E948F0FA091A209A830BD
:105D580009F447D6A091A209A53009F442D10895C3
:105D6800E2E0EA930E946E61E1E0E0930906E881CF
:105D7800EA9396DFA881AF3721F4E0911008E37029
:105D880009F403C0E2E0E093A109A881A13239F047
:105D9800A33421F40E94EA72109709F004C0A0917C
:105DA800A209A23009F00FC0A091A409A33009F4F8
:105DB800C2DDA091A409A23009F4BCDFE091A409D6
:105DC800E03009F4B6DDA881AD3311F00C94452F0D
:105DD8000E94AF50E091A409E030A1F4E091AD0930
:105DE800F091AE09FA93EA930E94BE22E03041F4A2
:105DF800E091AD09F091AE090E9475729BDF01C078
:105E080098DD3FC0E13069F478DFEF3F41F0E3E02F
:105E18000E94FB720E94DB720E94017301C08ADF3C
:105E280030C0E23001F50E94EA72A034E0E0BE071B
:105E3800C4F4E091AD09EA930E940873E1E0E093AD
:105E480009060E94326B0E94326B0E946D510E94BB
:105E5800B36E0E94F26D0E948A10E3E0E093A409F9
:105E680001C069DD0EC0E33061F4E091AD09EA9349
:105E78000E94E519E091AD09EA93EEEFEA9339D86B
:105E88005ADDA881AD3409F452DDA881A43521F486
:105E9800A091A209A23009F001C04BDDA881AB3264
:105EA80021F4EEEFEA930E944A26A881AD3221F44C
:105EB800EFEFEA930E944A26A881A73421F4E1E093
:105EC800EA930E944A26A881AB3421F4ECEFEA93C6
:105ED8000E944A261AC00E9422220E949251E0E0A3
:105EE800E093A409A881A13039F40E949D7221F0A1
:105EF800A091530DA03009F402C01BDD06C00E941A
:105F08008F0F0E943E720E949522219608951A933F
:105F18000A930E94CD720E940C7391F10E9414732F
:105F280078F10E94E6720CDDE03051F50E941C7396
:105F38000E945B22EF3F09F0F0C40E943E720E946B
:105F4800BE22E03021F40E940821E13009F018C097
:105F58000E94F720E83119F40E94217309F001C06A
:105F6800DCC40E941C730E947D270E2F013021F48F
:105F7800A091220DA03009F403C01A930E94651164
:105F8800A0911308AF3F61F110911308EFEFE09370
:105F980013081A930E94E5190E943E720E94BE22BD
:105FA800E03021F40E940821E13009F019C00E9474
:105FB800F720E83119F40E94217309F001C0ADC43B
:105FC8001A93EEEFEA930E947D270E2F013021F4F9
:105FD800A091220DA03009F403C01A930E94651104
:105FE8009CC40E9422220E94AA21E89421F8E0E0A1
:105FF800E093A7090E9428730E9492510E94326B75
:106008000E94326B0E946D51E09117080E94F16C5A
:10601800E09118080E94F16C0E94326B0E94886C13
:106028000E946D51E09124080E94F16CE0911E08D5
:10603800F0911F080E94E06C08950E94487C0E941D
:10604800CD72A2D90E94A663E03049F00E94147371
:1060580030F00E94E67274DCE03009F40EDBE09167
:10606800E50DF091E60D0E948C6D0E943268E030DB
:1060780011F40C94A1300E9428730E94326BE2E064
:10608800F0E00E94BA6CE0911C08F0911D080E9493
:10609800E06CE0912008F09121080E94E06C00E09B
:1060A800013010F00C94A130A7E10A9FF001EC5EDA
:1060B800F74F9F01F901A381AF3FE9F1D9011A9682
:1060C8000E94647A0E9486797F936F93FF93EF937F
:1060D8000E942F73AF91BF918F919F910E948679F3
:1060E8000E94C979DF01CB010E943473D9011C9643
:1060F800ED93FC93F90104841584D9011E960E943E
:10610800647AE015F105B9F0F90104841584A685CF
:10611800B785F001EA1BFB0BE093350DF093360DC4
:10612800ACDAE13041F4D9011C960E94647AD901B5
:106138001E96ED93FC930F5FB3CF0E944F7C0EC465
:106148000E94487C0E94CD720E940C7311F40C943A
:1061580037310E94A9630E2F0A9302DE003820F01F
:10616800A091C107A03808F429C00F770A930E94AC
:106178003B730E9442721E2FA0916B0DA03011F448
:106188001F3F09F416C030E0333098F4ABE03A9F73
:10619800F001E952F84FE081E11749F43A9FF00124
:1061A800E752F84FE081EF5FE093C107232F3F5F8D
:1061B800EBCF0A930E941C732A9354C0A0916B0DD5
:1061C800A03021F4003810F0033808F00AC00F7727
:1061D8000E94E5711081EFEFEA930E941C730A9305
:1061E80054D9A0916B0DA03011F0003808F43BC0D1
:1061F8000F770A930E94E519A3DBE030A1F50E940E
:106208003E730E945B22EF3F19F00E944F7CA6C3A9
:106218000E940821E13039F50E94FC20E03049F461
:106228000E943E730E947D27E03011F00E94437364
:106238001AC00E94F720E83141F40E94217321F02E
:106248000E943E730E947D270EC0A091A709E02FEF
:106258000E94486CAE0FBF1F1C910A930E941C73CA
:10626800EFEFEA9312D9A0911308AF3FF9F000912C
:106278001308EFEFE09313080A930E943B730E9400
:1062880042721E2F0A931A93EEEFEA93EFEFEA9306
:10629800FCD81F3F41F4A091260DA03021F4A09115
:1062A800290DA03009F002C00E94437320FE0AC0E5
:1062B800E89420F8E0916B0DE03019F4EAD339D571
:1062C80001C098D530E0333098F5ABE03A9FF00143
:1062D800DF01EF51F84FE081E03049F0A152B84FAB
:1062E8000E944973E8EEF3E00E942570B1F4ABE038
:1062F8003A9FF001EF51F84FE081E23069F43A9F9C
:10630800F001E152F84FDF010E94647A0E948C6D1F
:106318000E943268E03009F409C0ABE03A9FF0010E
:10632800EF51F84FA0E0A083689420F83F5FCBCFEF
:106338000E944F7C13C30E94467CA091A209A330FF
:1063480011F40C945A33E091C209ED3411F00C9415
:106358008332E091C309EA3511F00C94383224FCF9
:1063680083C0E091C409E0532E2FE091C509E053A2
:106378003E2FE6ECF9E00E946C720E946072AC91CC
:10638800AB3429F40E944E730E94223C0E2F0E94C7
:106398006072AC91A43529F40E944E730E94223C8D
:1063A800AF01E091560DE31731F5E0E0E093DE0D23
:1063B8000E94A7724093AF095093B009A091B80901
:1063C8000A1759F0E7E0E093A1090093B809209370
:1063D800DD0DE0E0E093B7090DC0A091DD0D2A17AF
:1063E80021F0A091B609A03009F004C02093A109BA
:1063F8002093DD0D35C0A091B809A03049F4A091D3
:10640800570D0E94B46BE255FF4FE491EA2309F45B
:106418000CC0E7E0E093A1092093DD0DE0E0E093F4
:10642800B709E091C109E093DE0DE091C109A0919F
:10643800DE0DEA17A9F44093AF095093B009009311
:10644800B8090E94A772A091DD0D2A1721F0A0912A
:10645800B609A03009F004C02093A1092093DD0DEE
:10646800273011F40E944F70E091C309E93439F4E0
:10647800E7E00E94FB720E94AE72E093B709E091D8
:10648800C309E23439F4E4E00E94FB720E94AE7260
:10649800E093B709E091C309E03519F4E1E0E0932E
:1064A800A109E091C309EC3449F4E4E0E093A109BF
:1064B800E091C409E053EA930E94B116E091C30940
:1064C800E334E9F4A091C409A13320F0A091C409F0
:1064D800A93308F014C00E945173E091AA09EA9305
:1064E8000E94421CE091C109EA93E1EEF9E1FA93B6
:1064F800EA930E94726F0E94777A0E94F33DE091BE
:10650800C209E03521F4A091A209A13009F003C025
:106518000E94E07299DAE091C209EF3459F4E091EF
:10652800C309EE3439F4E091C109EA93E4EEF9E1E4
:106538000E945773E091C209E33569F5E091C309F8
:10654800EF3349F5A091C409A03320F0A091C50903
:10655800A03308F420C00E945173E091C509E053AC
:106568001E2FA091AA09A63010F41A3008F013C003
:10657800103011F40E948C1BE091C109EA93E7EEF8
:10658800F9E1FA93EA930E94A56F0E94886F0E942E
:10659800777A0E94F33DE091C209E33411F00C943C
:1065A8002233E091C309EF3311F00C942233E091C8
:1065B800C509E03319F4EFEFE093AB09A091C409E2
:1065C800A033F8F00E945173A091AA09A630C8F42C
:1065D800E091AB09EF5FE093AB09E091AA09EA9378
:1065E800E091AB09EA930E94081CA091A70DB09115
:1065F800A80D109721F4A091AB09A03408F001C0B0
:10660800E7CFE091AB09EA930E94E5190E945D7318
:10661800EAEEF9E10E9452720E940F6E0E94E46C49
:106628000E9462730E94186E0E94777A0E946273B9
:106638000E94B36E0E947E3D0E94C73DE091C20950
:10664800E434A1F5E091C309E43481F514E0E1E014
:10665800E093C10A103538F40E94856CE054F64F77
:10666800E081E03208F41AC00E94856CE054F64FCD
:10667800E081E33259F40E94856CEF53F64FE081D4
:10668800E053EA930E949C381F5F06C00E94856C05
:10669800E054F64F0E9496711F5FDCCF0E945D7335
:1066A800EDEEF9E10E9452720E94C73D8AC41A9326
:1066B8000A930E94747111F40C94C533E0E0E093DE
:1066C800EA0DE091A109EF770E2F0093A1090E942E
:1066D80092510E94506E0E94D56C013021F0A09119
:1066E800A209A13009F00BC0EAEBF4E00E94926C19
:1066F800E2D90E94B76D0E94C4630E94925107308C
:1067080049F40E942222E0E0E093A4090E949D112E
:106718000E949929043031F4E0EFF9E10E94926C6B
:106728000E943B0E083019F40E9468735AD1053054
:1067380019F40E94687355DC013039F40E947573AE
:106748000093A20981D90E948F0F093059F40E9441
:1067580075730E948F0F0A93E1E0EA9318D9E1E07C
:10676800E093EA0D023029F40E946873E1E0EA93AD
:10677800B2DB033011F40E9420610093A2090E9449
:10678800BA20A091A209A73011F00C947234E091BC
:10679800E30DF091E40D0E948C6D0E943268E030A8
:1067A80021F0A091A409A03009F00AC00E94067245
:1067B800E091DF0DA0910808EA1711F00E949929CD
:1067C8000E94A663E030E9F0E2E00E94D4721A93D6
:1067D80067DA1D3409F4ABD81D3399F40E94AF5021
:1067E8008CDAEF3F41F0E3E0E093A1090E94DB720D
:1067F8000E94017306C0E7E8E093A109E0E0E09396
:10680800A409A091B709A03031F0E091B709A0918F
:10681800B609EA1709F453C0E091B709E150EA93C1
:106828000E944A1AA091BD0DE1E0EA23E13021F46B
:10683800E0911008EF7C09F429C0E0E0E093B60984
:10684800E091DD0DE03019F0E093A1091EC012E0DF
:10685800E0911008EC7009F018E0E0914D0DA0915E
:10686800B709EA1781F0E0911008E07439F011E0F7
:10687800EAE2EA93E5EFF9E10E945773E091100824
:10688800E07809F019E01093A10919C00E9492510B
:106898000E949D110E94506E0E94D56CEBE4EA9311
:1068A8000E940051E091B709EA930E940962E8EF5B
:1068B800F9E10E94926CE091B709E093B609A091C2
:1068C800B709A03021F4A091B609A03009F406C098
:1068D800E0E0E093B609E7E8E093A109A091A209F6
:1068E800A33011F40E941F5FA091A209A13009F4FE
:1068F80039D9A091A209A23009F409DBA091A20913
:10690800A83009F41DDCA091A209A53009F495DB93
:10691800A091A209A93009F425D9099119910895DE
:106928000E94316EED59F64FA6E0A0830E94316EA9
:10693800EE59F64FAB81A0830E94316EE859F64FAD
:10694800AA81A0830E94316EEC59F64FA881B981C3
:10695800A083B1830E946E710E94744324960895A7
:106968000E948073A881B981AC91A53020F0A881DC
:10697800B981E0E0EC938BC0A0919C09BB27E09122
:106988009B0905C0A0919A09BB27E0919909F0E0FD
:1069980031960E94F56F3596DF01E5E0F0E00E9440
:1069A800217A08951A9310919C09E0919B09E117A7
:1069B800A9F0ABE01A9FF001ED59F64FE081E13004
:1069C80011F0E23019F4E1E00C94183AEDB7FEB793
:1069D800FA93EA931F93C4DF1F91E7CFE0E00C948A
:1069E800183A1A930E942222E7EDF7E00E94BC6F42
:1069F800E1E2F0E00E946E6F10E0133068F40E944C
:106A08002B70AFEFA083ABE01A9FF001E352F84F71
:106A18000E9401721F5FF1CF10E0113048F4A7E126
:106A28001A9FF001E75EF74FAFEFA0831F5FF5CF26
:106A3800E0911008E37019F00E949D7209F402C0F9
:106A4800689401C0E89421F8EFEFE093B509E0916C
:106A58006B0DE03029F41DD06CD1E89420F804C007
:106A68000E9492510E94C40F0C94183A1A9310E095
:106A7800133058F40E942B70E081AE2FE981EA1799
:106A880011F4E12F03C01F5FF3CFEFEF18812296B7
:106A9800089522970E94467C00E0033058F40E9433
:106AA8008673A0E00E948C73E652F84FA0E0A083A2
:106AB8000F5FF3CF00E00330C0F50E94E571E0817D
:106AC800EF3F89F10E94E571E0810E943A70B9F0C8
:106AD8000E94EB71DF010E94647A0E940870EA1735
:106AE800FB0751F00E94EB710E940870A083B183EC
:106AF8000E949173A1E0A0830E94867312C0ABE04C
:106B08000A9FF001EF51F84FE081E03061F40E94F4
:106B1800E571AFEFA0830E94EB710E9401720E94A1
:106B28009173A1E0A0830F5FC6CF0E94CD1F1E2FD7
:106B38001F3F11F0E1E001C0E0E0E093EA0D1F3FE4
:106B480011F40C94F93550E000E0033048F40E9449
:106B5800E571E0811E1711F451E002C00F5FF5CF17
:106B68005030E1F500E00330C8F50E94E571E0819E
:106B7800EF3F91F50E94E57110830E94EB710E942E
:106B88000870A083B183ABE00A9FF001E552F84F8B
:106B9800A091B20D0E948C73E452F84FFF93EF93CB
:106BA8000E9435700E94466FAF91BF91EC930E948E
:106BB8009173A1E0A0830E948673A1E00E948C7368
:106BC800E152F84FFF93EF930E942668AF91BF916F
:106BD800ED93FC9351E002C00F5FC5CF503029F010
:106BE8001A930E94D41F1E2FAACF30E0313010F024
:106BF8000C943F36A7E13A9FF001EC5EF74FEE8325
:106C0800FF8350E000E0033048F5503029F5ABE051
:106C18000A9FF001E452F84F20812A930E94E51957
:106C28000E948673E081E13059F42A930E9418216A
:106C3800E13031F4A32FAF5FE091260DEA1709F098
:106C48000BC0E22FAE81BF811396EC93E02FAE818B
:106C5800BF811596EC9351E00F5FD5CF503049F4C2
:106C6800AE81BF811396EFEFEC93AE81BF8115968D
:106C7800EC933F5FBBCF0E944D7C289608950E94FD
:106C8800487CAC81BD81EBE4EC93EC81FD813196CD
:106C98000E949773E552F84FE0810E94A27300E0CA
:106CA8000E94AC73EC91E03011F00F5FF9CF0E94B5
:106CB800AC73E0E2EC930F5F0E94B2730E9497738B
:106CC800E352F84FDF010E94647A0E94E46C0E944C
:106CD800B973EE81ABE0EA9FF001E452F84F1081FE
:106CE8001A930E94E51900E00E94AC73EC91E03021
:106CF80011F00F5FF9CF0E94AC73E8E7EC930F5FD8
:106D08000E94AC73E0E2EC930F5F30E03A3050F44D
:106D18000E94B2730F01A3E1BDE00E94BE730F5F32
:106D28003F5FF4CF0E94AC73EC930E944F7C279690
:106D3800089564970E94487C00E010E0133040F406
:106D48000E942B70E081EF3F09F40F5F1F5FF6CFC1
:106D5800033021F0A091B509A03009F406C0E0E0A5
:106D6800E093B509EA930E94DF1010E0133088F52C
:106D7800ABE01A9FF001E652F84FE081E03039F1BC
:106D88001A9FF001E852F84FE081E030B1F01A9311
:106D9800FE0135960E94F171ABE01A9FF001E452B2
:106DA800F84F30813A930E94E5191A93FE013596FF
:106DB800FA93EA930E9414110AC01A930E940311CD
:106DC800ABE01A9FF001E652F84FA0E0A0831F5FE6
:106DD800CDCF033021F4A091B509A13009F406C044
:106DE800E1E0E093B509EA930E94DF100E944F7C2E
:106DF800689608950E94467CA0916B0DA23009F414
:106E0800E0C030E0343168F40E94C5730E94C97351
:106E1800DA011296E0E0EC93DA01EFEFEC933F5FD2
:106E2800F1CF0E94CD1F0E2F0F3F11F0E1E001C0FE
:106E3800E0E0E093EA0D0F3FA1F10E943570FA936C
:106E4800EA930E9499191E2F1F3F31F1A091A709BB
:106E5800E12FEA1B3E2F3431F8F40E94C5730E94DB
:106E6800C973FA0132960F01E081AE2F0E94CF73E9
:106E7800B0E0EA0FFB1FD001EC93FA01A281A4361F
:106E880020F0DA011296E3E6EC93DA01AC91AF3F19
:106E980019F4E02FDA01EC930A930E94D41F0E2F05
:106EA800CACF0E94D21530E0343110F00C94E53787
:106EB8000E94C5730E94C973FA01A381AF3F11F400
:106EC8000C94E3370E94D4730E943C6FE83139F484
:106ED8000E94D473EA930E94D218E03009F408C0E3
:106EE8000E94D473EA930E94D218DA011296EC93A6
:106EF800A091230DA07839F4FA010280DA011196E5
:106F0800EC91E01509F45BC0DA0113962C91ADE021
:106F18002A9FF001E45FFA4F0F01DA011296EC9113
:106F2800D001EC930E94D473EA930E943822EF3F79
:106F380041F0ADE02A9FF0010E94A570E058DB0106
:106F4800EC93DA011296EC91E03089F00E94D97343
:106F5800DF010E94DF73EC93ADE02A9FF001E75F49
:106F6800FA4FDF01E091210DEF70EC9313C00E94FE
:106F7800DF73E03021F40E94D973A0E003C00E94BF
:106F8800D973A8E0A083ADE02A9FF001E75FFA4F2C
:106F9800A7E0A0830E94D473EA930E943822EF3FAF
:106FA80019F0ECE0E0930A06DA011296EC91DA01A6
:106FB8001196EC932A93E1E0EA930E94F6513F5F21
:106FC80073CF0E944D7C26960895E7E0E093A109CF
:106FD8000E942219A8950E94951DA8950E94E91F54
:106FE800A895EFEFE0933B0DE093120DE093BC0DF5
:106FF800E093B70DE09313080E94E473EC7F29F047
:10700800A8E0B0E0E0E00E94A67A0895AC81A03341
:1070180010F0AA3308F006C00E94E973E0530E94FA
:10702800F17399C4AC81A13410F0A73408F006C0FC
:107038000E94E973E7530E94F1738DC4A881B98156
:10704800E0E0EC9388C4AA93EA93FA93EFB7EA9343
:107058001A930A931BB10CB1E091230EF0E0EF50A4
:10706800F24F0083A091230EAF5FA093230EA233AB
:1070780019F4E0E0E093230E09911991F8C21A93EC
:10708800E091240EA091230EEA17D1F3F0E0EF501F
:10709800F24F1081A091240EAF5FA093240EA2336B
:1070A80019F4E0E0E093240EBEC1A091230EAE5C7B
:1070B800E091240EAE1BE2E30E941E7A08950A9224
:1070C8001A92FA926A937A938A939A93AA93BA93A2
:1070D800EA93FA93EFB7EA930E94F67349F0A09106
:1070E800C10AA03021F00E94210EE13009F401C04C
:1070F80011C0E0918A0EF0E0EB5DF14FE081ECB950
:10710800A0918A0EAF5FA0938A0EA43619F4E0E02E
:10711800E0938A0EE991EFBFF991E991B991A991AC
:107128009991899179916991F99019900990189597
:107138001A930E94F67359F45D9B09C0A091C10A85
:10714800A13021F40E94210EE03009F013C0109103
:10715800890E0E94856CEB5DF14FA981A0831F5FAA
:10716800143609F410E0E0918A0EE117E1F3109368
:10717800890E02C0E981ECB91881E8C40E94F6734F
:1071880021F40E94210EE13009F001C01CC354C152
:107198000E94487C8ADFE03011F40C94CE396FDF0E
:1071A8001E2FA091EE0DA53618F0E0E0E093C20A7C
:1071B8003091C20AE091C20AE03011F00C943539DE
:1071C800A0916D0DA13041F0A0916D0DA23021F07C
:1071D800A0916D0DA53031F4E12FEF77E093C80A47
:1071E800EBE4CEC01A3521F4E1E0E093C20ACAC04C
:1071F800123049F4E4E1E093C20AE0E0E093C30A04
:10720800E093C50ABFC0A0916D0DA33069F417378C
:1072180029F01A3310F4103308F402C0E7E001C073
:10722800E0E0E093C40A05C01A930E948240E0930C
:10723800C40AA091C40AAF3F99F01093C80AE1E0CC
:10724800E093C30A1093C50AE091C40AE03011F430
:10725800E5E404C0EAE0E093C20AE0E0E093C70A8C
:1072680091C0E13069F4103039F4E2E0E093C20AE9
:10727800E0E0E093C70A03C0E0E0E093C20A82C0FE
:10728800E23059F41093C40A1093C50AE0E0E09381
:10729800C30AE3E0E093C20A75C0E330F1F40E9448
:1072A800FC730E940274EA0F0E940C74A9F4E09126
:1072B800C50AE03071F4E4E0E093C20AE091C30A41
:1072C8000E94E26E0E9415740E94FC73A0E0A083E5
:1072D80003C0E0E0E093C20A55C0E43049F41D3031
:1072E80019F4EAE5E093C70AE0E0E093C20A4AC06D
:1072F800EA3079F40E94FC730E940274EA270E9423
:107308000C7431F4E0E0E093C20AE5E4E093C70AC4
:1073180039C0E431B9F40E94FC731083E12FA091C5
:10732800C50AEA27E093C50AE091C30AEF5FE09334
:10733800C30AE0E0E093ED0D133019F4E5E1E093C2
:10734800C20A20C0E53111F0E63159F41A93EDEE86
:10735800FDE0FA93EA93E2ECFAE0FA93EA9356DE58
:1073680011C0E73179F4E0E0E093C20A173131F453
:10737800E091ED0DA091C50AEA1709F003C0E3E416
:10738800E093C70AA091C20A3A1719F0E0E0E09327
:10739800EE0D00CF0E944F7C38C4AA93BA93EA93AB
:1073A800FA93EFB7EA931A930A9310919B0000910E
:1073B8009C00E12FEC71A9F4E091530FF091540F68
:1073C800E557F14F0083A3E5BFE00E94B16DE83CAB
:1073D800A0E0FA0731F4E0E0F0E0E093530FF09317
:1073E800540F09911991E991EFBFF991E991B99178
:1073F800A99118951A930E941A740E941F74D9F3C0
:107408000E941A74E557F14F1081A5E5BFE00E946C
:10741800B16DE83CA0E0FA0731F4E0E0F0E0E09379
:10742800550FF093560FE12F199108950E941A7481
:107438000E941F7409F0C7C1E0E008950E94487CCB
:10744800F5DFE03021F0A091EC0DA03009F0E5C0A7
:10745800D1DF1E2FA0915F0FA53618F0E0E0E09372
:10746800590F3091590FE091590FE03059F411300C
:1074780019F4E4E0E093590F1A3519F4EAE0E093BF
:10748800590FC3C0E430C1F4E0E0E093590F1A3259
:1074980029F00E94536EE05DE11769F41093C0096A
:1074A80010935A0FE5E0E093590FE0E0E093EC0DFC
:1074B800E1E0E0935C0FA9C0E530A9F4E0E0E093D7
:1074C800590F0E94536EE05DE11761F00E94267427
:1074D8000E942F74E0915C0FEF5FE0935C0FE6E091
:1074E800E093590F92C0E63091F4E0915C0F0E944E
:1074F8002F740E942674EF5FE0935C0FE0E0E09346
:107508005D0F133019F4E7E0E093590F7EC0E730C0
:1075180011F0E83059F41A93EDE5FFE0FA93EA9395
:10752800E9E5FFE0FA93EA9371DD6FC0E93081F491
:10753800E0E0E093590F173131F4E0915D0FA0912D
:107548005A0FEA1709F003C0E4E5E093EC0D5DC0BB
:10755800EA3041F4103011F4EBE001C0E0E0E093D0
:10756800590F53C0EB3071F4E0E0E0935C0F1093D7
:107578005B0F10935A0FECE0E093590FE0E0E093B3
:10758800EC0D43C0EC30A1F5E0915C0FF0E0E8535E
:10759800F54F10830E942674EF5FE0935C0FE09133
:1075A8005B0FE150E0935B0FA0915B0FA03021F4DB
:1075B800A0915A0FA03009F00EC0EDE0E093590FEA
:1075C800E0915C0F0E94E26E0E941574E0915C0FDE
:1075D800F0E00E941574A0915B0FA03021F4A091F7
:1075E8005A0FA03009F403C0E0E0E093590F0DC032
:1075F800ED3059F4E0E0E093590F1D3031F4EAE53D
:10760800E093EC0DEFEFE093EB0DE091590FE317EA
:1076180019F0E0E0E0935F0F13CF0E944F7CF5C2B2
:10762800AA93EA93FA93EFB7EA93E0916110A091D5
:107638006010EA1791F0E091BF09E03019F0E89482
:1076480026F80AC00E943474F0E0E030A1E0FA079E
:1076580019F4E0E0E093611003C0E89425F826F8F7
:10766800E091EB0DE03019F0E0E0E093590FE9917B
:10767800EFBFF991E991A99118951A93E0916110DA
:10768800A0916010EA1721F4E0919B00E072C1F428
:10769800E0916010F0E0E05AF04FA981A0831091CA
:1076A80060101F5F0E94836BA030E1E0BE0709F401
:1076B80010E0E0916110E117E1F31093601003C04E
:1076C800E981E0939C00188141C2E0E0E0936110F9
:1076D800A0916010A13020F00E943474689426F8BC
:1076E8000895AA93BA93EA93EFB7EA93E091EB0D62
:1076F800E03041F4E0E0E09361100E94536EEF5FE8
:10770800E093BF09E991EFBFE991B991A991189563
:107718000E94427418F00E94467409F403C00E9443
:107728004E73F6CF0E94467411F40E944E7308956A
:107738000E946072AC91E881EA1729F40E944E73A6
:107748003197E1E01EC2E0E01CC20E94487C00E0E4
:1077580010E0EEE20E944A74F1F420E030E0EC819F
:10776800D9010E944F74BCF4D8010E9453748F0150
:107778000E94587418F00E945C7408F009C00E94B6
:107788006072EC910E94F4720E0F1F1F0E944E73DC
:107798002F5F3F4FE4CFF801DCC00E94427420F015
:1077A8000E946074E03208F410C00E946072EC918C
:1077B800E093CA0C0E944E730E946072EC91E093B1
:1077C800CB0C0E944E73E1E0089536C41A930A93D5
:1077D80000E010E0123088F40E946674EF3F59F020
:1077E800E02FE295E07FEF930E946674AF91EA0F75
:1077F8000E2F0E944E731F5FEDCFE02FCDC31A935B
:107808000A9310E00E9460720C910B3311F0003261
:1078180008F412C0013310F0093308F007C0E02F54
:107828000E94F472E255FF4FE4911E2B0E944E73A2
:107838000E9460720C91E9CFE12FAEC30E94487C90
:1078480000E010E00E946072AC91AD3221F40E9419
:107858004E7331E001C030E00E94587418F00E9465
:107868005C7408F009C0D8010E9453740E946B74BC
:107878008F010E944E73F0CF303021F4F8010E943E
:107888004F7CC3C1F8010E945E790E944F7CBDC144
:1078980024971A93E0E0E983EA83EB83EC830E9460
:1078A8006072AC91AD3221F40E944E7311E001C0B8
:1078B80010E00E94587418F00E945C7408F022C00E
:1078C800A981BA818B819C81EAE0F0E060E070E0F8
:1078D8000E94C9797F936F93FF93EF930E94607220
:1078E800EC91E053AF91BF918F919F91FF2766274D
:1078F80077270E945979E983FA836B837C830E94F6
:107908004E73D7CF103031F4E981FA816B817C81D5
:10791800188121C0E981FA816B817C810E9462799A
:10792800188119C00E94487C20E030E000E010E097
:10793800EC81D8010E944F745CF4D9010E94537401
:107948000E946B749F010E944E730F5F1F4FF0CF10
:10795800F9010E944F7C259608950E94487C6EDFAD
:107968008F0120E030E0EEE20E944A7411F466DFF5
:107978009F01112322F4F9010E945E799F01A091D1
:10798800A40DA13030F0D8010E946571E20FF31FF9
:107998008F01F8010E944F7C38C11A9310E00E94B1
:1079A8007074A1F00E94427458F00E946072AC9109
:1079B800A23231F00E94467419F0E9811E1708F0CE
:1079C80005C00E94856C0E947674ECCF0E94856C7D
:1079D8000E947F741881BAC0E8810E9484740E9452
:1079E8008974E881A091E40CEA0FE093E40CE88143
:1079F800A091E50CEA27E093E50CC3C01A9310E0C8
:107A08000E948D74E03029F00E948D740E94957454
:107A1800F7CF1881E4C31A9310E00E949A74E030FB
:107A280029F00E949A740E949574F7CF1881D7C3E1
:107A38000E94A1740E94A674E88DF98D0E94E46CDE
:107A48000E94B9730E94AB74669608950E94A1744F
:107A5800E9E0FAE1FA93EA93E88D0E94A2730E94A2
:107A6800AB74659608951A93ECE3EA93B5DF11E0D9
:107A7800193080F40E94856CE255FF4FE491A9818A
:107A8800EA2319F0E12FE05D01C0E0E2EA93A4DF08
:107A98001F5FEECFEEE3EA939FDF188157C064972C
:107AA8001A930E94B0740E94A674EA8DFB8D0E94FE
:107AB800E46C0E94B9730E94B0740E94C4681E2FBF
:107AC800ED891E1720F4E0E30E949574F9CF0E9417
:107AD800B074A1DF18810CC00E94A1740E94A67422
:107AE800E88DF98D6A8D7B8D0E94B5740E94AB7408
:107AF800689608950E94B8740E94BC748CDF0E9436
:107B0800B87424C0A881B981E4E6F0E00E94EF7956
:107B18000E94C174EEE2EA935FDFA881B981E4E6CE
:107B2800F0E00E94217A0E94C574B9DF0FC0A091CD
:107B3800A40DA13020F00E94BC74E4DF07C00E94AD
:107B4800BC7476DFEEE0FAE10E9452722296089544
:107B580025FE06C0E5E0F0E00E944C6EA895F8CF3F
:107B6800E0E6FFE0E093E60CF093E70CE1E00E942A
:107B7800A171E093E40C0E94CA740E94536E0E94A3
:107B8800CE74219608951A930A93E091EB0DE03094
:107B980009F002C2E3E0EA931FDFE091E40CE2950A
:107BA800EF70EA930E9415681E2FE091E40CEF70C5
:107BB800EA930E9415680E2F1A930EDF0A930CDFC2
:107BC800E7E1EA9309DFE0E6FFE00E9484740E949F
:107BD800877AEA1BE0936010689425F8DDC1EE818E
:107BE800EA93B6DFEC81FD810E9452720E94D27442
:107BF80073DFC9DF27960895EB81EA93A9DF0E9416
:107C0800AF70FCDE0E94CA74BEDF24960895ED8131
:107C1800EA939EDFEB81FC810E945272EA81EA932B
:107C2800DBDEE981E03011F0EA93D6DEE881E0306E
:107C380011F00E94CA74A7DF269608950E94467C18
:107C480010E0E2E1FAE1A885B985EA17FB0719F423
:107C580044E150E002C048EC50E0EA85E093C00AF5
:107C6800E89431F8EA930E94D974EA85EA93EA85A0
:107C7800EA93E0E0EA93CBDF0E9426689F010E9426
:107C8800DB150E94DE740E9432680E2F31FC02C0A0
:107C9800003009F001C0F3CF31FE04C0E89431F898
:107CA800E1E004C01F5F1230C0F2E0E00E944D7CAA
:107CB8002B9608951A930A93E091C80BE03009F4C3
:107CC8006BC1E0E0E093C10AE2E0EA9331DA10E048
:107CD80003E00E94856C0E94E37461F00E94856C49
:107CE8000E94E8740E94856CE853F44FE0810E27E7
:107CF8001F5FEFCFE3E0EA931BDAE02FE295EF7026
:107D08000E94EB74E02FEF700E94EB74E7E1EA93B6
:107D18000FDA42C11A930A93E091C80BE03009F4D4
:107D28003BC10E945D6EE03021F0E091CA0BEA325F
:107D380009F405C00E945D6EE05DE093CA0BE0E0C7
:107D4800E093C10AEAE5EA93F3D9E0E0EA93F0D9CF
:107D580010E00E94856C0E94E37411F01F5FF9CF58
:107D68001F5F012F0A93E4D910E00E94856C0E94DE
:107D7800E37461F00E94856C0E94E8740E94856C2F
:107D8800E853F44FE0810E0F1F5FEFCFE02FE1952E
:107D9800EA93CED9EDE0EA93CBD9FEC01A930A93C1
:107DA800F894E0E0E093BF09E0916110E09360107F
:107DB8007894E091C80BE03009F4EEC0EAE5EA9364
:107DC8005CDCE0E0EA9359DC10E00E94856C0E94DC
:107DD800E37411F01F5FF9CF1F5F012F0A934DDC89
:107DE80010E00E94856C0E94E37479F00E94856C13
:107DF800E853F44FE081EA9340DC0E94856CE85335
:107E0800F44FE0810E0F1F5FECCFE02FE195EA936E
:107E180034DCEDE0EA9331DCBFC0E881EA9398DE18
:107E2800EAE5EA93D9DDE091C80AEA93D5DD0E9434
:107E38006072EC91E03041F00E946072EC91EA933C
:107E4800CBDD0E944E73F3CF9EDE48C41A930E9486
:107E58009A71E091C309EA93BFDDE4E4EA93BCDDDB
:107E6800E091C109EA93B8DD14E00E94856CE05402
:107E7800F64FE081E43040F00E94856CE054F64F04
:107E8800E0810E949574F1CFE0E0EA93A5DD42DF3E
:107E980033C11A930A937CD9E091C70AE03011F4F0
:107EA8000C94C93FA091C70AAA3541F4A091C30A0E
:107EB800A33020F0E091C90AE43409F04BC00E94D5
:107EC8005D6EE03021F0E091CA0AEA32C1F40E9406
:107ED800536EE05DA091CA0AEA1721F0E091CA0A40
:107EE800EA3221F40E94874F15DF08C0EBECFAE074
:107EF8000E946C72E091CA0A0E94F1742BC00E9421
:107F08005D6EE05DA091CA0AEA1721F50E94536EE2
:107F18001E2FE091CB0AED3421F4E091CC0AE33234
:107F280009F007C0EDECFAE00E946C7287DC1E2FA6
:107F3800EFDB0E94536EE11729F0E12FE05D0E940C
:107F4800F17408C00E94536EE05DE093CA0A0E9473
:107F5800874FE0DEA091C70AA53441F4A0916D0DCA
:107F6800A33019F40E94032C01C03BD1A091C70A89
:107F7800A33411F40E94B42BA091C70AAB3411F4B6
:107F88000E94AF2BE0E0E093C70AA0916D0DA330EB
:107F980011F40E94032CE0E00991199108954EDA3A
:107FA800A091EC0DA43529F4A0E025FCA1E0A030B7
:107FB80009F038C0E091C209E03581F4E091C309C5
:107FC800EA93E6E0EA930E949463A091C309A0387B
:107FD80020F0E091C309E093600721C0E03721F465
:107FE800E0E0E09360071BC0EA3519F40E940450F2
:107FF80016C0EA3711F42ADF12C0E23511F4FDD2B7
:108008000EC0E23711F429D30AC00E949F31E091D3
:10801800C109A091C00AEA1711F4689431F8E0E0A8
:10802800E093EC0DA091EC0DAA3531F40E94874F36
:10803800B5DEE0E0E093EC0DE0E00895A091EF0DEF
:10804800A13050F0E091EF0DE150E093EF0DE030FA
:1080580019F4E1E0E093F00DA0E025FCA1E0A130E7
:1080680049F4A0E026FCA1E0A03021F4A091BF09CA
:10807800A03009F001C029DBE091BF09E03019F018
:10808800E150E093BF090895E0915F0FEF5FE0933F
:108098005F0FE091EE0DEF5FE093EE0DE091EB0DD9
:1080A800E03019F0E150E093EB0D0895A0916D0DCB
:1080B800A13041F0A0916D0DA23021F0A0916D0D7D
:1080C800A53029F4E1E0E0939000ECE9E9B90895DE
:1080D8001A93EFEF0E94A171E093C10A10E00E9489
:1080E800856CE853F44FE081EF3F31F00E94856CD6
:1080F8000E94E8741F5FF3CF199108951A930A93A9
:108108000091580DAA81A53411F4E0E066C0AA8157
:10811800A23539F4A091BD09A13019F40E94F87470
:1081280009F405C00E94821DE0E0E093BD09AA8120
:10813800AB3411F0A33599F4E02FE470E43011F476
:1081480014E001C013E0E02FE270E23009F41C5F94
:10815800E02FE170E13009F41F5FE12F3EC0AA81F2
:10816800A13511F0A13799F4E02FE470E43011F44F
:1081780017E001C016E0E02FE270E23009F41C5F5E
:10818800E02FE170E13009F41F5FE12F26C0AA81DA
:10819800A33421F0A13411F0A23441F413E0E02F0C
:1081A800E170E13009F41F5FE12F17C0AA81A737FA
:1081B80041F417E0E02FE170E13009F41F5FE12F8F
:1081C8000CC0AA81A03441F415E0E02FE170E13041
:1081D80009F41F5FE12F01C0EFEF19810881239691
:1081E800089524970E94467C2091580DA091C80AB2
:1081F800A53411F00C94BA41E0E0E093BD090E9467
:108208009A71E0E0E093E50CE0915C0DE03089F5CF
:10821800E0919909A0919A09EA1739F00E94FE7431
:10822800E45DF64FE081E13009F023C0E7E7EA9327
:10823800D3DB0E94FE74EF5CF64F0E94D770FA936E
:10824800EA930E940475E35DF64FDF010E944973CB
:108258000E940475EE5CF64FE0810E94CE74E2E065
:10826800E093BD090E94FE74E45DF64FA2E0A0838E
:108278002FDFE091BD09E03011F00C94BA410E9463
:10828800F87411F40C9496410E94771DE1E0E09394
:10829800BD09E22FE870E83079F40E940975E8EE2C
:1082A800F3E00E94EF79DF010E943C7C14F4E1E3E3
:1082B80001C0E0E3EA9390DBE22FE074E03411F4CC
:1082C80013E001C012E0E091AD0D0E940E751A9303
:1082D800E6DBE22FE470E43049F40E940975E0E13E
:1082E800F7E20E94217AAF0114E006C00E940975E6
:1082F8000E94EF72AF0113E0E22FE071E03111F458
:10830800415050405A934A931A93C9DBE22FE072C6
:10831800E03211F414E001C013E0E091B00DF091E7
:10832800B10D17C018E0E22FE470E43009F41F5FC4
:10833800E22FE870E83009F41F5FE22FE072E032C4
:1083480009F41F5FE22FE074E03409F41F5FE0E0F6
:10835800F0E0FA93EA931A93A2DBE22FE170E1309E
:1083680021F4E091E50CEA9337DBB2DEA091C80A6C
:10837800A73729F4E2E0E093BD09E03009F473C0BF
:108388000E949A710E9412750E9456721E2F0E94B6
:108398007172AF01E1E0EA93C5DA0E2FE091990915
:1083A800A0919A09EA1739F00E94FE74E45DF64F2D
:1083B800E081E23009F054C00E94FE74E35DF64F9C
:1083C800DF010E94647A4E175F0711F00C94304267
:1083D8000E94FE74ED5CF64F008011800E94536E7F
:1083E8000E942771EA17FB0771F10E94FE74ED5C89
:1083F800F64FDF010E94647A0E9418750E94FE748D
:10840800ED5CF64FDF010E94647AE351F34FE0819F
:108418000E9420750E9427750E94856C0E94C17475
:108428000E942A75E9E1FAE10E945272003021F0B7
:108438005A934A93FDDA03C0E0E3EA93CDDA0E9447
:108448002A75A1DB09C0003039F00E942E7520F48E
:108458000E943E730E947D27EAE9F9E00E94357583
:10846800E0E0E093BD09A091C80AA33421F40E947A
:10847800C034E03009F40BC00E949A710E94127552
:108488000E9439750E94326B43D30E94241EA0912A
:10849800C80AA13411F0A23421F40E949A710E94F2
:1084A8001275A091C80AA03421F40E94C034E030AB
:1084B80009F41FC00E945672E887F987E2E0EA9340
:1084C80031DA1E2F1A930E94D9740E943B190E9418
:1084D800316E0E943D75E859F64F10830E94316E47
:1084E800ED59F64FA7E00E94376E0E949A710E94DC
:1084F8001275A091C80AAB3439F0A33529F0A1351B
:1085080019F0A13709F075C00E94C034E03011F4A9
:108518000C94F7420E949A710E944475E9ECFAE0C3
:108528000E946C72E22FE270E23021F4E4E0EA93F8
:10853800F9D902C0E1E0F0E0E887F987A091C80A1C
:10854800A13511F0A13721F40E9471721E2F02C0CB
:1085580010916E0DE22FE470E43011F4E4E001C0F4
:10856800E3E0EA93DFD9AF01A091C80AA33511F07F
:10857800A13731F4E885F9850E945E79E887F987A3
:108588000E942E7520F0A0915C0DA13019F51A9368
:108598005A934A93EB85FC85FA93EA930E94431E0B
:1085A800FA93EA930E942A6BEE83FF83AE81BF8120
:1085B8000E943C7C7CF40E949A71E6E6EA930CDA0D
:1085C800EE81FF813197EE83FF83AE81BF810E94E8
:1085D8003C7C9CF31A935A934A93EB85FC850E9442
:1085E8002C7276DD06C00E9439750E94326B0E949B
:1085F800431E0E944D7C2A9608950E944875E8946F
:1086080022F80E945D73E2E7EA93E6D9E091C30994
:10861800EA93E2D9EFE0EA93DFD9A091C009AA3240
:1086280019F41A934FD318C0A091C3090E94856CFE
:10863800E351F34FE081EA1721F4E091C309E033F5
:1086480049F40E94836BA351B34FE091C309EC93A3
:108658001A9338D322FE97DAA9C20E944875E0918E
:10866800C309E053AE2F0E94856CE250F34FE081BE
:10867800EA1741F51A9326D3A091BE09A23019F43E
:108688000E94507509F402C00E945675A091BE0957
:10869800A33019F40E94507509F402C00E9456755F
:1086A800E0E0E093BE09E09364100E94856CE2501C
:1086B800F34FBF01E081EF5FAE2FEAE00E941E7A20
:1086C800DB01EC9373C2E881E03021F4E0E3EA9344
:1086D80083D904C0E881E8500E945975219608950D
:1086E8000E94467C25FC10C20E94507511F40C941F
:1086F800D2440E945B75EE59F64F9F01D90111963D
:10870800EC91E43039F50E9461750E946E75F901AB
:10871800A681A03021F4A281B381109709F007C087
:10872800ECE1FAE10E9452720E942A7510C00E9480
:1087380027750E9472750E942A75EFE1FAE10E947E
:1087480052720E9476750E947D750E9481750E9402
:108758008875DAC1E730A9F40E9461750E946E75C8
:10876800E2E2FAE10E9452720E9476750E942A752E
:10877800E5E2FAE10E9452720E9472750E948875C1
:10878800C3C1E93079F40E9461750E946E75E8E210
:10879800FAE10E9452720E948F750E942A750E9407
:1087A8008875B2C1E630F9F4EAE2EA93D1D9EBE28E
:1087B800FAE10E945272D901EC910E94CE74E091C4
:1087C800560D0E94CE74EBE4EA930E94F03C0E949E
:1087D8007275E4E5EA930E94F03C0E947675D3D95D
:1087E8000E94567591C1E530B9F40E942F730E941A
:1087F8001875D901EC910E9420750E9427750E9476
:1088080072750E942A75E9E1FAE10E9452720E948B
:1088180076750E94887578C1E83021F50E946175E7
:108828000E946E75EEE2FAE10E945272F901A68189
:10883800AA930E943B73309719F00E94416F04C0BD
:10884800D9011696EC91F0E0FA93EA930E941C3D48
:108858000E942A7598D9D9011196E0E0EC930E94FC
:10886800567552C1E130B1F5A091A209A53029F49D
:10887800E091560DE65F1E2F01C011E0E12F0E9426
:1088880092750E94856C0E9497750E949B750E9444
:1088980027750E9472750E942A75E1E3FAE10E9429
:1088A80052720E9476750E947D75D9011796EC91D7
:1088B8000E945975A091A209A53049F40E947D75BE
:1088C800F901A481B581BA93AA930E94863D0E94BA
:1088D8009F751AC1E330A1F40E942F73F0960E948D
:1088E800AE750E942F730E9497750E949B75E4E3F2
:1088F800FAE10E9452720E9476750E949F7504C127
:10890800EB3061F50E94B2750E94B5750E949B75A7
:10891800E7E3FAE10E945272F901A681AA93D3DE35
:108928000E947D75F901A781AA93CDDE0E947D750D
:108938000E9481750E947D750E9476750E947D75E2
:10894800F901A481B581BA93AA930E941C3D0E94A3
:108958007D750E948F750E949F75D6C0EC3079F4A2
:108968000E94B2750E94B5750E949B75EAE3FAE110
:108978000E9452720E948F750E949F75C5C0EE308A
:1089880069F40E94B2750E94B5750E949B75EDE36B
:10899800FAE10E9452720E949F75B6C00E94F87454
:1089A80061F0A091BE09A03041F4A0915B0DA13007
:1089B80021F40E94536EE13009F42CC0A0910E0DF1
:1089C800A03071F0E091100DF091110DFA93EA9337
:1089D800E8EEF3E0FA93EA930E943268E130D1F4CA
:1089E800E1E30E94AE75E091FF0C0E94CE740E94F4
:1089F8009B750E94536EEA9316D1E093BE090E94BC
:108A0800C73D0E942668E0936210F0936310E0E08F
:108A1800E0930E0DA091BE09A03051F0E0916210D4
:108A2800F09163100E948C6D0E943268E13009F069
:108A380025C0A091BE09A23019F40E94507509F40E
:108A480002C00E945675A091BE09A33019F40E9475
:108A5800507509F410C0A0916410A33030F00E9442
:108A68005675E0E0E093641006C00E945B75ED590E
:108A7800F64FA8E0A083E0E0E093BE09A0910F0DB7
:108A8800A13011F00C948845E091C20DA091C10D60
:108A9800EA17A9F1EAE20E94AE75E091FD0C0E9486
:108AA800CE740E949B75E091C20DEA930E94DB1F71
:108AB8000E942775E091B20D0E9459750E942A758F
:108AC800E0E4FAE10E9452720E9435700E94C1747B
:108AD8000E947D750E94CF730E94C1740E942A75FE
:108AE8000E94C73DE091C20DEA930E941D1EE091CD
:108AF800C20DEA930E94F01DE093C20D05C0E0E0AC
:108B0800E0930F0D689420F80E944D7C26960895F6
:108B18001A930A930E94C034E030D9F00E94316E53
:108B2800EE59F64F8F01EC81FD81D8011296ED9335
:108B3800FC93EA81FB81D8011896ED93FC93EE81B2
:108B4800D8011696EC93D8011196E4E0EC930E94B4
:108B58006E711981088127960895E091CA0CEA93ED
:108B68000E94F03CE091CB0CEA930E94F03C0895FF
:108B7800F4DF0E94BC740E94B9750E94B9750E9406
:108B88001C3D0E942A759CC01A930E94223C1E2FED
:108B9800103021F0E12FE150E093C80CDEDFE091C6
:108BA800C80CEF5F0E9459750E942A7519910895A3
:108BB8000E94487C31E00E94587428F00E9460723C
:108BC800AC91A43308F02AC030E00E946072EC91A6
:108BD800E270E6951E2F0E946072EC91E1700E2FF4
:108BE800A091E20C1A1729F4E1E0EA27E093E20CDD
:108BF80031E0A091E30C0A1729F0E1E0EA27E093BD
:108C0800E30C31E0E091E30CEE0FE05DA091E20CA3
:108C1800EA0FEA930E94F03C0E944E73E32F0E94F1
:108C28004F7C249608951A9310E00E94F87411F46A
:108C38000C9462460E94771DE4E4FAE10E945272A5
:108C4800E091AD0D0E9459750E942A75E7E4FAE19A
:108C58000E945272E091B00DF091B10D0E94C17462
:108C68000E942A750E940975A031E7E2BE074CF4FC
:108C7800EAE4FAE10E945272E091AE0DF091AF0D74
:108C880016C0EDE4FAE10E9452720E94616CA4E6FB
:108C9800B0E00E94C4790E940975EA0FFB1F0E9488
:108CA800F06FE091AE0DF091AF0DE051F742FA93FD
:108CB800EA930E941C3D0E942A7511E0E12F188159
:108CC8002296089524970E94467C0E94C0750E94AF
:108CD800D13BE13010F40C945549E091CA0CEB34C7
:108CE80041F4E091CB0CE33219F40E94223C1E2F90
:108CF800D5C2E435B9F4E091CB0CE33221F40E94FB
:108D0800223CEE83FF83E091CB0CEF3451F40E94B8
:108D1800223C1E2F1A93EF81F885FA93EA930E945A
:108D28003B19BCC2E23411F00C94EB47E091CB0C38
:108D3800E13251F4AA85AF3F29F40E9439750E94A7
:108D4800326BE6DE0E94241EE091CB0CE134E1F4A4
:108D58000E94223C1E2F113071F4A091BE09A1304F
:108D680019F40E94F87409F402C00E94821DE0E020
:108D7800E0930E0D09C0E1E0E0930E0D0E94266815
:108D8800E093100DF093110DE091CB0CE534A9F4AC
:108D9800E0E5FAE10E9452720E945F1DF3973CF0F1
:108DA8000E94223C0E94F06F0E94C47501C0E0E35B
:108DB800EA930E94F03C0E942A75E091CB0CE634BD
:108DC80039F50E94D07519F40E94223CAF01E8855C
:108DD800F9850E94466F0E2FE0916E0DE03011F07C
:108DE80010916E0D003420F0A0915C0DA13039F483
:108DF8001A930E94D9745A934A930E94431EAA85D3
:108E0800AF3F31F41A930E94D9745A934A9380DE83
:108E1800E091CB0CE23511F00C94A8470E94D07574
:108E280019F40E94223CAF0130E0A0915C0DA03003
:108E380021F40E94536EE13009F027C00E94C63425
:108E4800E03011F10E942072E35DF64FA885B985E4
:108E5800A083B1830E942072ED5CF64FDF01EA85A2
:108E68000E946A710E942072EF5CF64F10830E9484
:108E78002072EE5CF64F40830E942072E45DF64F4C
:108E8800A1E0A0830E9426725DC00E94C034E23037
:108E980010F40C94A6471A930E94D9740E94551F87
:108EA8003E2F3F3F29F00E940870A417B5070CF425
:108EB80012C00E94CF73E41BF50B0E9416700E942B
:108EC800FB7119F4E0E0E093B20D3A930E94E21FBF
:108ED800689420F803C0E0E0E887E9870E94316ED3
:108EE800EE59F64FDF01EA85F0E0E351F34FE081F8
:108EF800EC930E94316E0E943D75E659F64FDF01F2
:108F0800EA850E946A710E94316EE859F64F108313
:108F18000E94316EED59F64FA5E00E94376EE88544
:108F2800F985309779F01A930E94D974FA010E9452
:108F38005E790E942C721A930E94D9745A934A93AC
:108F48000E94D11D689422F8E091CB0CE335F1F52D
:108F58000E94223CE887F9870E945B75DF01ED5982
:108F6800F64FE081E23081F4FD01E659F64F0080CA
:108F780011800E94536E0E942771EA17FB0721F4A3
:108F8800A091BE09A23009F01FC00E945B75EC5980
:108F9800F64FDF010E94647ADF01E885F985EA1758
:108FA800FB0779F40E945B75DF01E459F64FE08115
:108FB800EA93FD01EE59F64FE081EA930E947D277E
:108FC80003C0E7E0E0930908689422F867C1E43435
:108FD80011F00C945148E091CB0CE33559F4E3E5DA
:108FE800FAE10E9452720E94C2380E94CE74E1E0F7
:108FF800E093C10AE091CB0CE03511F00C94504895
:109008000E94707411F40C94504820E00E9442743D
:1090180040F00E946072AC91A23219F00E9446742E
:1090280009F43AC0E22FE03071F40E946072AC910A
:10903800A33211F421E006C00E946072EC91EA9319
:109048000E949C3826C0E13051F40E946072AC91B5
:10905800A43211F422E001C020E010E01AC0E2308E
:1090680011F0E330B1F40E946674EF3F89F0E12F0C
:10907800E295E07FEF930E946674AF91EA0F1E2F8E
:109088002F5F243021F41A930E949C3820E001C0FD
:1090980020E00E944E73BACF01C1E33411F00C9462
:1090A800C148E091CB0CE534B9F4E0E5FAE10E945F
:1090B80052720E945F1DF3974CF00E94223CE05FC1
:1090C800F84D0E94F06F0E94C47501C0E0E3EA9376
:1090D8000E94F03C0E942A75E091CB0CE634D9F44A
:1090E80041E050E00E94223C0E2FEAE30E944A74BD
:1090F80019F40E94223CAF01E0916E0DE03011F0AE
:1091080010916E0D1A930E94CD6BE05FF84D0E948E
:10911800D8750E94431EE091CB0CE335A1F40E9460
:10912800DD750E943C6FE83141F4E091120DEA933D
:109138000E94DE18689420F806C0E885EA93EFEFED
:10914800EA930E947D27E091CB0CE134A9F4E6E58F
:10915800FAE10E9452720E94DD75EA930E94E519B5
:109168000E94B026E03011F0E1E301C0E0E3EA93A9
:109178000E94F03C0E942A7591C0E63511F00C94CB
:109188002C49E091CB0CE33411F00C942B490E944C
:10919800223C1E2F113010F40C942B49A091A209E7
:1091A800A13011F0A930B1F50E94E47521F0A09129
:1091B8002B081A1709F02DC011500E94223CAF014C
:1091C8001A930E9481223E2F0E94BA720E94D27086
:1091D8000F010E94BA720E94D96CE40FF51FD001EA
:1091E800ED93FC930E94E47589F00E94223CAF0144
:1091F8000E94C3720E94D2700F010E94C3720E9423
:10920800D96CE40FF51FD001ED93FC931A930E94DB
:10921800BB111DC01630D8F41150A12FEAE00E94EE
:10922800CE79A3E2EA9FF001EF5CF74FBF01A12FCF
:10923800EAE00E941E7AF0E0BB01AAE0B0E00E94DA
:109248009C79DB01AE0FBF1F14960E94557026C093
:10925800E93421F5E091CB0CE03551F40E94223C31
:109268001E2FE0E0EA931A930E94B819E0931308BE
:10927800E091CB0CEC3491F40E94EA3BE0930D08AA
:109288000E94E47521F00E94EA3BE0930E080E94D8
:10929800E47521F00E94EA3BE0930F080E948C3BA2
:1092A80016CD0E944D7C2B960895A091E00CA03518
:1092B80021F4A091E10CA03408F005C0E091E10C84
:1092C800EA930E940D1AA091E00CA33521F4A09115
:1092D800E10CAA3008F005C0E091E10CEA930E9485
:1092E800401AA091E00CAB3421F4A091E10CA03815
:1092F80008F005C0E091E10CEA930E947E1AA09163
:10930800E00CA63521F4A091E10CA03108F005C0CD
:10931800E091E10CEA930E94AC1AA091E00CA4350C
:1093280011F40E942519C2D60895ECE2F8E0FA93E8
:10933800EA93E091CA0CEA93E0E8F0E00E946E6FCD
:1093480008950E94EA75A0E0A083E091C80CE0931C
:10935800E10CE091CA0CE093E00C08950E94467C71
:109368000E94D13BE13010F40C94DF4CE091E00C0A
:10937800A091CA0CEA1709F098DFE091CA0CE33211
:1093880039F5E091CB0CEC3431F4CFDFE4E0E09335
:10939800A1090E94F075E091CB0CE435C1F4C5DF5A
:1093A800E0916710E03029F0EF77A9E0B0E00E9483
:1093B800A67AE0916810E03029F0EF77AEE0B0E0EF
:1093C8000E94A67A0E94F075E7E0E093A109F0C236
:1093D800E934E9F4E091CB0CE434C1F40E947074F0
:1093E800A9F010E010E0183178F4ACEAB8E00E9477
:1093F800856CEA0FFB1FFF93EF930E94EA3BAF9146
:10940800BF91EC931F5FEFCF0E94280ED1C2EB34BF
:10941800E1F5E091CB0CE13211F487DF35C0E5329C
:1094280011F443DF31C0E33299F40E94F67521F05C
:109438000E9401760E944A1A0E94EA75E081EB3484
:1094480029F4E0E0E093BD0DE093BE0D7ADF1CC087
:10945800E134D1F40E94223C9F012093BD0D0E946B
:10946800077691F00E94223C9F01A091BD0DF90161
:10947800E270F070EA2BE093BD0D0E94077621F0B0
:109488000E94223CE093BE0D93C2E33591F5E09132
:10949800CB0CE13211F449DF2BC0E33299F40E947E
:1094A800F67521F00E9401760E94221A0E94EA7540
:1094B800E081E33529F4E091C80CEA930E94641C2A
:1094C80040DF16C0EE34A1F4EAE0EA930E94D13CF2
:1094D80010E01A3068F4ACE3BDE0EE27A10FBE1F20
:1094E8000E94856CE453F34FE081EC931F5FF1CF4A
:1094F8005FC2E63511F00C94C94AE091CB0CE13219
:1095080011F413DF41C0E33299F40E94F67521F09B
:109518000E9401760E948A1A0E94EA75E081E63567
:1095280029F4E091C80CEA930E94BF1A0ADF2CC004
:10953800E63531F40E94223C9F012093B90D24C0E6
:10954800E53471F40E94223C9F012093B80D0E94DB
:10955800077629F00E94223C9F012093BB0D14C07E
:10956800E43591F440E050E00E94223C9F01022E35
:10957800032A11F042E050E00E94077619F00E9499
:10958800223CAF014093BA0D13C2E43511F00C949C
:10959800954BE091CB0CE33231F40E94223C319799
:1095A800E093C80CBDC0E03511F00C94944B10E06A
:1095B8000E94427450F00E946072AC91AD3329F061
:1095C8000E94467411F01E3008F005C00E94856C98
:1095D8000E947674EDCF0E94856C0E947F74EDE343
:1095E8000E944A7411F00C94944BE4E5E093E00C6B
:1095F80010E00E94856C0E94C96F3496E491EF3F99
:1096080011F40C94944BECECFCE00E94A76C0E94C3
:10961800C96F0E94966C0E949C68E03011F00C940F
:10962800924B0E94856C0E94C96F3496E491E03891
:1096380051F40E94223CE058FF4FE0936710E0E8A5
:10964800E09368106BC0E23839F40E94223CE0587D
:10965800FF4FE093681062C0E13839F40E94223C61
:10966800A8E0B0E00E94A67A59C0E03011F0E130DD
:1096780061F40E94856C0E94C16FFF93EF930E9472
:10968800223CAF91BF91EC9349C0E23069F40E944B
:10969800856C0E94C16FFF93EF930E94223CAF91AB
:1096A800BF91ED93FC933AC0E33061F40E94856C5E
:1096B8000E94C16FFF93EF930E94033CAF91BF914B
:1096C800EC932CC0E43051F50E94856C0E94C96F60
:1096D8003596E491EA930E94D13C0E94856C0E94E1
:1096E800C16FE0936510F093661000E00E94856CEE
:1096F8000E94C96F3596E4910E1780F40E94CD6BD5
:10970800E453F34FE081A0916510B0916610EC939B
:10971800A5E6B0E10E94B16D0F5FE8CF1F5F69CF8A
:1097280047C1E03511F00C94DC4CE091CB0CE332EE
:1097380099F40E94F67521F00E9401760E94E519BD
:109748000E94EA75E081E03529F4E091C80CEA93BB
:109758000E94791CF6DD2CC1E13211F4E6DD28C146
:10976800E134C1F40E94223C1E2F00E00D3088F441
:109778000E940D763396E491E11749F40E940D7624
:109788003296E491A091230DEA2BE093230D0F5F0D
:10979800EDCF0EC1E63559F5E0E0E093C90C0E9423
:1097A8001676EA0FFB1FFF93EF930E94223CAF91BE
:1097B800BF91EC93EBE2EA930E949C3BE03059F0B6
:1097C8000E941C76EA0FFB1FFF93EF930E94223C36
:1097D800AF91BF91EC930E942276A091C90CA3305F
:1097E80018F40E94077609F401C0D9CFE1C0ED341E
:1097F800D1F4E0E0E093C90C0E942876EA0FFB1F41
:10980800FF93EF930E94223CAF91BF91EC930E948B
:109818002276A091C90CA33018F40E94077609F4A7
:1098280001C0EACFC5C0E735D1F4E0E0E093C90C48
:109838000E942E76EA0FFB1FFF93EF930E94223CB3
:10984800AF91BF91EC930E942276A091C90CA230EF
:1098580018F40E94077609F401C0EACFA9C0E434DD
:10986800B9F5E0E0E093C90C0E94223C9F01E2E0D8
:10987800EA930E94A93BAF01E3E70E944A7459F4B6
:109888000E943476BF01D9010E946571E40FF51F6B
:10989800DB01ED93FC93E9E40E944A7469F40E94A9
:1098A8003476208331830E943A76EA0FFB1F0F013A
:1098B8000E943A760E94C6720E942276A091C90C34
:1098C800A33018F40E94077609F401C0CDCF70C008
:1098D800EE34A9F4EAE0EA930E94D13C10E01A3091
:1098E80068F4A3E1BDE0EE27A10FBE1F0E94856CBE
:1098F800E453F34FE081EC931F5FF1CF59C0E33499
:1099080059F4E2E2EA930E949C3B0E94223CE093D5
:109918001E0DF0931F0D4CC0E33589F40E94223CC4
:109928009F0100240216030624F42B30E0E03E07D2
:109938000CF004C0F9013197E093200D39C0E535EA
:1099480029F40E94223CE093220D32C0EF3491F4B6
:109958000E94223C1E2FECE2EA930E949C3BE12FDE
:10996800E295E07FEF930E94223CAF91EA0FE093EB
:10997800210D1EC0E035E1F4E0E0E093C90CA5E359
:10998800BDE00E9440760E94D270FF93EF930E9440
:10999800B13CAF91BF91ED93FC930E942276A091C8
:1099A800C90CA23018F40E94077609F401C0E7CF69
:1099B8000E948C3BD5CC0E944D7C269608950E942F
:1099C800487C0E94D13BE13010F40C94844FE09124
:1099D800CA0CE332A9F4E091CB0CE03519F4E9E5BF
:1099E800FAE109C0E83419F4EAE7FAE104C0E3351A
:1099F80031F4E5E9FAE1FA93EA930E94023D7DC267
:109A0800E934C1F4E091CB0CE43499F40E94270EB8
:109A1800A4D80E94B87410E0183148F4ACEAB8E051
:109A28000E944476EA930E942A3D1F5FF5CF0E9468
:109A3800B87463C2E43511F00C94A54DE091CB0CD9
:109A4800E43221F40E947E6D93D87AC0E33211F497
:109A58009BD876C0E03511F00C94A44D7ED8A09127
:109A6800C80CA83210F00C94A44D0E9449760E94AC
:109A7800966C0E94023DEDE3EA930E94F03C0E943E
:109A880049763496E491E03829F40E94536E0E9496
:109A9800597556C0E23829F40E945D6E0E945975C6
:109AA8004FC0E13829F40E94E4730E94597548C0F8
:109AB800E03011F0E13039F40E944D760E94D77001
:109AC8000E94C1743DC0E23041F40E944D76DF012E
:109AD8000E9449730E941C3D33C0E33039F40E9450
:109AE8004D76E081EA930E94373D2AC0E43041F583
:109AF8000E944D76E0936510F093661010E00E9486
:109B080049763596E4911E1790F40E94856CE453CB
:109B1800F34F0F01A0916510B0916610EC91D00140
:109B2800EC93A5E6B0E10E94B16D1F5FE8CF0E94FB
:109B380049763596E491F0E00E947F740E94517650
:109B4800DCC1E33579F5E091C80CEA930E94221A4A
:109B5800E091CB0CE43229F4EAE0F0E00E94577679
:109B680020C0E33219F40E94C8451BC0EE34C9F482
:109B78000E94B14510E01A3068F40E94856CE453E5
:109B8800F34F0F01ACE3BDE00E944476D001EC93A3
:109B98001F5FF1CFE0E0E093D60C0E9451760E945F
:109BA8002A75ABC1E63511F00C94194EE091C80C3A
:109BB800EA930E948A1AE091CB0CE43229F40E94BD
:109BC800886C0E94BC4530C0E33219F40E94C84535
:109BD8002BC0E53459F40E94B145E091B80D0E94BC
:109BE80059750E945B76E091BB0D19C0E63529F4E2
:109BF8000E94B145E091B90D12C0E435A9F40E9464
:109C0800B145E091BA0DE03011F0E1E301C0E0E3C5
:109C1800EA930E94F03C0E945B76E091BA0DF0E076
:109C28000E94C1740E942A7568C1E03511F00C9435
:109C3800504FE091C80CEA930E94E519E091CB0CD3
:109C4800E43229F4E0E4F0E00E94577624C1E332DC
:109C580019F40E94C8451FC1E13411F00C94764EE6
:109C68000E94B14512E0A091230DECEDEA233E2FAE
:109C780000E00D3068F40E940D763296E491E31707
:109C880029F40E940D763396149102C00F5FF1CF2C
:109C98000E94856C0E94C1740E942A75E091210D72
:109CA800E03089F0E0EBFAE10E9452720E94DF7323
:109CB8000E9459750E945B76E091210DEF700E9419
:109CC80059750E942A75E091220DE03051F0E3EBBE
:109CD800FAE10E945272E091220D0E9459750E9489
:109CE8002A75D9C0E43469F50E945F76A091C90C41
:109CF800A33030F5E091C90CE03011F00E945B769A
:109D08000E943A760E94657661F4ACE2BDE00E945A
:109D180040760E94D96CFA93EA930E94863DE3E765
:109D280009C0ACE2BDE00E9440760E94D96C0E9456
:109D3800C174E9E4EA930E94F03C0E942276D6CFEF
:109D4800A6C0ED34A1F40E945F76A091C90CA3309F
:109D580068F4E091C90CE03011F00E945B760E9433
:109D680028760E946A760E942276EFCF90C0E73567
:109D7800A1F40E945F76A091C90CA23068F4E0912A
:109D8800C90CE03011F00E945B760E942E760E948A
:109D98006A760E942276EFCF7AC0E635E1F40E9417
:109DA8005F76A091C90CA330A8F4E091C90CE0300B
:109DB80011F00E945B760E9416760E946A76EBE2AA
:109DC800EA930E94F03C0E941C760E946A760E94E8
:109DD8002276E7CF5CC0EE34C1F40E94B14510E0B2
:109DE8001A3068F40E94856CE453F34F0F01A3E125
:109DF800BDE00E944476D001EC931F5FF1CFE0E014
:109E0800E093D60C0E94517642C0E33499F40E9444
:109E1800B145ECECFCE0FA93EA93EBEBFAE1FA9348
:109E2800EA930E94416F0E94E46C0E94B9730E94F9
:109E380051762DC0E03599F40E94B1450E94147204
:109E4800FA93EA930E949B3D0E945B76E091370D5E
:109E5800F091380DFA93EA930E949B3D18C0E335C0
:109E680031F40E94B145E091200DEF5F0DC0EF3451
:109E780091F40E94B1450E94DF730E9459750E94B7
:109E88005B76E091210DEF70F0E00E94C174EBE386
:109E9800EA930E94F03C31C0EB3479F5E091C80CAC
:109EA800EA930E944A1AE091CB0CE43229F4E0E8E4
:109EB800F0E00E94577621C0E33219F40E94C845A9
:109EC8001CC0E134D1F40E94B145A091BD0DE1E080
:109ED800EA230E9459750E945B76A091BD0DE3E0CC
:109EE800EA230E9459750E945B76E091BE0D0E949C
:109EF8005975EEEBFAE10E9452720E948C3B61CDDB
:109F08000E944F7C09C21A930E949A71E8ECFAE009
:109F18000E946C720E946074E43471F40E946E7640
:109F280002800E94536EE05DE01529F00E946E7673
:109F3800E281EA3209F401C060C0A6EEBCE00E94EA
:109F4800B16D0E9460740E9484740E9489740E949A
:109F58006E76E2810E9484740E9489740E94607205
:109F68001C910E946E7633960E946C72E12FE2314A
:109F780039F40E9484741397E6E0EC93EFD93DC05E
:109F8800E13139F40E9484741397E2E1EC9317DD10
:109F980034C0EF30B1F40E9484741397EEE0EC9370
:109FA8000E94DC45E13039F4A091BD09A03019F0D8
:109FB8000E94F87409F402C00E94821D0E94737600
:109FC8001CC0EE30D1F40E9484741397EFE0EC9338
:109FD8000E94DC45E13089F4A091BD09A03019F058
:109FE8000E94F87409F402C00E94821DE0E0E09328
:109FF800BD09EFEFEA930E9466460E94C07559C4F6
:10A008001A930E945D730E949E6FEAE7EA930E948A
:10A01800F03C0E94607211971C91E12FE23131F4FB
:10A02800E6E0EA930E94F03C99D937C0E13131F477
:10A03800E2E1EA930E94F03CC2DC2FC0EF3099F4D1
:10A048000E949B750E94DC45E13039F4A091BD095E
:10A05800A03019F00E94F87409F402C00E94821D11
:10A068000E9473761AC0EE30C1F4EFE0EA930E94C2
:10A07800F03C0E94DC45E13081F4A091BD09A0309C
:10A0880019F00E94F87409F402C00E94821DE0E0F1
:10A09800E093BD09EA930E9466460E94C075A091AC
:10A0A800C009AA3211F00E94C73D03C4EFEFE09344
:10A0B800E00CE093E10C0895EA81E0937A07E881E7
:10A0C800E0937B07E0910506E061E093050624C173
:10A0D8000E94467CA0917A07A43120F4A0917B07C6
:10A0E800A33008F034C0E0917A07F0E0ACE0B0E0CB
:10A0F8000E94C4798F01E0917B07F0E0A4E1B0E011
:10A108000E94C4799F010E947A76ECE0F0E00E94F8
:10A118007F76F0E00E9472790E94EE6CEE81E0306A
:10A12800B1F0E0917A07A3E0EA9FF001E158F84F17
:10A13800DF01E0917B07F0E0AE0FBF1F4C91552780
:10A148000E947A764A93E0E0EA930E943C560E9485
:10A158004D7C27960895E0910506E07141F0E2E014
:10A16800EA93B6DFE0910506EF7EE09305060895D1
:10A178000E948476AF39E0E0BE0744F4A091C70D91
:10A18800B091C80DAF37E0E0BE070CF033C00E94B5
:10A1980089760E944A6F0E943C56A0915807B09158
:10A1A8005907549734F4A0915A07B0915B07139755
:10A1B8000CF010C00E949472A3E0B0E00E949C7959
:10A1C800E158F84FA0915A07B0915B07EA0FFB1FBF
:10A1D800A981A083E0910806ACE0EA9FF0010E9403
:10A1E80084760E9496760E949A760E94947231969E
:10A1F8000E949F760C94FC54E881EA93E0910B0648
:10A20800EA93B6DF219608951A9310E00E949A7493
:10A21800E03031F00E949A74EA93EEDF1F5FF6CFC8
:10A228001881239608951A930A9300E010E00E947B
:10A23800A476E03021F00832E0E01E070CF007C0F9
:10A248000E94A476EA93D8DF0F5F1F4FF0CF1981E1
:10A25800088162C01A930A9300E010E0F801AB810C
:10A26800BC810E94AB7629F0EA81D8010E944F7424
:10A278000CF009C0F801AB81BC810E94B076BCDF4C
:10A288000F5F1F4FEBCF19810881FBC20E94487CEA
:10A298000E948476EFE9F0E0EA1BFB0B31978F010F
:10A2A8000E94B5760E947A760E94416B0E944F7C8C
:10A2B80033C00E94487CAC810E94BD760E2F1127C6
:10A2C8000E94B5760E947A760E94416B0E944F7C6C
:10A2D800D8C2EA81FB810E949F76E881F981E093E8
:10A2E8005A07F0935B07AA81BB81ECE0F0E00E947B
:10A2F800C4790E949A76A881B981E4E1F0E00E94CD
:10A30800C47906C0EA81FB810E949A76E881F981C6
:10A31800E093C70DF093C80D249608950E94C57662
:10A32800143128F41A930E94E6631F5FF9CF0E9444
:10A33800326B0E94326B0E94376BEFE7F0E00E94AD
:10A34800EE6C10E0153048F4A5E11A9FF001E551D4
:10A35800F94FA0E0A0831F5FF5CF10E0143148F457
:10A36800ABE01A9FF001E15FF94FA0E0A0831F5F07
:10A37800F5CFE0910506EF7EE09305069AC20E94AC
:10A38800C5761431F0F4ADE01A9FF001BF010E94C8
:10A39800B46C0F01DF01EB81FC81AE17BF075CF0E5
:10A3A800E981FA81E015F10534F0FB01E55FFA4F28
:10A3B800E081E03009F403C01A930E94E6631F5F4E
:10A3C800E0CF0E94326BED81FE81FA93EA930E94FE
:10A3D800376BA985BA85EF81F885EA1BFB0B0E94CC
:10A3E800EE6C4EC2A2970E94467CE9A5ADE0EA9FBA
:10A3F800F001E050FB4F8F01D8011B96EC91E03043
:10A4080009F4FDC1D8011B96EC91E9A3E07849F065
:10A418000E94CD76A5E1EA9FF001E551F94F0E942F
:10A42800D476E9A1E07449F00E94CD76ABE0EA9FCA
:10A43800F001E15FF94F0E94D476FE0136960E9442
:10A44800D876E8A3E0910806EB8FE0910906EA8F39
:10A458000E949B6BD80111962D913C91D8011396BF
:10A468004D915C91D80115960E94647AEEA3FFA3E2
:10A47800D8011796EC91F0E0ECA3FDA3D80118964B
:10A48800EC91EC8FE0910906A0E10E94DC76EAA34A
:10A49800FBA30E94DE740E94E0760E94E076ECA1A5
:10A4A800EA930E947855D8011996EC91EC8FAC8DFF
:10A4B800AF3011F4E8E0EC8F0E94DE740E94E5767C
:10A4C8000E94D8750E94EA760E94EE760E94F57680
:10A4D8000E94F8760E94DE743A932A93EAA5FBA5B7
:10A4E800E40FF51F0E940177EEA1FFA1E20FF31F11
:10A4F8000E94D8750E94E5760E94F876A8A5A1303A
:10A50800A1F43A932A93FA0131960E94F576FA93C8
:10A51800EA93FA0131960E940177F90131960E9477
:10A52800D875F90131960E94F876A8A5A230D1F421
:10A538000E94EE7631970E94F576FA93EA93EAA59F
:10A54800FBA5E40FF51F31970E940177EEA1FFA14B
:10A55800E20FF31F31970E94D8750E94E576319774
:10A568000E94F876E8A5E03011F40C94D353D80192
:10A578001996EC91EC8FE0910806ACE00E94047704
:10A588000E94EF79ED8FA8A1EA1710F40C941153EB
:10A59800E1E0E0930906E03021F0ECA1FDA1B597D8
:10A5A8000CF402C00E940A77AAA1BBA1ECA1FDA1EC
:10A5B800EA1BFB0BDF010E941277EAA3FBA3ABA106
:10A5C800AA231AF4E0E0EAA3EBA3A8A10E94BD76AF
:10A5D800AEA1BFA1F0E00E941777EE8FA8A5A13029
:10A5E80021F40E941A770E941F77A8A5A23021F4AF
:10A5F8000E941A770E942977E0E0E9A30E94317748
:10A60800AE0FBF1FEC91E03039F00E9431770E9405
:10A61800B0760E943677F2CFC2C0E1E0E093090637
:10A62800E03031F0ECA1FDA1E734A0E0FA070CF42A
:10A6380002C00E940A77E8A1EF8FEAA1FBA1EE0F02
:10A64800FF1FACA1BDA1AE1BBF0BE3E0F0E00E9471
:10A65800EF79EAA3FBA3ABA1AA2322F4E1E0F0E09F
:10A66800EAA3FBA3EF8DE150EF8FEF8DF0E0DE0161
:10A678001696AE0FBF1FAC91A03219F0AF8DA13066
:10A6880008F404C0EF8DE150EF8FEFCFAF8D0E943B
:10A69800BD76AE2FEEA1FFA1B0E0EA17FB0714F3D9
:10A6A800EF8DE03011F4ED8DEF8FAF8DECE00E946F
:10A6B80004770E941777EE8FA8A5A13021F40E9495
:10A6C8001A770E941F77A8A5A23021F40E941A7752
:10A6D8000E942977E0E0E9A30E9431770E94AB76D7
:10A6E80021F0EF8DA9A1AE1708F007C00E943177BD
:10A6F8000E94B0760E943677EFCFAF8DE8A1EA1BB3
:10A70800AE2FED8DEA1768F0AF8DE8A1EA1BACE03B
:10A71800EA9FF001A09108060E9404770E9417772B
:10A7280001C0E0E0EE8FA8A5A13069F40E941A7775
:10A7380031960E947F76AFE00E94DC760E943E77D9
:10A7480031960E94886DA8A5A23059F40E941A7704
:10A758000E947F76AFE00E94DC760E943E770E94DE
:10A76800886D0E943177AE0FBF1FAC91A03219F4EB
:10A77800E9A1EF5FE9A30E9431770E94AB7639F037
:10A78800AF8DE9A1EA1BAE2FED8DEA1708F407C0DB
:10A798000E9431770E94B0760E943677ECCFD801BC
:10A7A8001C96EC91E03029F10E949B6B0E94DE74AC
:10A7B800A9DDF801A485A43698F4E0E0E0930B063F
:10A7C800F801A485AA3028F0A485AA930E940962FA
:10A7D80006C0D8011C96EC91E05DEA930DDD09C036
:10A7E800ECE0E0930B06E2E5EA9306DDEDE4EA939C
:10A7F80003DDEB8DE0930806EA8DE09309060E94DD
:10A808004D7CAA9608951A9310E0E89427F814311D
:10A8180070F40E94BC6DE03011F00E94C36D1F5FA0
:10A82800A895E12FE37011F40E94D215F0CFE0E073
:10A83800E0930B060E94D2153CC01A9310E0143125
:10A84800E0F40E94C86D99F0AD5FBA4F0E94647A37
:10A85800DF01EB81FC81EA17FB074CF4F0010E9451
:10A86800B46CDF01E981FA81AE17BF070CF002C0B2
:10A878000E94C36D1F5FA895E2CFE0E0E0930B064E
:10A888001881259608951A9310E0143190F40E94C7
:10A89800C86D31F0FD01E65FFA4FE081E17009F41F
:10A8A80006C01A93E0910506E170EA939BDD1F5FED
:10A8B800ECCF199108952C970E94467CAD89BE89EA
:10A8C8000E941277ED8BFE8BAB89BC890E941277B0
:10A8D800EB8BFC8BED89FE89A98DBA8DEA0FFB1FE6
:10A8E800E98FFA8FEB89FC89AF89B88DEA0FFB1FD6
:10A8F800EF8BF88FED89FE89AD89BE890E94447778
:10A90800EE87FF87688B798BEB89FC89AB89BC89DB
:10A918000E9444770E944B770E94F37BEA87FB876B
:10A928006C877D8700E010E0EB89FC89E017F10770
:10A9380014F40C94E054F8010E9486790E941D7B5F
:10A948000E945077AE81BF81888599850E94A57B3A
:10A95800AA85BB858C859D850E94A57B0E944B7727
:10A968000E9455770E94E67AAF015A934A930E9453
:10A978008F6A2E2F33270E945A77E98DFA8DE01BB4
:10A98800F10B0E946177ED8DFE8DE01BF10B0E94AB
:10A998006B770E945A77F801A98DBA8DEA0FFB1FD1
:10A9A8000E946177F801AD8DBE8DEA0FFB1F0E94F2
:10A9B8006B770F5F1F4FB8CF0E944D7C6B96089541
:10A9C800E981EBBBE7E1E09365001F98E6E1E093DE
:10A9D8006500E7E1E0936500E881EBBBEFE1E09318
:10A9E8006500EEE1E0936500EFE1E09365001F9AF2
:10A9F800229608951F9808951F9A08950E94836DBE
:10AA08000E944979EBE1E0936500EAE0F0E00E94FA
:10AA18004C6EEFE1E09365000E94E96C0E94497971
:10AA2800E1E0EA93E2E0EA93CBDF0E944B6B21F48A
:10AA3800E2E0EA93E2E403C0E2E0EA93E2E8EA93C0
:10AA4800BFDFE7E0EA93EFE7EA93BADFE8E0EA93EB
:10AA5800E7E1EA93B5DF0E947177E1E2EA93E8E87B
:10AA6800EA93AEDFE2E2EA93E3E3EA93A9DFE3E203
:10AA7800EA93ECECEA93A4DFE4E2EA93ECECEA93E1
:10AA88009FDFE5E2EA93EBEBEA939ADFE6E2EA93EB
:10AA9800EBEBEA9395DFE7E20E947777E8E20E9422
:10AAA8007777E9E20E947777E5E0EA93E8E0EA93CE
:10AAB80087DFE6E0EA93E7ECEA9382DFE0E0F0E0A4
:10AAC8000E949F76E0E0F0E0E0935A07F0935B077E
:10AAD8000E949B6BE3E00E94A16BE0E0E0930D060F
:10AAE800EDE0E0930E06089521970E94467C4A8582
:10AAF800EF810E947C770E94737A8F01E0E1EA93EC
:10AB0800EF85EA935DDFE2E1EA93EB85FC85AF85AB
:10AB1800B889EA0FFB1FEA9353DFE9E00E948077C8
:10AB2800E1E1EA930E948577EA0FFB1FEA9348DF89
:10AB3800E9E1EA93EF850E948A770E9480775ADFDD
:10AB48002EE13FE1E0E0EE83E885F985AE81B0E0F3
:10AB5800EA17FB079CF050E0451760F01BBB2093F9
:10AB68006500309365000BBB20936500309365004A
:10AB78005F5FF2CFEE81EF5FEE83E6CF0E94005574
:10AB8800E0E10E948F77E2E1EA93EFE9EA930E941D
:10AB9800E454E9E00E948F77E1E1EA93EFE7EA9372
:10ABA8000E94E4540C94DE560E94467CEE810E947A
:10ABB8007C770E94737A8F010E948577EA17FB07DA
:10ABC80039F4EF81F885AB85BC85AE17BF070CF06B
:10ABD80023C0E7E10E948F77E7E10E948F77E9E1E0
:10ABE800EA93EE850E948A770E9494772EE13FE1EE
:10ABF8005B854F81451760F01BBB20936500309340
:10AC080065000BBB20936500309365005F5FF2CF52
:10AC18000E9400550E9471770E948577AE17BF0782
:10AC28003CF4EF81F885AB85BC85EA17FB0709F092
:10AC38001BC0E9E1EA93EE850E948A770E94947727
:10AC48002EE13FE15D854985451760F01BBB2093E8
:10AC58006500309365000BBB209365003093650059
:10AC68005F5FF2CF0E9400550E944D7C2F96089599
:10AC780024970E94467CEB85F0E0EE0FFF1F0E94B0
:10AC88007279E887F98730910806EA850E947C770F
:10AC98000E94737A0E947B791E2FEA850E947C7736
:10ACA8000491E0E0EF83AF81A03110F00C94DE5600
:10ACB800E0E0EE83E0910906AE81AE1710F00C9447
:10ACC800D456E8E10E94807740E0423010F00C94BE
:10ACD800CA56E42FEE0FEE0FEE0FE39FF001AE859C
:10ACE800BF85F0E0EA0F5E2FE42FA885B9850E94A2
:10ACF8009676E451FB4F2491203011F40C94C756FA
:10AD080027FF3BC0E9E1EA935A930E94E4541F9855
:10AD1800EFE1FEE10BBBF0936500E09365001BBB20
:10AD2800F0936500E093650031FF0AC00BBBF09318
:10AD38006500E09365001BBBF0936500E093650038
:10AD480026FF1AC00BBBF0936500E09365001BBBA0
:10AD5800F0936500E093650031FF0BC00BBBF093E7
:10AD68006500E09365001BBBF0936500E093650008
:10AD78005F5F220F5F5FE4CF1F9A220F31FD5F5F95
:10AD88005F5F0C9480564F5F0C946956EC85FD8587
:10AD98003196EC87FD87EE81EF5FEE830C945E566B
:10ADA800E885F9853296E887F987EF81EF5FEF83C9
:10ADB8000C9457560E944D7C6096089523970E94E4
:10ADC800467CA895E9850E947C770E94737A0E9448
:10ADD8007B790E2FE9850E947C77149130910806C3
:10ADE800E0E0EF83EA85AF81AE1710F00C9484574A
:10ADF800E0E0EE83E0910906AE81AE1710F00C9406
:10AE08007F57E8E10E948077E0E0E887EB85A88536
:10AE1800AE1710F00C947557E885F0E00E9474792D
:10AE2800DF010E94B46B0E94C479AE85BF85EA0F2A
:10AE3800FB1FAF01E889F98924913196E88BF98BDA
:10AE4800203011F40C94705727FF3DC0E9E1EA93D4
:10AE58004A930E94E4541F98EFE1FEE10BBBF09384
:10AE68006500E09365001BBBF0936500E093650007
:10AE780031FF0AC00BBBF0936500E09365001BBB74
:10AE8800F0936500E093650026FF1CC00BBBF093B0
:10AE98006500E09365001BBBF0936500E0936500D7
:10AEA80031FF0CC00BBBF0936500E09365001BBB42
:10AEB800F0936500E09365004F5F5F4F220F4F5F8F
:10AEC8005F4FE2CF1F9A220F31FF02C04F5F5F4FE3
:10AED8004F5F5F4F0C942457E885EF5FE8870C9429
:10AEE8000A57EC85FD853196EC87FD87EE81EF5F8B
:10AEF800EE830C94FE56EF81EF5FEF830C94F656C9
:10AF08000E944D7C6296089524970E94487C0E9476
:10AF1800BB62E4ECFAE10E94BC6F0E944A630E94A3
:10AF2800E162E091AA09E03061F0EFECFAE10E94F9
:10AF3800BC6F0E944A63E091AA090E940E750E94A4
:10AF48009B770E94E1620E948C1B00E00A30A0F40B
:10AF58000A930E94221A0E94ED6DEFE0EA930E9484
:10AF68002163E02FACE2B8E00E949F770E94886FCF
:10AF78000E94A3770F5FEACF0E94F562E8EDFAE13D
:10AF8800FA93EA93EFE0EA930E944A630E94D56D30
:10AF98000E94FE620E94E1620E94F7620E94E162E2
:10AFA80010E0103110F00C946C580E94536EE117A9
:10AFB800D9F5EEEDFAE10E94BC6F0E944A630E9447
:10AFC800856CFA93EA930E949B77E0E0E093A709E7
:10AFD800A091A709A03430F5E091AA09EA93E0917D
:10AFE800A709EA930E94081C0E940F6E3097B9F0D7
:10AFF800E091A709EA930E94E5190E940F6EFA935F
:10B00800EA930E94A9770E944A630E94B36EEAE01D
:10B01800EA930E9421630E94186E0E94A3770E94FF
:10B02800216ED6CF0E94AF770E94856C0E948D6FEB
:10B0380011F00C946A58EEEDFAE10E94BC6F0E9480
:10B048004A630E94856CFA93EA930E949B770E9458
:10B05800B377E0E30E94996F29F40E949E6F0E94E3
:10B06800223C9F0100240216030674F50E944E73C9
:10B078000E944C3CEC83FD836E837F830E944E7359
:10B08800EAE0EA930E94D13C3A932A930E94A97776
:10B098000E944A63ECECFCE0FA93EA93EAE0EA9354
:10B0A8000E942163EC81FD816E817F810E94A377DC
:10B0B8000E94B377E1E30E94996F29F40E949E6F82
:10B0C8000E94223C9F01CECF0E94AF771F5F69CFBD
:10B0D8000E94BC620E944F7C289608950E94487C7A
:10B0E800AD81BE812C910E94BC770E94856C0E9424
:10B0F800DA6B0E94D56CECE3EA930E940051EC8174
:10B10800EA930E945D512A93ED81EA930E94B2610D
:10B11800EEE3EA930E9400510E94C1770E9499725F
:10B128000E94C577333409F431E2313320F0EC81E1
:10B13800E05DE31708F407C0E32F0E94F472E255BC
:10B14800FF4FE4912E273D3311F0313209F401C04D
:10B15800CCCF3D3319F4AD81BE812C93E32F0E94EF
:10B168004F7C279608950E94467C20E0AF81B885E1
:10B178005C910E94BC770E94856C0E94DA6B0E94E9
:10B18800D56CE2E0EA930E945D515A930E940962ED
:10B198000E94C1770E9499720E94C577303310F0DF
:10B1A8003A3308F00EC0203009F450E021E0A52F12
:10B1B800EAE00E941E7AAAE0EA9FF001E30FE0535A
:10B1C8005E2F3B3211F4533608F001C05F5F3D3209
:10B1D80011F4513008F401C05150333429F42030AF
:10B1E80009F431E250E020E03D3319F4EE81E5172F
:10B1F80008F005C0AF81B8855C9130E020E03D33B0
:10B2080011F0313209F401C0B6CF3D3319F4AF81E2
:10B21800B8855C93D0C00E94467C20E0AF81B88599
:10B228004D915C910E94BC770E94856C0E94DA6BFC
:10B238000E94D56CAE81A23051F4E6E0EA930E94F8
:10B248005D51FA010E94E46C0E94DF6108C0E5E0EC
:10B25800EA930E945D515A934A930E94EB610E94BF
:10B26800C1770E9499720E94C577303310F03A3343
:10B2780008F01EC0203011F440E050E021E04031D9
:10B28800E7E25E0734F0DA01E0E1F7E20E94217AB2
:10B29800AF01493BEBE05E0724F0DA010E94EF7250
:10B2A800AF01DA010E9453740E94CA77D097AD01AA
:10B2B8003B3221F44033E5E75E070CF002C04F5FF4
:10B2C8005F4F3D3221F40024041605060CF002C03D
:10B2D80041505040333431F4203009F431E240E039
:10B2E80050E020E03D3311F0313209F401C09CCF29
:10B2F8003D3321F4AF81B8854D935C935CC00E94C7
:10B30800467C0E94BC7720E050E04FEF0E94856C9D
:10B318000E94DA6B0E94BA6CEF81F885FA93EA937F
:10B32800E885EA930E942E51E52FE10FF0E00E9494
:10B33800DA6B0E9499720E94C577303310F03A3365
:10B3480008F021C03053431729F04F3F09F05F5FE1
:10B3580020E005C0A22FAF5FEA2FE3702E2FE52F64
:10B36800AF81B8850E9496760F01E32FA8E0B6E179
:10B378000E949F77AE0FBF1FE22F0E949676E4913E
:10B38800D001EC93432F3B3219F4EE815E1708F09D
:10B3980002C05F5F4FEF3D3211F4513008F402C034
:10B3A80051504FEFEE815E1720F4313211F03D33EA
:10B3B80009F401C0ABCFE32F0E944D7C2996089574
:10B3C8001A930A93A091230DECEDEA231E2F00E0B7
:10B3D8000D3040F40E940D763296E491E11711F099
:10B3E8000F5FF6CF0E940D760E94737A0E94926CCE
:10B3F800E02F099119910895A3E2BDE0E881F0E0FA
:10B408000E94657611F4E3E701C0E9E4EA930E943B
:10B418000051219608950E94467C0E94BC770E94A4
:10B42800856C0E94DA6B0E94BA6CCADF5E2F0E949C
:10B43800C1770E9499720E94C5773D3211F0363368
:10B4480011F4503009F401C051503B3211F033333C
:10B4580011F45C3008F001C05F5FA091230DE1E0BA
:10B46800EA232E2FE52FA0E0B2E00E949F77EA0F93
:10B47800FB1F3296E491E20FE093230D3D3311F068
:10B48800313209F401C0CBCFE32F0E944D7C2696C0
:10B4980008950E94487C0E94BC770E94856C0E9497
:10B4A800DA6B0E94BA6C0E94CF770E94657619F415
:10B4B800EBEEFAE102C0EFEEFAE1FA93EA930E94AA
:10B4C80017510E94C1770E9499720E94C577303344
:10B4D80010F03A3308F00EC00E94CF77EA0FFB1F36
:10B4E8000F010E94CF77AE0FBF1FAC91E1E0EA27B2
:10B4F800D001EC933D3311F0313209F401C0CDCFC6
:10B50800E32F0E944F7C259608950E94487C0E9454
:10B51800D3770E94D9770E94326B0E946D510E94A6
:10B52800B36EEAE0EA93EBDEE13209F4CBC20E94A3
:10B53800326B0E94326B0E94B272E3EFFAE10E9412
:10B54800926CEEE1FDE00E94BC6F65DEE13209F429
:10B55800B9C20E94326B0E94326B0E94B272E9EF4C
:10B56800FAE10E94926CE091200DEF5F0E2FEDB78B
:10B57800FEB7FA93EA930F93EAE0EA93F4DD0F91AA
:10B58800E13209F49FC200240216030624F4E02FD6
:10B59800E150E093200D0E94326B0E94326B0E94B2
:10B5A800B272E2E0FBE10E94926CE5E3FDE00E94EA
:10B5B800DD7709F487C20E94326B0E94326B0E94C9
:10B5C800B272E8E0FBE10E94926CE7E3FDE00E94C2
:10B5D800DD7709F477C20E94326B0E94326B0E94B9
:10B5E800B272EEE0FBE10E94926CE2E2FDE00E94A2
:10B5F800E67709F467C20E94326B0E94326B0E94A0
:10B60800B272E7E1FBE10E94926C05DFE13209F4D6
:10B6180059C210E0133010F00C94C65B0E94326BD4
:10B628000E94326B0E94B272E12F0E94B672EDE165
:10B63800FBE10E94926C0E94EE770E946D51A6E297
:10B64800BDE00E94856C0E94F27709F43BC2E9E0F4
:10B65800F0E00E94946B0E946D51A9E2BDE00E9447
:10B66800856C0E94F27709F42DC20E94326B0E9409
:10B67800326B0E94B272E12F0E94B672E8E2FBE1DF
:10B688000E94926C1A9305DFE13209F41BC20E94F2
:10B69800EE770E94FC77E17059F40E947E710E9457
:10B6A800D2700E94C574B7DDE13209F40BC20AC03A
:10B6B8000E947E710E94D2700E94BC6FACDDE132A4
:10B6C80009F400C20E94326B0E94326B0E94B2726F
:10B6D800E12F0E94B672EAE2FBE10E94926C0E949E
:10B6E800EE770E946D51A2E3BDE0EE27A10FBE1FC9
:10B6F8002C913327EDB7FEB73197FA93EA933F932E
:10B708002F93E0E0EA9387DD2F913F91E13209F42E
:10B71800D9C1A2E3BDE00E94856CEA0FFB1F20831C
:10B72800123070F50E94326B0E94326B0E94B27226
:10B73800E12F0E94B672E1E3FBE10E94926C0E9445
:10B74800EE770E946D51A9E3BDE0EE27A10FBE1F61
:10B758002C913327EDB7FEB73197FA93EA933F93CD
:10B768002F93E0E0EA9357DD2F913F91E13209F4FE
:10B77800A9C1A9E3BDE00E94856CEA0FFB1F2083E5
:10B788001F5F48CF9FC10E94487C10E01A930E9417
:10B7980008730E94D9770E94326B0E9401780E9438
:10B7A800F26D0E94416F0E94E06C0E94326B0E9411
:10B7B800886C0E946D510E9414720E94E46C0E9471
:10B7C800C9610E940E780E94886C0E946D51E091B8
:10B7D800370DF091380D0E94E46C0E94C9610E94F7
:10B7E800326B0E94F36CE8E3FBE10E94926CE091FB
:10B7F800200D0E9413780E940E780E94F36CE0DD01
:10B808000E94146EE091220DE03029F0E091220DA3
:10B81800EA930E94096200E00330C8F50E94326B87
:10B82800E02F0E941E6C0E946D510E94B371EA9332
:10B838000E940962EBE2EA930E9400510E94BA71E9
:10B84800EA930E9409620E94146E0E94C17151F429
:10B858000E94C9710E94D96C0E94E46C0E94DF6149
:10B86800E3E707C00E94C9710E94D96C0E94E06C8E
:10B87800E9E4EA930E9400510E94146E0E94D37179
:10B88800EA930E940F620E9417780F5FC5CF0E944B
:10B89800A9633E2F3B3211F4103408F001C01F5F3A
:10B8A8003D3211F4113008F401C011503D3439F41F
:10B8B8001A930E94E51929DE1A930E940D1A313253
:10B8C80009F064CFFFC00E94487C10E00E949251AA
:10B8D800012F0E94326B0E94326B0E946D51ECE383
:10B8E800FBE10E94926C31E0363020F5103800F50B
:10B8F8000E94326B0E94B46B0E94D56C1A930E940E
:10B908004A1AE12F0E9413780E94146EA091BD0D6F
:10B91800E3E00E941B78A091BE0DE7E00E941B782F
:10B92800E0911008EA93E8E0EA930E94B261139567
:10B938003F5FDACF0E943B0E0E94A9633E2F3D3441
:10B94800F1F50E947A72102F1038C8F51A930E94E8
:10B958004A1A0E94326B0E94326B0E94B272E0E572
:10B96800FBE10E94926CE12F0E9413780E942178DB
:10B978000E9425780E946D51E3E5FBE10E94926CDC
:10B98800EDEBFDE0FA93EA93E3E00E94297809F4ED
:10B9980099C00E9425780E94B272E9E5FBE10E94F5
:10B9A800926CEEEBFDE0FA93EA93E7E00E942978C7
:10B9B80009F488C01A930E947E1A1F5FC5CF3132DE
:10B9C80011F0103808F001C081CF7CC00E94487C7B
:10B9D8000E9492510E94D9770E94326B0E946D5149
:10B9E800EFE5FBE10E94926C10E0113008F51A9324
:10B9F8000E948A1A0E94326B0E94CC6C0E94D56CFD
:10BA0800E12F0E9413780E942178E091B80D0E94DE
:10BA18002E78E091BB0D0E942E78E091B90D0E941E
:10BA28002E78E091BA0DEA930E940F621F5FDDCF76
:10BA38000E94A9630E2F0D3411F00C94665D0E94CC
:10BA48007A7210E01130F0F51A930E948A1A0E9457
:10BA5800326B0E94326B0E94B272E2E7FBE10E94F5
:10BA6800926CE12F0E9413780E94217830E03430E4
:10BA780020F50E9425780E94B2720E94B46B0E9441
:10BA88007479E851FA4E0E94737A0E94926C0E946F
:10BA9800376F0E94886C0E94B2720E94B46B0E9439
:10BAA8007479E851FA4E0E943378FD013596E49195
:10BAB8000E94297839F03F5FDACF1A930E94AC1AB6
:10BAC8001F5FC0CF0E944F7C249608951A930A9353
:10BAD8000E94D37700E0083210F00C94495E0E946F
:10BAE800300E0E94326B0E94326B0E9437780E949F
:10BAF800C96F0E94737A31960E94926C0E94146EEC
:10BB08000E94376F0E94886C0E9437780E94C96F24
:10BB18003496E491E038B1F40E94536E1E2FEDB7CD
:10BB2800FEB7FA93EA931F93E0E1EA931CDB1F91B7
:10BB3800E13211F40C94AF61E12FA9E0B0E00E946A
:10BB4800A67A9FC0E238B1F40E945D6E1E2FEDB751
:10BB5800FEB7FA93EA931F93E0E1EA9304DB1F919F
:10BB6800E13211F40C94AF61E12FAEE0B0E00E9435
:10BB7800A67A87C0E138E9F40E94E4731E2FEDB776
:10BB8800FEB7FA93EA931F93E3E0EA93ECDA1F9186
:10BB9800E13211F40C94AF610E94300E0E94E473FC
:10BBA800E11731F0E12FA8E0B0E00E94A67AFFCFBC
:10BBB80068C0E03071F40E94CD6B0E94C96F329664
:10BBC8000E94966CE1E00E94297811F40C94AF6110
:10BBD80058C0E13079F40E94CD6B0E94C96F0E9471
:10BBE8003378FD013596E4910E94297811F40C947C
:10BBF800AF6147C0E23079F40E94CD6B0E94C96FF3
:10BC080032960E94966CEFE0EA9305DBE13211F47C
:10BC18000C94AF6136C0E330F1F40E94CD6B0E9402
:10BC2800C96F3596E491ABE00E948A7AEA1B0E94BC
:10BC38000E750E94886C0E9437780E94C96F0E9416
:10BC48003378FD013596E491EA9348DAE13211F44C
:10BC58000C94AF6116C0E430A1F40E94CD6B0E9431
:10BC6800C16FE0936910F0936A100E94DA6B0E942A
:10BC7800C96F3596E491EA9342DBE13211F40C94F2
:10BC8800AF610E9425190F5F26CF0C94AF61E88140
:10BC98000E94B672E6EFFAE10E94926C0C94B962C7
:10BCA8001A930E947A7210E0133010F00C94AC5E74
:10BCB8000E94326B0E94326B0E94B2721A93E7DFC5
:10BCC800ECE0F0E00E94946B0E946D511A9394DBB3
:10BCD8000E94EE770E94FC77E17051F40E947E7119
:10BCE8000E94D2700E94C57496DAE13289F109C0C7
:10BCF8000E947E710E94D2700E94BC6F8CDAE13281
:10BD080039F1123018F50E94326B0E94326B0E9492
:10BD1800B2721A93BCDFE5E7FBE10E94926CECE09B
:10BD2800F0E00E94946B0E946D510E941778EAE03F
:10BD3800F0E00E94946B0E946D51A9E3BDE00E945F
:10BD4800856CEA0FFB1F0E94E67711F01F5FACCFEE
:10BD5800199108950E94487C10E01A930E94087374
:10BD68000E94D9770E94326B0E9401780E94F26D7E
:10BD780021E000E0033058F50E948D6CE22F0E940C
:10BD88000D720A9384DF0E94C17141F40E94C97147
:10BD98000E94D96C0E94E46C0ED306C00E94C9713F
:10BDA8000E94D96C0E94E06C0A9326DB2F5F023058
:10BDB80060F40E940E78E22F0E940D720E94CC71EE
:10BDC8000E94F16C0E9417782F5F0F5FD3CF0E94FB
:10BDD800A9633E2F3B3211F4103408F001C01F5FF5
:10BDE8003D3211F4113008F401C011503D3439F4DA
:10BDF8001A930E94E51954DF1A930E940D1A3132E2
:10BE080009F0ABCF0C9478620E947A720E94326B70
:10BE18000E94326B0E946D51EBE7FBE10E94926C2D
:10BE2800E1E0E093AA09EAEAF9E0FA93EA93E5E0A7
:10BE3800EA9399D9089522970E94467C0E94A963A3
:10BE48000E2FE091A409E03011F00C94CE6001327D
:10BE5800D1F4EEE8F5E1A091C30DB091C40DEA1755
:10BE6800FB0761F4E7E0E093A109EAE2EA93E4E87A
:10BE7800FBE10E94BC6F0E94003EDAC1E0E0E09363
:10BE8800BB070E943B780D3331F4E091BB07F0E02B
:10BE98000E94DD6B04910D3441F4EAE2EA93E7E88D
:10BEA800FBE10E94BC6F0E94003E063449F4E6EBB9
:10BEB800F5E1E093C30DF093C40DE0E0E093BB0718
:10BEC800003311F00B3229F4E091BB07EF5FE093E8
:10BED800BB070D3229F4E091BB07E150E093BB07A3
:10BEE800013329F491DFED3311F40E9442780333D2
:10BEF80029F48ADFED3311F40E948857063329F4B8
:10BF0800E0E0E093AA090E948857043329F4E0E0AE
:10BF1800E093AA090E944278A091AC09A13010F4DC
:10BF28000C946860023301F56FDFED33E9F40E9489
:10BF38004F78D1F4E091AA09EA930E94421C30E0BC
:10BF4800303190F40E94B46B0E948D6F59F4E32F46
:10BF5800E05DEA93EAE8FBE10E94926FE0E3EA938E
:10BF68000E94223E3F5FECCF053331F5E0E0E093DD
:10BF7800AA090E944F7801F511E01630E8F41A93E7
:10BF88000E94421C30E03031A8F40E94B46B0E9439
:10BF98008D6F71F4E32FE05DEA93EAE8FBE1FA9331
:10BFA800EA93E12FE05DEA93E0E3EA930E94223E00
:10BFB8003F5FE9CF1F5FE1CF013451F4EAE2EA9332
:10BFC800EDE8FBE10E945773E1E0E093A10930C17D
:10BFD8000A3409F4BFDE073311F00C9468600E943C
:10BFE8009251E0E0EA930E94900EE1E0E093A50907
:10BFF800E0E0F0E0E0939D09F0939E09E4E1F8E0C9
:10C008000E94BC6FE7E1F0E00E946E6F0E94266814
:10C01800EE83FF83EE81FF81FA93EA930E947E6D9F
:10C028000E943268E030B1F00E94FF110E94266839
:10C03800EE83FF83A091A20DA03021F00E94C034AE
:10C04800E03009F407C00E94316EED59F64FAEE0BA
:10C058000E94376EE5E0F0E0FA93EA930E94C46329
:10C0680040E050E00E94E522E03868F00E94E522B6
:10C07800EF573E2F313010F0313108F004C0E32F74
:10C088000E948470AF015A934A930E94942040936F
:10C098009D0950939E090091D607E0E0E093D607EA
:10C0A800013211F00B3209F401C0B4CF0B3221F484
:10C0B800E1E0EA930E94900E013209F09FCFE0E0A0
:10C0C800E093A509E093D607A091AC09A23011F03E
:10C0D8000C94C760093309F4F9DC053409F476DCFB
:10C0E800083309F450DB023409F4EDDB0334B1F50D
:10C0F8001091C20D0E94925100E0E091C10DE1172C
:10C1080011F0063008F01DC00E94326B0E94CD6B02
:10C118000E94D56C1A930E94DB1F1A9376D10E9455
:10C12800146EE091B20D0E942E78E091B50D0E9438
:10C138002E780E9435700E94E06C0E941B70039557
:10C14800DCCF0E943B0E0E94A9630E2F013221F022
:10C15800E091C10DE11709F401C0CCCF043499F482
:10C168000E944F7881F4A0915C0DA03021F4A09139
:10C178005A0DA03031F00E9439750E94326B0E942E
:10C188008C450E94241EE091A409E03011F40E941D
:10C19800BE0E49C0E130D1F4A091A909AB3010F42A
:10C1A800013209F405C00E9461160E943B0E0DC0C1
:10C1B800E0E0E093A7090E9458780E945773E0E0F6
:10C1C8000E945D78E2E0E093A4092DC0E23059F5C1
:10C1D800013269F4E0E0E093A4090E949251EAE296
:10C1E800EA93E7E8FBE10E9457730E94BE0E0B3208
:10C1F80011F00D3359F40E945878FA93EA93E1E369
:10C20800EA930E94003EE1E00E945D780D3259F405
:10C218000E945878FA93EA93E2E3EA930E94003E78
:10C22800E2E00E945D78A091A109A33009F406CE4E
:10C238000E944D7C289608951A93E3E0E093A209A2
:10C248000E9492510E94326B0E94326B0E946D5183
:10C25800E3E9FBE10E94926C0E94326B0E94886CB9
:10C268000E946D51E8EFF7E00E94BC6FE0E1F0E05A
:10C278000E946E6F10E0E091520D1E1700F50E94AB
:10C28800536EE117D1F0E12FE05DEA93EBE9FBE1B2
:10C29800FA93EA93E0E3EA93E0E00E94996F49F4A5
:10C2A8000E94856CE850F84FA1E0A083E12FE05D83
:10C2B80001C0EEE2EA930E9400511F5FDCCF0E94AA
:10C2C8003B78E0E0E093BB07E093A4090E94BE0E30
:10C2D8000C945966E881E03011F40E946278A881D4
:10C2E800A13021F4E0E3F6E10E946978A881A23048
:10C2F80021F4ECE3F6E10E946978A881A33021F4E7
:10C30800EAE4F6E10E946978A881A43021F4E0E526
:10C31800F6E10E94697829C10E94627808951A930B
:10C328000A93E0E0E0937807E093790710E014318E
:10C3380090F400E0033068F4A3E01A9FF001E1589C
:10C34800F84FDF01EE27A00FBE1FE0E2EC930F5F6E
:10C35800F1CF1F5FECCF0991199108951A9311E05D
:10C36800E981E11788F00E94856CE255FF4FE4915E
:10C37800AA81EA2319F0E12FE05D01C0E0E2EA9327
:10C388000E9400511F5FECCF29C12A97A091A40DEC
:10C39800A13040F0EA85FB856C857D850E94777A1F
:10C3A8000AD008C00E946E780E9472780E946E7847
:10C3B8000E94085133C12A970E946E780E947B78A8
:10C3C8000E9481780E946E780E94085127C12A979E
:10C3D8000E946E780E9494780E94B9730E946E78C9
:10C3E8000E94085128C12A970E946E78E9EBFBE168
:10C3F800FA93EA93EE85FF850E94E46C0E94B97374
:10C408000E946E780E94085116C12A970E946E7881
:10C41800ECEBFBE105C02A970E946E78E0ECFBE1AB
:10C42800FA93EA93EE850E94A2730E946E780E94A6
:10C4380008512B9608950E94487C10E0E1E3E093B0
:10C44800C00AE89431F8EA930E94AC3DE4ECFBE1C1
:10C458000E94527200E0E0917D070E17E0F40E94FE
:10C46800CD6BE158F84FE081E03258F4E3E2EA930B
:10C478000E94F03C0E94CD6BE158F84FE081E05DEE
:10C4880005C00E94CD6BE158F84FE081EA930E9405
:10C49800F03C0F5FE0CF0E94C73D0E9426689F01D5
:10C4A8000E94DB153A932A93E8ECF0E0FA93EA93BA
:10C4B8000E9432680E2FA0E031FCA1E0A03011F4F8
:10C4C800003009F001C0ECCF31FE07C0E0E0E09396
:10C4D8007D07E89431F8E1E007C01F5F123008F4E7
:10C4E800ADCFE0E0E0937D070E944F7C249608954D
:10C4F800E0917C07E03021F4E881EA930E949C38BF
:10C50800A0917C07A13079F4A0E09299A1E0A13034
:10C5180031F4A8950E94836D0E944979F5CFE8818E
:10C52800EA930E94413BA0917C07A230F1F4E0918C
:10C538007D07F0E0E158F84FA881A083E0917D07DE
:10C54800EF5FE0937D07E0917E07EF5FE0937E0762
:10C55800A03218F4EF5FE0937E07A0917E07A8331E
:10C5680020F069DFE0E0E0937E07219608950895C2
:10C578000E94AF770E94AF7720D0EBE1EA93B8DF53
:10C58800E9E6EA93B5DFA0917C07A13051F40E9457
:10C598008F6DE0919A00E069E0939A00E9E1E093F9
:10C5A8009900A0917C07A23021F445DFE0E0E093F8
:10C5B8007E07E0E0E0937C070895EDE0EA9398DFDA
:10C5C800EAE0EA9395DF08951A9310E0E9811E17CF
:10C5D80028F4EA81EA938CDF1F5FF8CF188123964D
:10C5E8000895EDE201C0EDE3EA93E8E2EA93ECDFB7
:10C5F800E4DF08952A97A091A40DA13038F00E9495
:10C608006E780E947B780E94817804C00E946E78C0
:10C618000E947278FE010E94BC6F0FD02E9608957A
:10C628002A970E946E780E9494780E94B973FE013E
:10C638000E94BC6F02D02C9608951A930A9310E0BA
:10C64800EA81E03011F408E201C00A81AB81BC81C3
:10C65800EE27A10FBE1FAC91A03011F0101708F003
:10C6680007C0AB81BC810E9444760E949C78EECFC3
:10C67800EA81E03039F0EA811E1720F4E0E20E94F6
:10C688009C78F9CF198108810C949A681A930A93B7
:10C6980010E0EA81E03011F408E201C00A81E12FDC
:10C6A800AB81BC810E949676E491E03011F01017BE
:10C6B80008F009C0E12FAB81BC810E949676E49115
:10C6C8000E949C78ECCFEA81E03039F0EA811E17AD
:10C6D80020F4E0E20E949C78F9CF198108810C943B
:10C6E8009A68E091BF07A091BE07EA17C1F00E94BF
:10C6F800A1780E94CA70EC91E093C1070E94A178CA
:10C708000E94D270E181E093C007A091BF07AF5F9C
:10C71800EAE00E941E7AE093BF07E1E00895CAC2EA
:10C728000E94A778A981A0830E94A7783196A88142
:10C73800A083A091BE07AF5FEAE00E941E7AE09353
:10C74800BE0715C3E091D60708951A93E091D6075E
:10C75800E03059F40E94DB150E94747121F4A09115
:10C76800D607A03009F001C0F5CF1091D607E0E058
:10C77800E093D6070E94747109F011E2E12F95C287
:10C788000E94487C0E9426688F010E94DB15EC817C
:10C79800FD81E00FF11FFF93EF930E942668AF9190
:10C7A800BF91AE1BBF0B9D010024021603061CF4AB
:10C7B8000E94747109F001C0E8CFE0E00E944F7C4C
:10C7C800269608951A930E947A70E050FB4FA0E0D5
:10C7D800A0830E947A70E55FFA4F108117FF09C0A5
:10C7E800E12FEF73A5E1EA9FF001E551F94FA0E0D1
:10C7F800A08316FF09C0E12FEF73ABE0EA9FF001B9
:10C80800E15FF94FA0E0A0830E947A70E55FFA4FDC
:10C81800A0E0A0830E947A70E65FFA4FA0E0A083B0
:10C82800A5C20E94487C30E0EE81ADE0EA9FF001AD
:10C83800E55FFA4F108116FF17C0E12FEF730E2F37
:10C848000E94AE7811F03A3008F009C00E94B6781C
:10C85800DF010E94B46B0E94BC783F5FF1CF0E9459
:10C86800B6780E94CA77EC9317FF17C0E12FEF73D1
:10C878000E2F0E94AE7811F0343108F009C00E94E2
:10C88800C278DF010E94B46B0E94BC783F5FF1CF91
:10C898000E94C2780E94CA77EC930E944F7C0C9445
:10C8A8002C69A0970E94467CEDA5FEA5A9A9BAA966
:10C8B800EA0FFB1FAF01E0E0F5E0EE83FF8310E035
:10C8C8001431C0F5AE81BF81AC91A03049F1EE8141
:10C8D800FF81A381B481EFA5F8A9EA17FB0701F549
:10C8E800EE81FF81A181B281E9A9FAA9AE17BF073C
:10C8F800BCF0EE81FF81A181B2814A175B0784F009
:10C908000E94C878AE0FBF1FE9A9FAA9AE17BF07E2
:10C918003CF00E94C878AE0FBF1F4A175B070CF4A3
:10C9280002C01A934FDFEE81FF813D96EE83FF83AD
:10C938001F5FC6CFE0E0F5E0EE83FF8310E014311F
:10C9480010F00C945265AE81BF81EC91E03011F08B
:10C958000C944B65EAA5EC93E9A9FAA9AE81BF81CD
:10C968001196ED93FC93EFA5F8A9AE81BF811396BC
:10C97800ED93FC93EDA5FEA5AE81BF811596ED93D1
:10C98800FC93EBA5AE81BF811796EC93E09104066A
:10C99800A0910A06EA27AE81BF811896EC93E09130
:10C9A8000B06AE81BF811996EC93E0910C06AE811F
:10C9B800BF811A96EC93AE81BF811B960E94396C99
:10C9C8001C96E0E0EC93E887E8A5F9A5309751F0CC
:10C9D800FE013896FA93EA930E94E076E4E1EA933E
:10C9E8000E94ED68EEA1FFA1309761F0FE01389634
:10C9F800FA93EA93E8A5F9A5FA93EA93E4E1EA93AE
:10CA08000E94D968E0E0EC8FFE0138960E94D87643
:10CA18003E2F3B30D8F000E00E94C278E081E03041
:10CA280011F0053008F002C00F5FF6CF0E94C278FF
:10CA3800E081E03059F40E94C2780E94D37830E057
:10CA4800E02FE058AE81BF811B96EC93E0E0EA8BC3
:10CA58003130D8F000E00E94B678E081E03011F083
:10CA6800043108F002C00F5FF6CF0E94B678E0816B
:10CA7800E03059F40E94B6780E94D37830E0E02F75
:10CA8800E05CAE81BF811B96EC93E12F08C0EE817C
:10CA9800FF813D96EE83FF831F5F51CFEFEF0E942A
:10CAA8004D7CE39608951A930A930E94D87830979C
:10CAB800A9F1E0915D07E03061F50E94D878049013
:10CAC80000925D07E0915D07E03031F4E0E0F0E0CE
:10CAD8000E946978E0E01AC00E94DD780E94D87848
:10CAE8000E94737AF595E7958F01D801E0E0F1E0AF
:10CAF8000E94EF79E0938700D801E0E0F1E00E941E
:10CB0800217AE09386000E94DD78E0E4E0938B00D0
:10CB180005C0E0915D07E150E0935D070C942F6834
:10CB28000E94487C00E020E035E010E01431B8F5C0
:10CB3800D901EC91E03079F111960E94647A0E9453
:10CB4800E57824F5D90113960E94647AAC81BD81F9
:10CB5800EA17FB07DCF4F90101801280D901159668
:10CB68000E94647AE00DF11DAE81BF81AE17BF0748
:10CB78006CF4F90103801480D9011796EC910E9496
:10CB88007A71AC81BD81AE17BF070CF004C0E12FEC
:10CB9800EF5F0E2F04C0235F3F4F1F5FC7CF0030EA
:10CBA80049F0E0915E07E01721F0A0915E07A03000
:10CBB80009F401C022C0A0915F07A53079F40A9357
:10CBC800E1E0EA93ADDD00935E0700936007D901C9
:10CBD800EC91E0936107E3E0E0935C07A0915F07C5
:10CBE800AE3119F4E4E0E0935C07A0915C07A33050
:10CBF80018F0E5E0E093630707C0E0E0E0935F0723
:10CC0800E0935C070E94EA78FFC0E0915E07E0309D
:10CC180091F0A0915F07A93220F4EA93E2E0EA9349
:10CC28007FDDA0915F07AD3330F0E0915E07EA93B6
:10CC3800E4E0EA9375DDE0E0E0935C07E0935F07EA
:10CC48000E94EA78E0E0E0935E07E09362070895C7
:10CC58000E94925164DB0895E091EA0CE093710020
:10CC6800E0E0E0937400E2B3E360E2BBE1B3E360C9
:10CC7800E1BB8BE18A95F1F7E1B3EC7FE1BBE4E43A
:10CC8800E093740085E88A95F1F708951A9314EAF9
:10CC9800E4EA0E94F07841F40E94F578183011F027
:10CCA800103111F4E0E001C0E2E019910895E4E9DF
:10CCB800E0937400E0E008951A93E981E1600E942E
:10CCC800FA7831F40E94F578103411F4E0E04EC09F
:10CCD8004CC01A93E9810E94FA7831F40E94F578E1
:10CCE800183111F4E0E042C040C01A93E9810E9473
:10CCF800FA7831F40E94F578183211F4E0E036C081
:10CD080034C01A93E981E03011F0E4EC01C0E4E8A2
:10CD18000E94F07879F40E94F578E0917300AA8176
:10CD2800BB81EC93103511F0183521F4E0E018813F
:10CD38000C94FA6AE1E018810C94FA6A1A93E98172
:10CD4800E093740010E0E0917400E07811F4163973
:10CD580008F005C08DE08A95F1F71F5FF4CFE091E8
:10CD68007400E07811F0E0E001C0E1E0188122965B
:10CD780008950E94487C3D810C8120E087DFE030E7
:10CD880021F5EE810E94756E01F53A93AEDFE03031
:10CD9800E1F40E94FE78C9F479DFE030B1F4EE8165
:10CDA800EA938ADFE03089F4EDB7FEB7FA93EA93A5
:10CDB8001F93E0E0EA93A5DF1F91E03031F477DFBD
:10CDC800E12F0E944F7C0C942C6946DFD7CF0E943C
:10CDD800487C30E00E811D8159DFE03099F4EF8105
:10CDE8000E94756E79F40E94FE7861F41A937DDFD3
:10CDF800E03041F4EC81EA9378DFE03019F457DF52
:10CE0800E0E002C029DFE8CF0E944F7C2896089511
:10CE180022970E94467C50E02B853A85A89536DFFC
:10CE2800E03011F00C947067EE850E94756E11F079
:10CE38000C9470672A9359DFE03011F00C947067F6
:10CE48003A9353DFE03011F00C9470671FDFE03045
:10CE580011F00C947067EE85EA932EDFE030E1F56F
:10CE6800E0E0EE83EF83EC85FD8531970E94E5785D
:10CE780051F4EDB7FEB7FA93EA931F93E0E0EA9313
:10CE880040DF1F9109C0EDB7FEB7FA93EA931F93ED
:10CE9800E1E0EA9336DF1F910E2FEE81FF81A8852E
:10CEA800B985EA0FFB1F1083EE81FF813196EE836F
:10CEB800FF83003039F4EC85FD85AE81BF81AE1764
:10CEC800BF0708F001C0CFCFEC85FD850E94E5784B
:10CED80019F4EDDEE0E002C0BFDEA1CF0E944D7C78
:10CEE8002F96089568970E94467C20E0E0E0EC8F3A
:10CEF800ED8F31E0A895E9A1FAA1662777270E946E
:10CF08001D7BEA87FB876C877D87EE8D0E940379FE
:10CF18000E945077AA85BB858C859D850E94F37BEE
:10CF2800EA8BFB8B6C8B7D8B0E94777AFE01729665
:10CF3800FA93EA930E94FC6AEE8BFF8B688F798FD5
:10CF48000E9409790E94E47AAF010E940979AE8DA6
:10CF5800BB27882799270E947E7A0E945577DE0191
:10CF68005A960E94E47AED93FC930AA119A18EDEE9
:10CF7800E030D1F5EDA10E94756EB1F50E94FE7802
:10CF880099F51A93B2DEE03079F5303051F14F5F00
:10CF98005F4FEC8DFD8D3196EC8FFD8FAC8DBD8D87
:10CFA8001197EBA1FCA1EA17FB0711F430E018C0B8
:10CFB800EC8DFD8D3197AF8DB8A10E94B07695DECE
:10CFC800EE8DDA01F0E0EA17FB0751F470DEEA8D26
:10CFD800FB8DA9A1BAA1EA0FFB1FE9A3FAA38BCF86
:10CFE800D4CF65DEE0E002C037DEC1CF0E944D7CC1
:10CFF800A6960895A881A03310F0AA3308F004C0BB
:10D00800E881E0530C940569A881A13410F0A73495
:10D0180008F004C0E881E7530C940569EFEF0C941D
:10D028000569A881AA3020F4E881E05D0C940569BF
:10D03800A881AA3020F0E881E95C0C940569E8E54C
:10D048000C9405691A930A93F8940091EB0C1091CB
:10D05800EC0C7894F8010991199108951A930A93A0
:10D06800F1DF8F01EA81FB81AC81BD81EA0FFB1FF3
:10D07800E01BF10BDF010E943C7C2CF4E0E01981FD
:10D0880008810C94286BE1E0198108810C94286BC5
:10D09800E1E0F0E00E94946B0E946D510E94516D96
:10D0A800E8ECFBE10E94926C0E949B6B0895EAE613
:10D0B800F6E1FA93EA93EAE6F0E0FA93EA930E943B
:10D0C8006B6DE4E0EA93E6E2EA93EEE0EA930E940D
:10D0D800E256E2E0F7E10E94866BE3E5F0E0FA93BE
:10D0E800EA93E8E0EA93E2E3EA93E1E0EA930E9454
:10D0F800E256089599818881009641F0BD81AC81FE
:10D10800FB81EA8105900D920197E1F7FD81EC81A1
:10D118000C94286BB981A881109631F0FC81EB81C1
:10D128006A8161931197E9F7EB81FC81259608954F
:10D13800E991F991A991B9911D900590011421F4F3
:10D148000020D1F7EE2708951018E1F3E1E008F484
:10D15800E2500895E991F991A991B991CD016191B0
:10D168006D936623E1F7FC010895E991F991A9917E
:10D17800B991CD0105900D920020E1F7FC010895C9
:10D18800A991B991EE27FF276D91662311F0319689
:10D19800FBCF0895AA27BB27E991F99105900020B4
:10D1A80011F01196FBCFFD0108957991E991F9915C
:10D1B800A991B991CD01772351F07A9561916D9339
:10D1C8006623C9F7772319F07A956D93FBCFFC0195
:10D1D80008956991E991F991A991B991CD016623D1
:10D1E80051F06A9505900D920020C9F7662319F051
:10D1F8006A950D92FBCFFC0108955D9BFECFE881F7
:10D20800ECB9219608951A930A93AC81BD810E94C6
:10D21800647A3097C1F0AA81BB810E94647A8F0139
:10D22800309749F00230E0E01E0760F0F8013197CE
:10D238008F01ED93FC93AC81BD810E94B16D319754
:10D24800AE81A08303C0EE81EA93D7DF19810881FC
:10D258002796089526970E94467C10E0EA89FB8964
:10D268003196EA8BFB8B3197E4912E2FE03011F445
:10D278000C94646AE12FE03041F4253211F411E096
:10D2880003C00E941579BFDF1AC1E130B1F425321D
:10D2980021F40E941579B7DF11C112E040E000E0E7
:10D2A8002D3211F401E00BC12B3211F44BE207C10E
:10D2B800203211F440E203C102C0E23039F450E0F8
:10D2C80013E0203311F40068FAC004C0E33011F011
:10D2D8000C94636A203310F02A3308F009C0A52F94
:10D2E800EAE0EA9FF0015E2FE22FE0535E0FE7C00D
:10D2F800E22FE33651F40E941C79E889F989A48168
:10D30800AA930E9422797FDFD9C0E33741F40E94B3
:10D318001C790E9428790E94D8761E2F0CC0E0370D
:10D3280071F40E941C790E942879FA93EA930E946A
:10D33800CE681E2F086002600F7730E035C0E436F3
:10D3480011F0E93611F4046002C0E53731F4E2E97E
:10D35800F8E1EE83FF8315E00DC0E83511F40860AD
:10D3680004C0E83711F00C94626AECE9F8E1EE8346
:10D37800FF8314E002FF14C00E941C790E943079D8
:10D38800AB85AA233AF4EA85FB850E945E79EA8791
:10D39800FB874DE2403011F01F5F01C00B7F04C0D6
:10D3A8000E941C790E94307900FD12C0151780F484
:10D3B80007FF08C002FF04C00B7F242F115001C0D3
:10D3C80020E301C020E20E9415791DDF5150EECF05
:10D3D800312F01FF1BC03030C1F003FF08C0EE81C0
:10D3E800FF813196EE83FF833197E49105C0AE81CA
:10D3F800BF81ED91AE83BF83EA930E94227903DF58
:10D40800503009F051503150E6CF4DC020E3EE8145
:10D41800FF810E94737AE887F987EE81FF8132964F
:10D42800EE83FF83E885F985AA85BB85AE17BF071C
:10D4380050F02F5FA885B985EA85FB85EA1BFB0BB1
:10D44800EA87FB87EFCF2A3328F003FF02C0295F62
:10D4580001C0295D04FD1BC0213320F4A885B985CE
:10D46800119709F409C0531710F000FF01C015C047
:10D4780020E207FF0CC020E3006102FF08C00B7F19
:10D488004A930E942279BFDE503009F051500E9421
:10D498001579B9DE503009F051503150A885B98559
:10D4A800129708F0B3CF00FF09C0503039F051503F
:10D4B800E0E2EA930E942279A6DEF7CF10E0CECE12
:10D4C8000E944D7C64960895FF92F82E22971A9335
:10D4D8000A93DE010E9455798D01DE0116960E949D
:10D4E80055790E94647AEA83FB83DE0114960E94D0
:10D4F80055790E9449731A930A93FE0136960E9441
:10D50800946BA8DEAA81BB81E0E0EC9319810881C5
:10D518002496FF900895A991B991EE27002460E818
:10D52800E894162E169407941E2A1EF0A015B1052D
:10D5380018F0A019B109E62BB7FBAA0FBB1F669517
:10D5480080F708957B816A81F981E88177FB770FFD
:10D5580067FD7160972F9E5781F078F0983190F4AD
:10D56800AA27BB27882708948795B795A7959A95E2
:10D57800D1F7EA23FB23682305C0E8947727EE2731
:10D58800FF2766276F77769508F4606877F9A99181
:10D59800B99189919991EA17FB076807790797FB71
:10D5A80008950E94D2740E94387919F40E943F7934
:10D5B8001DC0E6F7A881B9818A819B81E0E0F0E08F
:10D5C80060E87FE30E94557711C00E94D2740E94E0
:10D5D800387919F40E943F7909C0E6F30E943F792F
:10D5E800A0E0B0E080E89FE30E94577B249608956E
:10D5F8000E9444790E94387C39F4A881B9810E943C
:10D60800726F0E946E7A20C0AA81BB818C819D8135
:10D618000E94407C34F40E9444790E94777AC1DFEA
:10D6280005C00E9444790E94777ACFDFA881B9812A
:10D638000E946E7AA881B9810E94687AAA81BB810A
:10D648008C819D810E94557726960895E991F991DC
:10D6580030971AF4E095F09531960895E0E0F0E0FF
:10D66800FA93EA930895EFE9F0E0FA93EA930895BC
:10D67800E0E2F0E0FA93EA930895EFE0EA930C947D
:10D688007855E0E0E0930A06E0930B060895A8E0D9
:10D69800B0E00E94927AE0300895EBE9F0E0FA9366
:10D6A800EA930895E4E1F0E0FA93EA93EEE1F0E01A
:10D6B800FA93EA9308950E945564EFCFEDE2EA9356
:10D6C800CDCFE0E4F0E0FA93EA93ECCFEBE2EA9313
:10D6D800C5CFE1EFFFEFFA93EA9308950E945564EE
:10D6E800F8CFE0E6F0E0FA93EA93DCCFEDE4EA93D2
:10D6F800B5CFA5E01A9FF001E45CFD4F0895A12F76
:10D70800B0E00895FA93EA93EAE5F0E0FA93EA9331
:10D718000895FA93EA93E3E2F0E0FA93EA9308951E
:10D72800FA93EA939BCF0E943B0E0C940754E1E0D6
:10D73800E0930806E09309060895E0930A06E0E0FE
:10D74800E0930B060895FA93EA93E4E0F0E0089575
:10D75800EEE1F0E0FA93EA930895FA93EA93F8CFAA
:10D76800E32FF0E00895A091C30DB091C40DBD0161
:10D77800A3E0B0E00E949C79E60FF71FE491E03047
:10D788000895A091BB07E3E0EA9FF001EF5F0E2F39
:10D798000895E02FF0E00895E4E0F0E0FA93EA93CA
:10D7A8000895E6E9F0E0FA93EA930895FA93EA9384
:10D7B800F0CFA091C30DB091C40DBD01A3E0B0E0BE
:10D7C8000E949C79E60FF71F0895ABE03A9FF0019D
:10D7D800E45BFD4F0895FE013F96FA93EA9308959E
:10D7E800E0914A0DA0EA0E94CE792E2FE0914B0DD0
:10D7F800A0E80E94CE795E2F08953A930E94E51919
:10D80800A091130DAD320895E091210DE295EF70CE
:10D81800E0930A06E091210DEF70E0930B0608955E
:10D82800A02FBB27E22FF0E00E94C4793396FA9329
:10D83800EA930895ED5FF0E0FA93EA930895E22FF2
:10D84800E450F0E0FA93EA93E52FE450F0E0FA931D
:10D85800EA93E32FE058EA9301CFE3E1FDE0FA937E
:10D86800EA930E9455644E2F0895E0E0EC93AE8150
:10D87800BF810895E1E0E0930806E2E0E09309063D
:10D888000895E52FF0E00895EA1BABEDB8E0F0E06D
:10D898000E9476790895A0E021FCA1E0A1300895C6
:10D8A800E1E6F0E0FA93EA93EAE4F0E0FA93EA9327
:10D8B800ECE1F0E0FA93EA930895E981F0E0089545
:10D8C800EE0FFF1FEA5CFD4F0E94737A0895A4E3F0
:10D8D800B2E0F0E0EE0FFF1FEA0FFB1F0E94737A21
:10D8E8000895DB01AE1BBF0BE2E0F0E00E94877AEF
:10D8F800EA1B0895FA93EA93E4E1F0E0FA93EA93D5
:10D908000895E12FF0E00895E1E0F0E0FA93EA935A
:10D918000895E3E0F0E0FA93EA930895FA93EA931E
:10D928000C9417510E94737AFA93EA930895EA8146
:10D93800F0E00895EC81F0E00895ABE0EA9FF00193
:10D94800E752F84F0895FA93EA93DBCFE4E6F0E064
:10D95800FA93EA930895E150ADE0EA9FF001089543
:10D96800ED5FFA4FDF010E94647A0895FA93EA9313
:10D978000E946D510C944A51EA930E94E519E3E123
:10D98800FDE0FA93EA93EAE0EA930E942E5166CE0C
:10D99800E12FEF5FF0E00895E6E0F0E0FA93EA9314
:10D9A800F7CFFA93EA930C946D51EE0FFF1FAE0F69
:10D9B800BF1F0E94647A0895FA93EA930C94EB616E
:10D9C8000E9486790E94777A0895E4E1F0E0FA935C
:10D9D800EA930895FA93EA9350CEF0E0EDCFE2E0AF
:10D9E800F0E0DFCFE0916807F09169070895E091D2
:10D9F8006407F09165070895AE0FBF1FE3E0F0E0FC
:10DA08000E94EF790895FA93EA931A930A930C9473
:10DA18004D12FA93EA933A932A930C944D12A091DB
:10DA28006C07B0916D070895A0916E07B0916F07CC
:10DA38000895A0E0B0E00E948E7A08950E94877A47
:10DA4800EA1BFB0B0E9486790895A2E0B0E00E94D1
:10DA58008E7A08950E9486790E94197A0895A4E022
:10DA6800B0E00E948E7A0895EC83FD836E837F83F5
:10DA7800AC81BD818E819F810895A6E0B0E00E94AF
:10DA88008E7A0895E0E9F1E0FA93EA930C944979E3
:10DA9800E6E3F0E0FA93EA930895E2E0E0930806FB
:10DAA800E09309060895EA930E94005140CEEAE007
:10DAB800EA930E946E61E0916C07F0916D070895FA
:10DAC800E8E1F0E0FA93EA93E8E2F0E083CFE6E4F5
:10DAD800F0E0FA93EA930895E8E8F0E0FA93EA931D
:10DAE800D7CFEAE0EA930E946E61E0916E07F09169
:10DAF8006F070895E8E2F0E0FA93EA930895E2E305
:10DB0800F0E0FA93EA930895FA93EA930C94865115
:10DB1800FA93EA931BCFE8ECF0E0FA93EA930C94BB
:10DB28004979EFEFEA27F0E0E0930B08F0930C084F
:10DB38000895EB81F0E0E753F24F08950A921A92A4
:10DB4800FA926A937A938A939A93AA93BA93EA93E6
:10DB5800FA93EFB7EA931A930895ED91FD913196F0
:10DB6800FE93EE930895E4EFF1E0FA93EA930895B3
:10DB7800ADE01A9FF001E050FB4FE08108951A9341
:10DB8800E1E0EA930C94F651ADE01A9FF001DF0151
:10DB9800E050FB4FE081E0300895E2E0EA930C9416
:10DBA800F651E091B109F091B2096091B309709111
:10DBB800B4090E94777A0895E091A909E150ACE28E
:10DBC800B8E0F0E00E947679AE0FBF1F0E94687A35
:10DBD8000895ECE3FDE0FA93EA930895EAE0EA9306
:10DBE8000C942E51E091AA09EA93E091A709EA93CF
:10DBF8000E94081CA091A70DB091A80D1097089538
:10DC0800A091A90DB091AA0D8091AB0D9091AC0D8A
:10DC18000E94407C0895E091A70DF091A80D089509
:10DC2800E0E2EA930C940051E091A90DF091AA0D5D
:10DC38006091AB0D7091AC0D0895E091A709EF5F6D
:10DC4800E093A7090895EF5F0E94A67AE150EAE001
:10DC5800F0E0FA93EA930C944979E0919B09ABE0E0
:10DC6800EA9FF0010895A083EBE9F9E0FA93EA93BB
:10DC78000C94B434E5E0F0E094CEE1E0EA930E943D
:10DC8800290E3DCF0E944979E0E0EA930C94290ED1
:10DC9800FA93EA930C944979E1E0F0E054CDA9E0D5
:10DCA800B0E00E94927A0895E1E0EA930E94290E7A
:10DCB80078CDAEE0B0E00E94927A08951A93E0EA37
:10DCC800EA9335CEE054F14FFA93EA930E94BD6689
:10DCD8001E2F0895E054F14FFA93EA931A930C9487
:10DCE800EB66EA930E946D66E0300895E0EAEA93F5
:10DCF800EEE5F0E0FA93EA93E0E0FFE0FA93EA93C6
:10DD0800E7E4FDE00895FA93EA93E0E2EA930C94DD
:10DD18007667E0EAEA93E981FA81E050FE4EFA93E9
:10DD2800EA930895A8E2B0E00E94C4790895E0EA71
:10DD3800EA93E2E0F0E0FA93EA931A930A930895DB
:10DD4800FA93EA930C940C67A0914A0DE0914B0D5D
:10DD5800EA9FF0010895FA93EA930C94BD66E3E113
:10DD6800FDE0FA93EA930895EDE2EA93EAE0F0E041
:10DD7800FA93EA930E948E68E0E008951A930A9352
:10DD8800D6CDABE0B0E00E94C479E050F24F8F01ED
:10DD9800AA81AA300895E0EAEA93EBE0F0E0FA936A
:10DDA800EA931A930A93EBE3FDE00895EE0FFF1F41
:10DDB800E050F04F8F01AA81A0380895E150F0E0BB
:10DDC80008950E947679E058F14F8F01AA81A13019
:10DDD8000895E8EBFDE0FA93EA93E0E0EA93DCCCFF
:10DDE800E5EAFDE0FA93EA93E0E0EA93E8E0F0E0A0
:10DDF800FA93EA930C948E680E9476790E9472795D
:10DE0800DF01EA85F0E0AE0FBF1FE8E0F0E00E9416
:10DE1800C479E050FA4E8F01E0EAEA93E8E0F0E0D6
:10DE2800FA93EA931A930A93E5EAFDE089CFAE8163
:10DE3800BF81888599850E945979EE83FF83688719
:10DE4800798708954093A70D5093A80DEE81FF811F
:10DE580068857985E093A90DF093AA0D6093AB0DC1
:10DE68007093AC0D0895E8E0F0E0FA93EA93089512
:10DE7800EA930E94E5190C94F720E0911E0DF091A9
:10DE88001F0D0895FA93EA930C948819ED81EA938B
:10DE9800ED81EA930895E091350DF091360D0E94D9
:10DEA80086790895F0E0A4E6B0E00E94C479089568
:10DEB800E091AF09F091B0090895E093B00DF093A7
:10DEC800B10D0C94651DECE2F8E0FA93EA93E0E0FA
:10DED800EA930895FA93EA930C948E68E0E0F0E0F0
:10DEE80060E070E00895E093B109F093B20960939F
:10DEF800B3097093B4090895E091200DACE2B8E03D
:10DF0800F0E00E9476790895AE0FBF1F0E94687AEC
:10DF18000895E850F84FE081E1300895FA93EA93C4
:10DF2800E091AA09E05DEA930895EA930E94223EEF
:10DF3800E1300895E4ECF9E0E093E80CF093E90CA3
:10DF48000895E12FACE2B8E0F0E00E9476790895F8
:10DF58000E947E68A881AF5FEAE00E94CE79E05D0A
:10DF68000895A881AF5FEAE00E941E7AE05D0895F7
:10DF7800FA93EA93E0E0EA9308950E947479E854EA
:10DF8800FF4F32960E94737A08950E947479E8547C
:10DF9800FF4F08953696E491D901EC930895E881EE
:10DFA800F0E0A5E0B0E00E94C4790895E0EAEA93C1
:10DFB800E5E0F0E0FA93EA930895EA930E945A1D87
:10DFC800FA93EA93EDEAFDE00895FA93EA93EFEF06
:10DFD800EA93E5E0F0E07ECFE093AE0DF093AF0D6D
:10DFE80008950E94877AEA1BFB0B0895E2EBFDE097
:10DFF800ECCFA091B30DB091B40D0895E0E0E0939B
:10E00800C10DE093C20D0895A091B50DB091B60D64
:10E018000895E091B50DF091B60DAC81BD81EA0F80
:10E02800FB1F0895E093B50DF093B60D08951A936C
:10E038000E94F01D1E2F0895E093B30DF093B40DC8
:10E048000895FA93EA930E943268E0300895ABE0AD
:10E058001A9FF001E952F84F08951A930E94DB1FA6
:10E06800D3CFE091B30DF091B40D0895EA930E94D7
:10E07800DB1F0E94781FE0300895EB81EA930E942D
:10E08800171EFA93EA93E2EBFDE008951A930A93B8
:10E09800A091A2090895E0E0E093DE0DE093DD0D84
:10E0A8000895E0E0F0E0ED93FC930895EA81D8014B
:10E0B800EC93EBE9F9E0FA93EA930E94B4341981FE
:10E0C80008810895E12FACE8B0E0F0E0EE0FFF1F03
:10E0D800EA0FFB1F0E94737A0895A3E21A9FF001CA
:10E0E800DF01E45DF74FE081E0300895E981ADE0BC
:10E0F800EA9FF0010895E65FFA4FA1E0A083089532
:10E10800ACE8B0E0F0E0EE0FFF1FEA0FFB1F0E9443
:10E11800737A0895A0919F09B091A009EA2BFB2B6F
:10E12800E0939F09F093A0090895E150A7E1EA9FC1
:10E13800F0010895A7E10A9FF001EC5EF74FAF01E7
:10E148000895E45FFA4FBF01E0810895E881F0E0A7
:10E15800E45DF74F0895E981FA81FA93EA93089507
:10E16800A3E2BDE0E091A309F0E00895A6E2BDE0D6
:10E17800E091A309F0E0AE0FBF1F0895A9E2BDE04A
:10E18800E091A309F0E0AE0FBF1F0895EE0FFF1F47
:10E19800AE0FBF1F0895ACEAB8E073CBEE0FFF1FB8
:10E1A800EA0FFB1F0895E081F0E00895A7E11A9FA8
:10E1B800F001EC5EF74FEE83FF83AE81BF810895D7
:10E1C800EE81FF81A481AA930C944D210D901C909F
:10E1D800AE81BF811296EC91F0E0E00DF11DDB01FC
:10E1E800ED93FC930895ED91FD913197FE93EE9395
:10E1F80008950E94E522EF770E2EAA85BB85129618
:10E20800EC91E0150895A3E20A9FF001EF5CF74F47
:10E218000895BD01AAE0B0E00E949C79E60FF71FBF
:10E22800E887F987A1810895EE59F64FEC87FD87B5
:10E23800AC85BD85119608951296EC91AC85BD8587
:10E248001696EC930895D001F0E00895A885B98555
:10E2580018960E94647A0895AC85BD85EC93EBE925
:10E26800F9E0FA93EA930C94B434E885F985A2812D
:10E27800AA930895EA85FB85FA93EA930E942E21D2
:10E28800E0300895AA85BB85EC91EA93E3E0EA9330
:10E298000C949463AA85BB85E0E0EC93E2E0E093FC
:10E2A80009080895BF0100801180AE81BF811296D0
:10E2B800EC910895DB01ED93FC93AE81BF8112963A
:10E2C800D4CAE4E6F0E00E94C4790895F0E0ED9342
:10E2D800FC930895EBE9F9E0FA93EA930C94B434CB
:10E2E800E091A209A091A109EA170895F0E0E00DD4
:10E2F800F11D0895ACE2BDE004CBA6E2BDE0EE2737
:10E30800A10FBE1FEC910895A9E2BDE0EE27A10F71
:10E31800BE1FEC910895BD01AAE0B0E00E949C796F
:10E32800DB010895E081EA930C949C38E8ECFBE06B
:10E33800E093E60CF093E70C0895EA930E94F03C12
:10E34800E0E00895EA930E94F03C0C945E3EBD0123
:10E35800AAE0B0E00E949C79E60FF71F0895A6E2B4
:10E36800BDE0EE27A00FBE1FEC910895A9E2BDE025
:10E37800EE27A00FBE1FEC910895A3E2BDE0EE27A3
:10E38800A00FBE1FEC91E1700895ACE2BDE001CA98
:10E39800A9E3BDE0EE27A00FBE1FEC910895A2E30C
:10E3A800BDE0EE27A00FBE1FEC910895EA81ADE015
:10E3B800EA9FF001E65FFA4FA0E0A083EA81EA93C2
:10E3C8000895ABE00A9FF001E952F84F0895ABE0D9
:10E3D8000A9FF001E352F84F0895FA93EA930C94D8
:10E3E8004336FA93EA930E9415643A93D6CBE091A8
:10E3F800B50DF091B60D30970895AFEFBFEFA0833C
:10E40800B18308950E942668E093E30DF093E40D2C
:10E418000895F0E0C6CAFA93EA93E0E0F0E80895B8
:10E42800E091350DF091360D0895EE59F64FFA93B7
:10E43800EA930E94162A4ECFE0919909ABE0EA9F31
:10E44800F0010895E9E9F9E0FA93EA930C94B434F9
:10E45800FA93EA930C948C45E88DABE0EA9FF001BF
:10E468000895E0E1EA93E0910A08EA930E94B81956
:10E478001E2F08951DDDFA93EA930895FA93EA93FF
:10E488000C94A61FE0930A08E0E0E093E00DE1E3B6
:10E49800E093E10D0E94572B0C942727FA93EA93F7
:10E4A8000C94023DE9ECFAE0E093E80CF093E90CF7
:10E4B800E3E0EA930C94963CA091E80CB091E90C47
:10E4C80008950E942668E093D80DF093D90D089519
:10E4D800E093E80CF093E90C0895E3E0EA930C94D8
:10E4E800963CE093AF09F093B00908950E949251C9
:10E4F800E0E0EA930C94370FE0E0F0E0E093AD0938
:10E50800F093AE09E1E0E09309060895E0910E0664
:10E51800E550F0E005C9E091AD09F091AE094CCAAB
:10E52800E0915807F09159070895FA93EA930C94EB
:10E538006050A0E024FCA1E0A0300895E7E0EA9351
:10E54800E0E0EA938BC80E942668E093BB09F09349
:10E55800BC090895E0E0E093DD0D08950E946D5137
:10E568000C944A51EF5CEA930C940051ACE6B8E085
:10E57800F7C8ACE2BDE0E091A309F0E00FCEACEA49
:10E58800B8E0EEC8AE0FBF1FEC91E160D001EC938C
:10E598000895E091A209EA93E0E0EA930C94CB2C69
:10E5A800EA930E946E610E94A9631E2F0895EAE211
:10E5B800EA93EBEDF9E1DCCC0E945F2DE1E0EA9310
:10E5C8000C94472D1F771A930C94E519A091AD0967
:10E5D800B091AE090895E8EEF3E00E94217A08951B
:10E5E800E053F0E00895F2DFEA17FB070895E0939F
:10E5F800A109E0E0E093B80908950E94003E0E9456
:10E60800812EE093AC0908950E94E5190C9492516B
:10E618000E94C8290E94BA200E94A663E03008958B
:10E628000E94A9631E2F1A930E94B42E10380895D1
:10E638001A93E091C107EA930895E091120DEA93C5
:10E648000E94EE18E03008950E942668E093E50DD8
:10E65800F093E60D0895D90118960E94647A0895FA
:10E66800E4E6F0E060E070E00E94197A08950E9404
:10E67800E51903CC0A93E091C107EA930895E09164
:10E68800B709EA930A930C94251B0E94647AFA93BB
:10E69800EA930895A8EEBCE060CAE091C409E0538B
:10E6A800E093AA090895FA93EA93E0E3EA930C94B5
:10E6B800003EE091C109EA930C94AC3D0E94703D84
:10E6C800EBE3EA930C94F03CE89423F8E0E0F0E004
:10E6D80008DFE0E0E093A7090A93E1E0EA930C94ED
:10E6E800CB2CE89423F8E0E0F0E0FBDEE0E0E093F8
:10E6F800A709EA930C94472DA881B981EC91EF5FA3
:10E70800EC930895ABE00A9FF001E852F84F0895A2
:10E71800A083ABE00A9FF0010895ABE00A9FF001E7
:10E72800E652F84F0895FA93EA93E2E0FAE1FA9391
:10E73800EA93EA85ABE0EA9FF0010895FF27662790
:10E7480077270E94777A84E00E94686A289608955D
:10E75800AC81BD81EE27A00FBE1F0895E02FAC81CC
:10E76800BD81F0E0EA0FFB1F089584E00E94686A0B
:10E7780028960895EE27A30FBE1FEC91D001EC93C5
:10E788000895ABEDB8E00C94B46B0E947679EA0F6B
:10E79800FB1FAF010895E091B50DF091B60D0895F6
:10E7A800E32FA091A709EA0F0895ADE02A9FF00191
:10E7B800E85FFA4F0895E091210DE295EF70089512
:10E7C800A8E0B0E00E94927A0895AA81BB81EC91FA
:10E7D800E295E07FAE2FEC810895EA0FAA81BB8114
:10E7E800EC938ACFE0918A0EA091890EEA170895DA
:10E7F800E091C30AF0E0E853F54F08951083E091E3
:10E80800C30AEF5FE093C30AE12FA091C50A0895F8
:10E81800E093C50AE091C40AE150E093C40AE030ED
:10E828000895E853F54FA0E0A0830895E091550FAF
:10E83800F091560F0895A091530FB091540FEA1715
:10E84800FB070895E12FA0915A0FEA0FE0935A0FA2
:10E85800E0915C0F0895F0E0E054F64F10830895BE
:10E86800E0916110F0E0E05AF04FE081E0939C0005
:10E87800E0916110EF5FE093611008951DDEAC91A7
:10E88800A032089519DEAC91AB330895EA930E9443
:10E898009C3BE1300895F0E0AE17BF070895EAE029
:10E8A800F0E00E94C479089507DEAC91A033089582
:10E8B80003DEAC91AA330895E091E80CF091E90CDD
:10E8C800E1810895F9DDEC91EA930C94FE670F015C
:10E8D800F3DDEC91E0530ACDE2E2EA930E949C3B1F
:10E8E800E0300895E453F34F0F01E6DDEC91D001D9
:10E8F800EC931F5FCFCEE453F34FA0E0A0830895BD
:10E90800A091E60CB091E70C0895EC93A6EEBCE05C
:10E9180024C9E12FA981BA81F0E0EA0FFB1FE49135
:10E928000895EA930E94F03C1F5F0895A981BA8177
:10E93800EE27A10FBE1FEC9108956497FE01FA938C
:10E94800EA930895E6E0FAE1FA93EA930895FE015E
:10E95800FA93EA930C940F3DFE013196FA93EA93E9
:10E9680008950E94777A01CFE2E2EA930C94F03C92
:10E97800E881F981FA93EA930895FA93EA930C945B
:10E988001C3DFA93EA93E2E0EA930895E881EA935A
:10E998000C94F03CE05DEA930C94F03CE881F9813A
:10E9A8006A817B810E94777A0895E985FA85FA93CE
:10E9B800EA9308953A932A935A934A930895E85309
:10E9C800F44FE081E0300895E853F44FABCCEA937C
:10E9D8000E941568EA930C949C38EA930E94113FB0
:10E9E800EAE5E093C60A0895E091C00DA091BF0D35
:10E9F800EA170895E0919A09ABE0EA9FF0010895BB
:10EA0800E3E0EA930E94533DF5CFA091AE0DB0919B
:10EA1800AF0D0895F0E0FA93EA930895E2E5EA93DA
:10EA28000E94F03C0C946C40F096EA930E94AC3D36
:10EA3800E2E7EA930C94F03CEA930E94F03CEEE0A3
:10EA4800EA930C94F03CE6E1FAE128CDEBE3EA9393
:10EA58000C94F03C5A934A930E9488190E2F003464
:10EA68000895FA93EA930C94B434E0E0EA930C9492
:10EA7800326BEC59F64FA885B985A083B183EDC8F0
:10EA8800E2E5EA930C94F03C1A93E091C109E05353
:10EA98001E2FE5ECF9E01CCDE0919B09A0919C09A3
:10EAA800EA170895ECE9F9E0DCCFF0E066CFE091F1
:10EAB8009C09ABE0EA9FF0010895A091FD0CAF5FBF
:10EAC800EAE00E941E7AE093FD0CEAE2EA930E94D3
:10EAD800AC3DD6CFE091FD0CE05AAECFD9011696E9
:10EAE800EC91E3CFF901A281B381BA93AA930C9474
:10EAF8001C3DEAE3EA930C94F03CF901A085B1854A
:10EB0800BA93AA930C941C3DD9011196E0E0EC93BA
:10EB18000E94C73DC7CFD901EC91C7CFE05DEA930A
:10EB28000E94AC3DADCFE250F34FE08133CFEEE031
:10EB3800EA930C94F03C0E94C73D0E942668E0933B
:10EB48006210F0936310E2E0E093BE09D9011196D8
:10EB5800EC930895EA930E94AC3D92CFE091A20D08
:10EB6800DDCFE091A20DF0E0DECF0E941C3DECE28B
:10EB7800EA930E94F03CFCCEC3DEE0E0EC930895FB
:10EB8800EE81FF81E093B00DF093B10D1093AD0DC0
:10EB98000E94651DE1E3089541E050E00E94223C97
:10EBA800E887F987EAE372CEFA93EA935A934A938D
:10EBB80008950E94223C3197E887F987E8850895EF
:10EBC800EAE3EA930E949C3BE0300895E091C80C88
:10EBD800F0E0E45DF74F0895E0E0E0936710E0931C
:10EBE800681008950E94223C3197E093C80CE09188
:10EBF800E10CA091C80CEA1708950E945949E091C8
:10EC0800C80CEA930895ECE2EA930E949C3BE0303A
:10EC18000895E02FA0E0B2E0F0E00E947679EA0FD4
:10EC2800FB1F0895A6E2BDE0E091C90CF0E008954D
:10EC3800A9E2BDE0E091C90CF0E00895E091C90CAB
:10EC4800EF5FE093C90C0895A2E3BDE0E091C90C21
:10EC5800F0E00895A9E3BDE0E091C90CF0E0089563
:10EC6800ACE2BDE0E091C90CF0E098CAA3E2BDE0D7
:10EC7800E091C90CF0E00895E091C90CF0E0089526
:10EC8800EE27A10FBE1FEC910895E091C80CF0E0AB
:10EC98007CC9E091C80CF0E070C9ECECFCE0FA9398
:10ECA800EA930C947E3DFA93EA930C94BC45ECE20B
:10ECB800EA930C94F03C0E94B145E0E0E093C90C63
:10ECC8000895AE0FBF1FEC91E1700895AE0FBF1FFE
:10ECD800EC91EBCEE091E80CF091E90C0895E0E0BE
:10ECE800EA930E941746E093BD0908951A930A9380
:10ECF8003A932A930895FA93EA93E09109060895BE
:10ED0800A091C50DB091C60D0895E091C50DF09183
:10ED1800C60DFA93EA93E091C70DF091C80DFA93E6
:10ED2800EA930895F0E0EA0FFB1F0895E093C50DFC
:10ED3800F093C60D0895E0935807F0935907089586
:10ED4800F801AA81BB81EA0FFB1FE4910895AE0F79
:10ED5800BF1FAC91A0300895AE0FBF1FEC91EA938E
:10ED68000895A0910906E4E1EA9FF0012E2F3327C8
:10ED7800CCCFECE0EA9FF001A0910806EA9FF001F1
:10ED880008951A93E1E0E0930906E093080610E07D
:10ED98000895FE013696FA93EA93EBA1EF7308956E
:10EDA800FA93EA930C94AE68FA93EA930C94C468C5
:10EDB800EA9FF001F0E00895EAA5FBA5FA93EA932B
:10EDC8000895EAA5FBA5E20FF31F0895ECA1EA93C5
:10EDD8000C94D8553A932A93EEA1FFA1E40FF51F9E
:10EDE8000895FA93EA93EDCFFA93EA93EAA5FBA57F
:10EDF800E40FF51FFA93EA93E9CFFA93EA93E6CF83
:10EE0800EA9FF001AEA1BFA1F0E00895E2E0E0932F
:10EE18000906E0E2F0E0EAA3FBA30895E2E0F0E0EF
:10EE28000E94EF790895AE1BBF0BF8CFEE8DF0E08E
:10EE3800E20FF31F08953196FA93EA93ECA1FDA12E
:10EE4800E40FF51F31960C94886DFA93EA93ECA1C0
:10EE5800FDA1E40FF51F0C94886DE9A1F0E0DE0137
:10EE680016960895ED8DEA930E94BC50E9A1EF5FD4
:10EE7800E9A30895E40FF51FDF01ECA1FDA18EC9F8
:10EE88000E94C4790E9486790E941D7B0895AE85F0
:10EE9800BF85888999890895EE83FF836887798774
:10EEA80008950E94817A0E94507B0895E98DFA8D19
:10EEB800E21BF30BFA93EA930895FA93EA93F901A4
:10EEC800AD8DBE8DEA0FFB1FFA93EA930895FA936E
:10EED800EA93EA8DEA930C94D855E7E1EA93E1E0E6
:10EEE800EA930C94E454EA93E7E7EA930C94E45425
:10EEF800ACECB4E0F0E052C9EA93ED85EA930C94E7
:10EF0800E454E985FA85AD85BE850895EA930E94A3
:10EF1800E454E8E10895EA93E0E0EA930C94E454B9
:10EF2800EA93EC85EA930E94E4540C94FE540E9400
:10EF380014630C94E162F0E00E94767908950E94CF
:10EF4800777A0E94FE620C94E1620E941463E5EEF7
:10EF5800FAE10C94BC6F0E94E1620C94E16220E03B
:10EF680030E0E12FE05DEA93E8EEFAE10C94926F6D
:10EF78001091580700915A070895D2DA31970C94E6
:10EF8800DA6B0E94A9633E2F0C94AF50DF01EE2785
:10EF9800A30FBE1F0895A3E2BDE00C949E6C0E94CF
:10EFA8009251E1E0EA930C94370F0E943B0E0C94C7
:10EFB800326BFA93EA93E091A40DEA930E940F59F9
:10EFC800E1320895FA93EA93E3E6EA930E94B75888
:10EFD800E1320895E6E0F0E00C94946BEA0FFB1F31
:10EFE800FA93EA93E0E1EA930E94B758E132089570
:10EFF8000E946D51A3E2BDE043CE0E946D51E12F06
:10F00800EF5FEA930E940962EAE3EA930E940051E3
:10F018000C94B36EE7E0F0E0FA93EA930895EF5F9B
:10F02800EA930C940962E3E7EA930C940051EA230B
:10F03800EA930E940F620C94146EEAE3EA930C942C
:10F048000051E8E0F0E00C94946BEA930E94B75802
:10F05800E1320895EA930E940F620C94146EDF0166
:10F0680032960C94966C0E946D510C94CD6BEEE820
:10F07800F5E1E093C30DF093C40D08950E948C1B35
:10F08800E0E0E093A9090E9461160E943B0EE1E0CE
:10F09800E093A40908950E9492510E948A100E9448
:10F0A800A9630E2F0D330895EAE2EA93E0E9FBE144
:10F0B8000895EA930E94B1160C943B0EE6E3F6E13C
:10F0C800E093BC07F093BD070895E093BC07F09365
:10F0D800BD070895FE01FA93EA930895E8EAFBE173
:10F0E800FA93EA93EE85FF85688979893ACCECEA48
:10F0F800FBE1FA93EA93CBDEB3CA0E94777AAA8936
:10F10800BB898C899D89E4E6F0E060E070E00E94AC
:10F118002F7A0E94777A88E00E94686A2C96089570
:10F12800E5EBFBE1FA93EA93EE85FF850C94E46C3A
:10F13800EA930E947C621F5F0895E091BF07A2ECEA
:10F14800B7E0F0E00895E091BE07A2ECB7E0F0E088
:10F158000C94D270AC81BD81EE27A30FBE1FAC9179
:10F16800A0300895ABE00A9FF001E15FF94F0895E0
:10F17800EA0FFB1F0F01AC81BD81FCCAA5E10A9F04
:10F18800F001E551F94F0895EE81FF810180128069
:10F19800AE81BF8115960E94647AD0010895FA93D2
:10F1A800EA93FE013A96FCCDE091BC07F091BD07C9
:10F1B8000895ACEBB7E0ED91FD913296FE93EE9396
:10F1C8000895AE81BF81EA17FB070895E0E0E09358
:10F1D8006007E09361070895EA930E94A266E03011
:10F1E8000895E0917100E87F1E2F0895E093730061
:10F1F800E4E8F2CF0A930E947966E0300895FF2789
:10F20800662777270E941D7B0895EE8D40DEF7DF85
:10F218000E94A57BA9A1BAA1882799270E947E7A76
:10F2280040CE2A93EF85F889FA93EA930C94EF6B12
:10F23800E889F9893497E88BF98B0895EF85F8897F
:10F24800FA93EA930C94EF6BA889B98914960E94F3
:10F25800647AEE83FF830895A889B98914960E9479
:10F26800647AEA87FB8708950E94A66AE883F9838F
:10F278006A837B830895E881F9816A817B81089597
:10F28800EA81FB816C817D810895E991F99130963D
:10F2980039F080ED97E00197F1F7A8953197C9F714
:10F2A80008950024AF0DB01D0895EA0FFB1F681FD5
:10F2B800791F0895F195E195F0400895F0956095CE
:10F2C8007095E195FF4F6F4F7F4F0895EE230E2EF7
:10F2D800EA2F19F0EE0F0A94E9F70895EE0FFF1FD1
:10F2E800EE0FFF1FEE0FFF1FEE0FFF1F0895EF2F0A
:10F2F800FF27E7FDFFEF0895FE2FFF0FFF0B6F2F8E
:10F308007F2F08956F2F660F660B762F0895BA2FFB
:10F31800BB0FBB0B8B2F9B2F08958B2F880F880B50
:10F32800982F0895EA17FB07E1E00CF0EE270895FF
:10F33800FA9FF02DEB9FF00DEA9FE02DF10D089557
:10F348007A9F702D6B9F700DF89F700DE99F700D5F
:10F358006A9F602D710DFB9F600D711DE89F600D08
:10F36800711D8827FA9FF02D610D781FEB9FF00D16
:10F37800611D781FEA9FE02DF10D681F781F089521
:10F388007ED0D6DF0EF496DF089587D0D9DF0EF44D
:10F3980095DF0895002498E0AA0F001C0E1A10F4B7
:10F3A8000E0E01C0A1609A95B9F7EA2FA02D089515
:10F3B8000024112490E1AA0FBB1F001C111C0E1A77
:10F3C8001F0A18F40E0E1F1E01C0A1609A9599F726
:10F3D800FD01D001089553D0EBDF0EF46BDF0895E3
:10F3E8003F934F935F93002411244427552730E21D
:10F3F800AA0FBB1F881F991F001C111C441F551FF3
:10F408000E1A1F0A460B570B28F40E0E1F1E461F16
:10F41800571F01C0A1603A9559F7FD01BC01D00101
:10F42800CA015F914F913F91089537D0D9DF0EF40B
:10F4380045DF0895AFDFEA2F0895E894B7FF04C0C9
:10F44800A095B09511966894F7FD34DFB1DFFD0102
:10F458000EF430DF0895E89497FF09C0A095B095A1
:10F4680080959095AF5FBF4F8F4F9F4F689477FD02
:10F4780025DFB6DFFD01BC010EF420DF0895E89416
:10F48800F7FF02C017DF6894B7FF06C0A095B095D4
:10F49800119600F8039400FA0895E89477FF02C0E3
:10F4A8000DDF689497FF0BC00024A095B095809558
:10F4B80090951196801D901D00F8039400FA089508
:10F4C800ED91FC9111970895ED91FD916D917C91CD
:10F4D80013970895ED93FD936D937C93089505908C
:10F4E800F491E02D08957A936A93FA93EA93089534
:10F4F800689401C0E89401D09DD0182E862F612D04
:10F50800192E972F712D1B2EBF2FF12D1A2EAE2FCE
:10F51800E12D0895119602D0FE2F1197E199FECFA3
:10F52800FF93FFB7F894AEBBBFBBE09AEDB3FFBF44
:10F53800FF91089507D01196EF93EF2F03D0EF9125
:10F5480011970895E19B02C0A895FCCF9FB7F89446
:10F55800AEBBBFBBE09A8DB3E81719F0EDBBE29ADA
:10F56800E19A9FBF0895552342F4503811F4E0FF03
:10F5780004C03196691F791F6BF050E8572711F4C2
:10F588005F93CDC05F3F31F0660F000C57956795CC
:10F59800752F08955F9300200AF0CDC0C6C050E8CB
:10F5A800192E1522880F991F9527550F879550E812
:10F5B800072E0522660F771F7527550F6795089543
:10F5C800689401C0E8945F93F2DF703818F07F3FC9
:10F5D80008F4A5C056E1571BAAF4519558300EF40B
:10F5E800593030F0EFEFFFEF6FEF7FE777F91AC090
:10F5F80077275523B9F0EE0FFF1F661F771F5A951F
:10F60800D1F710C07727583028F0EF2FF62F672F43
:10F618005850F9CF552331F076956795F795E795CA
:10F628005A95D1F700200AF449DE5F91089568944D
:10F6380001C0E894309760407040B1F0002426F093
:10F64800772312F400943ADE172E7EE1112032F06F
:10F658007A95EE0FFF1F661F111CF9CFEF2FF62FBB
:10F66800612D5F938ADF5F9108954F93AF01FD018C
:10F67800DA01AB01BC01CA01402D012C142E4F91B7
:10F688000895EA0FFB1F681F0895E095F0956095AF
:10F69800EF5FFF4F6F4F08955F9381DF903871F1EF
:10F6A80050E8152604C05F937ADF903839F1703836
:10F6B80021F1572F591B13F112F4D7DFFACF583124
:10F6C80018F0AA27BB278827583028F0AB2FB82F67
:10F6D80088275850F9CF552329F08695B795A795CF
:10F6E8005A95D9F7502D512562F0CBDF38F467953C
:10F6F800F795E795739513F41EC0B7DF3EDF5F916A
:10F708000895EA1BFB0B680B51F010F40094BDDF61
:10F718006623A2F3EE0FFF1F661F7A95CBF7EE273D
:10F72800FF27662777275F910895EFEFFFEF6FE7D1
:10F738007FEF5F910895EFEFFFEF6FE77FE75F914E
:10F7480008955F932CDF703851F3903841F301240A
:10F758000894791F23F41CF300203AF3ECCF0F929E
:10F768001F932F933F934F93112722279927689F21
:10F77800A0018F9F302D410D591F6B9F300D411DEA
:10F78800591F8E9F27D0BF9F25D06A9F23D0BE9F29
:10F798001DD0AF9F1BD0AE9F110D291F391F491FC8
:10F7A800591FE32FF42F652F522F4F913F912F911F
:10F7B8001F910F9066232AF0550FEE1FFF1F661F3B
:10F7C80002C073954BF2CFDE5F910895100D211D95
:10F7D800391F02C0200D311D491F591F08955F931D
:10F7E800DEDE703821F411200AF49FCFA4CF9038C0
:10F7F80009F495CF01240894970B1BF4D4F3002047
:10F80800F3CF792F1F932F933F934F9311241127F1
:10F81800222733274427552790E2AE17BF078607CC
:10F82800410730F0AE1BBF0B860B410B089401C09B
:10F838008894551F221F331F111CAA1FBB1F881F26
:10F84800441F9A9551F7F901612D4F913F912F91DE
:10F858001F91662332F0550FEE1FFF1F661F7A9522
:10F8680043F281DE5F9108953097604070400895BB
:10F8780000240A160B06089500240A160B0608062B
:10F88800090608955A934A933A932A931A930A9326
:10F8980008955D814C813B812A81198108810895F1
:00000001FF
